:100000000C94681A0C94991A0C94991A0C94991AD5
:100010000C94991A0C94991A0C94991A0C94991A94
:100020000C94991A0C94991A0C94991A0C94991A84
:100030000C94991A0C94991A0C94991A0C94991A74
:100040000C94991A0C9446D10C94991A0C94991A00
:100050000C94991A0C94991A0C9443BE0C94E3A92D
:100060000C94991A0C9417560C940D560C94991ADA
:100070000C94991A0C94991A0C94991A0C94991A34
:100080000C94F0330C94991A0C94991A0C94991AB4
:100090000C94991A0C94991A0C94991A0C94991A14
:1000A0000C94991A0C94991A0C94C2330C94991AC2
:1000B0000C94991A0C94991A0C94991A0C94991AF4
:1000C0000C94991A0C94991A0C94991A0C940B3755
:1000D0000C94D5360C94991A0C94991A0C94991A7C
:1000E0000C94991A084AD73B3BCE016E84BCBFFDE5
:1000F000C12F3D6C74319ABD56833DDA3D00C77FF8
:1001000011BED9E4BB4C3E916BAAAABE0000008090
:100110003F05A84CCDB2D44EB93836A9020C50B91F
:10012000918688083CA6AAAA2ABE000000803F004B
:100130000C94B8FC0D94A20B0C94EDFC0D94AB1038
:100140000C949CFC0C941EFC0C94DAA70C94B0FC50
:100150000C9487370C94C0A90C9492FC0D94770CE6
:100160000C94A9560C94F7FC0C944B440D94A90FD5
:100170000C94DEFC0D94BD0F0D94740F0C94B137EC
:100180000D943A0D0C9415FC0C943AFC0C94F7FB6E
:100190000D9482090D94241F0D94D2090C94CF372D
:1001A0000C9448FC0C94A2560C94F6A80D946F0580
:1001B0000C9453420C9488FF0D94470F0C94B55641
:1001C0000D94BC100D94CB0B0C9418FC0C94D4FC27
:1001D0000D94B8010C94C1560C94A5370D940908E0
:1001E0000C94BC370C9401FD0C94C7370D948A0C09
:1001F0000D949E090C94AD560D94061F0C9485FC2D
:100200000C9493560C9422FC0C9409FC0C94B53776
:100210000C942CFC0C94B9A70C9484560C94BD56E9
:100220000C9444FC0D94020C0C943EFC0C94493745
:100230000D946E0F0C94A1370C94F2FB0C940BFDF3
:100240000C94A9370D945F140C94B7A80C9411FC6E
:100250000C948C440C9455A40C9404420C948DFC86
:100260000C94C8560C9415FD0C949D370D94350CC8
:100270000D94DF0B0C9424A70D948E010D94770F31
:100280000C9455560C9496370C940DFC0D94340B2D
:100290000C94C0FC0C941FFD0C94DB560D942003B1
:1002A0000D946E0A0D94F1030D944F090C94AD3723
:1002B0000D94CA0F0D94FE0A0C94D3560D94160C8F
:1002C0000C941EA80C9430FC0C941F440C94CAFC93
:1002D0000C9436FC0C94D8A40C94D7A40C94A6FCD3
:1002E0000D94900F0C94C4440C94C9A80D949F0FC6
:1002F0000C9457420D94A9000C94B1560C94B95625
:100300000C9428FC0C9439A80C9441A70C947837D1
:100310000D947F114E414E494E495459494E46CD98
:10032000CCCC3D0AD7233C17B7D13877CC2B3295AC
:1003300095E6241FB14F0A000020410000C842008A
:10034000401C4620BCBE4CCA1B0E5AAEC59D740054
:10035000407A10F35A00A0724E18090010A5D4E894
:100360000000E87648170000E40B54020000CA9A27
:100370003B000000E1F50500008096980000004079
:10038000420F000000A086010000001027000000BE
:1003900000E803000000006400000000000A000004
:1003A0000000000100000000002C76D888DC674FB8
:1003B0000823DFC1DFAE59E1B1B796E5E3E453C6E8
:1003C0003AE651997696E8E6C28426EB898C9B62E0
:1003D000ED407C6FFCEFBC9C9F40F2BAA56FA5F48A
:1003E00090055A2AF75C936B6CF9676DC11BFCE0B2
:1003F000E40D47FEF520E6B500D0ED902E03009405
:100400003577050080841E080000204E0A00000099
:10041000C80C333333330F986E12831141EF8D21A3
:1004200014893BE65516CFFEE6DB18D1844B381B0A
:10043000F77C1D901DA4BBE424203284725E2281CF
:1004400000C9F124ECA1E53D27434F4D4D554E49E0
:10045000434154494F4E0044525952554E00455263
:10046000524F525300494E464F004543484F0045B6
:1004700072726F722077726974696E6720746F2070
:10048000454550524F4D210A0053544F505045445A
:100490002E20005072696E7465722073746F7070D4
:1004A00065642064756520746F206572726F727365
:1004B0002E2046697820746865206572726F7220FC
:1004C000616E6420757365204D39393920746F2051
:1004D000726573746172742E202854656D70657234
:1004E00061747572652069732072657365742E205E
:1004F0005365742069742061667465722072657337
:1005000074617274696E67290A004E6F20436865D2
:10051000636B73756D2077697468206C696E6520F4
:100520006E756D6265722C204C617374204C696E1F
:10053000653A20004E6F20436865636B73756D20CC
:1005400077697468206C696E65206E756D6265727E
:100550002C204C617374204C696E653A20006368EE
:1005600065636B73756D206D69736D617463682C61
:10057000204C617374204C696E653A20004C696EA2
:1005800065204E756D626572206973206E6F7420F0
:100590004C617374204C696E65204E756D62657296
:1005A0002B312C204C617374204C696E653A20000D
:1005B0004D3131300053657269616C207374617420
:1005C0007573206D69736D617463680A0077616982
:1005D000740A0053442072656164206572726F7200
:1005E0000A002121204B494C4C20636175736564DE
:1005F00020627920746F6F206D75636820696E6169
:1006000063746976652074696D65202D2063757249
:1006100072656E7420636F6D6D616E643A20004880
:100620006F74656E642049646C652054696D656FF4
:10063000757400486F74656E642049646C6520545D
:10064000696D656F75740A003D3D6F6E46696C613A
:100650006D656E7452756E6F75743D3D0070617599
:100660007365004D363030002066696C616D656ED3
:10067000745F72756E6F7574200066696C616D656C
:100680006E745F72756E6F757420540046696C618C
:100690006D656E7452756E6F75742054002A2A2A27
:1006A000496E6974696E67206361726420697320A2
:1006B0004F4B2A2A2A004D6564696120496E736593
:1006C00072746564004D656469612052656D6F7672
:1006D0006564004D313030305300627573793A20D3
:1006E00070617573656420666F7220696E707574D1
:1006F0000A00627573793A207061757365642066CB
:100700006F7220757365720A00627573793A207092
:10071000726F63657373696E670A002A2A2A6B69B0
:100720006C6C2A2A2A00706F7765726F6666004BC0
:10073000494C4C45442E20005072696E74657220FD
:1007400068616C7465642E206B696C6C2829206369
:10075000616C6C6564210A0053544F505045442E1F
:1007600020005072696E7465722073746F707065CA
:10077000642064756520746F206572726F72732EC9
:100780002046697820746865206572726F722061F6
:100790006E6420757365204D39393920746F20726D
:1007A0006573746172742E202854656D7065726172
:1007B000747572652069732072657365742E205399
:1007C0006574206974206166746572207265737443
:1007D000617274696E67290A006563686F3A004543
:1007E00072726F723A0042696C696E656172204C78
:1007F0006576656C696E6720477269643A0A002104
:10080000212053544F502063616C6C6564206265F5
:100810006361757365206F6620424C546F75636821
:10082000206572726F72202D20726573746172740C
:100830002077697468204D3939390A002121205305
:10084000544F502063616C6C656420626563617510
:100850007365206F6620424C546F75636820657223
:10086000726F72202D2072657374617274207769C3
:100870007468204D3939390A002F2F616374696F0C
:100880006E3A0070726F6D70745F00656E64005335
:10089000656E64204D31303820746F207265737539
:1008A0006D650A00496E736572742066696C616DCE
:1008B000656E7420616E642073656E64204D313006
:1008C000380A005265686561742066696E697368EC
:1008D00065642E0052656865617420446F6E650022
:1008E000526568656174696E672E2E2E00526568C8
:1008F000656174004865617465722054696D656F47
:1009000075740053656E64204D31303820746F204B
:1009100068656174206E6F7A7A6C650A004E6F7A32
:100920007A6C65205061726B656400486F74656E07
:100930006420746F6F20636F6C640A00706175735C
:1009400065640050617573650044697361626C652C
:1009500052756E6F75740050757267654D6F726574
:10096000005061757365640073686F770062757419
:10097000746F6E00626567696E004C6F616420463B
:10098000696C616D656E74004C6F61642046696CC2
:10099000616D656E74205400496E736572742066D3
:1009A000696C616D656E7420616E642073656E6440
:1009B000204D3130380A00726573756D65640052E0
:1009C0006573756D696E670057616974696E67203C
:1009D000666F72206865617475702E0A004C6561DF
:1009E00076696E6720473236003F537065636966EB
:1009F00069656420582C5920636F6F7264696E6159
:100A00007465206F7574206F6620626F756E6473F5
:100A10002E0A003F28522965706561742076616C4A
:100A20007565206E6F7420706C61757369626C659A
:100A30003B206D757374206265206174206C656164
:100A4000737420312E0A003F285229657065617445
:100A5000206D7573742062652073706563696669C3
:100A60006564207768656E206E6F74207573696E9B
:100A70006720616E204C43442E0A003F537065632B
:100A80006966696564206E6F7A7A6C652074656D3D
:100A90007065726174757265206E6F7420706C6120
:100AA000757369626C652E0A003F537065636966F1
:100AB0006965642066696C616D656E742073697A1E
:100AC00065206E6F7420706C61757369626C652E41
:100AD0000A003F53706563696669656420707269D6
:100AE0006D65206C656E677468206E6F7420706C25
:100AF00061757369626C652E0A003F5072696D659D
:100B0000206C656E677468206D7573742062652053
:100B1000737065636966696564207768656E206EC9
:100B20006F74207573696E6720616E204C43442E8C
:100B30000A003F537065636966696564206E6F7A69
:100B40007A6C652073697A65206E6F7420706C61B1
:100B5000757369626C652E0A003F52657472616339
:100B600074696F6E204D756C7469706C6965722064
:100B70006D7573742062652073706563696669655D
:100B8000642E0A003F53706563696669656420528C
:100B9000657472616374696F6E204D756C746970F1
:100BA0006C696572206E6F7420706C617573696218
:100BB0006C652E0A003F5370656369666965642041
:100BC0006C6179657220686569676874206E6F74FE
:100BD00020706C61757369626C652E0A0043292E62
:100BE0000A003F53706563696669656420626564E5
:100BF0002074656D7065726174757265206E6F74B6
:100C000020706C61757369626C65202834302D002A
:100C1000473236207374617274696E672E2E2E0A05
:100C2000004F46460A00466164652048656967686A
:100C3000742000426564204C6576656C696E67209F
:100C4000004661696C656420746F20656E61626C3A
:100C50006520426564204C6576656C696E670A00A4
:100C6000496E76616C6964206D6573682E0A005068
:100C7000726F62696E6720506F696E740025532031
:100C800025692F2569002E0A002F0050726F6269B6
:100C90006E67206D65736820706F696E7420002028
:100CA0002844525952554E29004732392041757413
:100CB0006F20426564204C6576656C696E67003F05
:100CC00020284C2C522C462C4229206F7574206F02
:100CD0006620626F756E64732E0A003F2856296580
:100CE00072626F7365206C6576656C20696D706CDF
:100CF00061757369626C652028302D34292E0A00D5
:100D0000426164205A2076616C75650A004E6F203E
:100D100062696C696E65617220677269640A004479
:100D20006576696174696F6E0025533A20257300FA
:100D300046696E6973686564210A003A207A3A2030
:100D400000206F662000476F696E6720746F3A203D
:100D5000580043570A00206469723A0020616E67A8
:100D60006C653A00537461727420726164697573C2
:100D70003A004D343820506F696E740025533A2084
:100D800025642F256400506F736974696F6E696EF6
:100D900067207468652070726F62652E2E2E0A00BF
:100DA0003F4C656773206F66206D6F76656D656E6D
:100DB0007420696D706C61757369626C6520283090
:100DC0002D3135292E0A003F2028582C5929206F13
:100DD0007574206F6620626F756E64732E0A005002
:100DE000726F6265206F7574206F6620626F756E1A
:100DF0006473003F53616D706C652073697A652080
:100E00006E6F7420706C61757369626C6520283434
:100E10002D3530292E0A004D3438205A2D50726F4E
:100E20006265205265706561746162696C6974798C
:100E300020546573740A003F2856296572626F73E7
:100E400065206C6576656C20696D706C6175736981
:100E5000626C652028302D34292E0A005374616E8F
:100E60006461726420446576696174696F6E3A20CA
:100E7000002052616E67653A2000204D61783A206B
:100E800000204D696E3A2000205369676D613A2059
:100E9000004D65616E3A20005741524E494E472140
:100EA000204C6F77205A204A65726B206D61792043
:100EB0006C65616420746F20756E77616E74656413
:100EC000207061757365732E0A004F4646004F4EC1
:100ED0000020204D61783A2000200020204D696ECE
:100EE0003A2000536F667420656E6473746F70737C
:100EF0003A20003D3D4F6E506F7765724C6F7373B3
:100F0000526573756D653D3D004D32342053256C3F
:100F1000642054256C64004739322E3920452573EE
:100F200000473120462564004739322E39205A25A2
:100F300073004731205A302046323030004731208C
:100F400058257320592573204633303030004D34F6
:100F5000323020532569205A2573004D3130362018
:100F600050256920532569004D32303020442573C7
:100F70000047323852305859004739322E3920450F
:100F800030205A300A47315A2573004D313039200C
:100F9000532569004D31393020532569004D3432D5
:100FA00030205330205A300020496E76616C6964DD
:100FB000206578747275646572200047322F47335C
:100FC0002062616420706172616D65746572730A7C
:100FD00000536C6565702E2E2E005A2050726F6281
:100FE000652050617374204265640A005A20507273
:100FF0006F62652050617374204265640047323827
:101000004C30004D3131372050726F62652066617F
:10101000696C65642E0A4732380A0070726F626527
:101020005F72657769706500473239205265747266
:1010300079696E670050726F62696E6720466169F8
:101040006C6564004D31313720426564206C6576F3
:10105000656C696E67206661696C65642E0A47304D
:10106000205A31300A4D3330302050323520533839
:1010700038300A4D333030205035302053300A4D4F
:101080003330302050323520533838300A4D333029
:1010900030205035302053300A4D3330302050321C
:1010A0003520533838300A4D333030205035302019
:1010B00053300A47342053310070726F62655F66A7
:1010C00061696C6564004D31313720426564206C84
:1010D0006576656C696E6720646F6E652E00205AB8
:1010E0003A200020593A200042656420583A2000F6
:1010F0004D65736820706F696E74206F7574206F12
:10110000662072616E67650A004D302053746F70FF
:10111000004D312053746F7000436F6E74696E75AB
:101120006500436C69636B20746F20526573756D45
:10113000652E2E2E004E6F204D6F76652E00456E6B
:10114000642066696C65206C6973740A0042656787
:10115000696E2066696C65206C6973740A004E6F55
:10116000206D656469610A00526573756D696E670B
:1011700020534400286E6F2066696C652900437512
:101180007272656E742066696C653A2000507269EF
:101190006E742074696D653A20000A53746174732B
:1011A0003A2046696C616D656E7420757365643AAA
:1011B00020002C204C6F6E67657374206A6F623A52
:1011C0002000546F74616C2074696D653A2000537F
:1011D000746174733A20002C204661696C65643A2E
:1011E00020002C2046696E69736865643A200050BF
:1011F00072696E74733A200053746174733A2000FC
:10120000436F6F6C696E672E2E2E0048656174699E
:101210006E672E2E2E0045202553006F6B006F66E3
:1012200066006A0465045E04570449044445425557
:10123000473A004D31313320530042656420436FFB
:101240006F6C696E672E2E2E0042656420486561C2
:1012500074696E672E2E2E00444458204D6178200C
:101260004F46462E002F2F00205200416363656CCD
:1012700065726174696F6E3A2050004D32303620CD
:10128000580046523A0020466C6F773A20003A20C8
:101290000020536572766F2000206F7574206F6692
:1012A0002072616E67650A00536572766F200020B8
:1012B000643A0020693A0020703A00496E76616C09
:1012C00069642065787472756465720A0020643AF6
:1012D0000020693A0020703A0064697300656E006E
:1012E00043290A0061626C656420286D696E207470
:1012F000656D702000436F6C64206578747275644E
:101300006573206172652000504944204175746FF7
:1013100074756E6500504944204175746F74756E24
:1013200065206661696C656421204261642068659E
:10133000617465722069640A0046696C616D656E4E
:10134000742072756E6F75742064697374616E6356
:101350006520286D6D293A200046696C616D656EC7
:10136000742072756E6F757420004D3432312069AF
:101370006E636F727265637420706172616D657403
:1013800065722075736167650A004D65736820702A
:101390006F696E74206F7574206F662072616E675E
:1013A000650A004F666673657473204170706C69DE
:1013B0006564004572723A20546F6F206661722135
:1013C00000546F6F206661722066726F6D207265C7
:1013D000666572656E636520706F696E740A00459C
:1013E0004550524F4D204F4B0A00506F7765722D7C
:1013F0006C6F7373207265636F7665727920004D30
:10140000383400446F6E65207072696E74696E675F
:101410002066696C650A004D3737004D3331004353
:1014200061703A004D4541545041434B00434F4F8A
:101430004C45525F54454D5045524154555245001C
:101440004348414D4245525F54454D5045524154E9
:1014500055524500424142595354455050494E4718
:101460000041524353004D4F54494F4E5F4D4F443E
:10147000455300544845524D414C5F50524F5445DE
:101480004354494F4E004C4F4E475F46494C454EE2
:10149000414D45004155544F5245504F52545F53B2
:1014A000445F5354415455530053445F5752495479
:1014B0004500524550454154005344434152440075
:1014C00050524F4D50545F535550504F5254004559
:1014D0004D455247454E43595F5041525345520086
:1014E000434153455F4C494748545F42524947483E
:1014F000544E45535300544F47474C455F4C494762
:1015000048545300534F4654574152455F504F572C
:101510004552004255494C445F50455243454E5454
:10152000004C4556454C494E475F44415441005A92
:101530005F50524F42450052554E4F555400415551
:10154000544F4C4556454C005052494E545F4A4FFB
:10155000420050524F4752455353004155544F5249
:1015600045504F52545F54454D5000564F4C554DC9
:10157000455452494300454550524F4D0042494E53
:101580004152595F46494C455F5452414E5346457E
:10159000520053455249414C5F584F4E5F584F4699
:1015A00046004649524D574152455F4E414D453ADE
:1015B0004D61726C696E20322E302E375F44573782
:1015C0002E3320426F6E64746563682035534D443A
:1015D0004242202841707220323420323032312091
:1015E00032333A32323A30302920534F5552434544
:1015F0005F434F44455F55524C3A68747470733A78
:101600002F2F6769746875622E636F6D2F496E7333
:10161000616E6974794175746F6D6174696F6E2F55
:101620004D61726C696E2F747265652F43726561CE
:101630006C6974794477696E5F322E302050524F56
:10164000544F434F4C5F56455253494F4E3A312EFB
:1016500030204D414348494E455F545950453A4426
:101660004458204D61782045585452554445525FA6
:10167000434F554E543A3120555549443A636564B9
:1016800065326132662D343161322D343734382D74
:10169000396231322D63353563363266333637661B
:1016A000660A0050726F6265204F6666736574202B
:1016B0005A0050726F6265204F6666736574205AD7
:1016C00000290A0020746F20003F5A206F75742093
:1016D0006F662072616E6765202800290A002074F9
:1016E0006F20003F59206F7574206F662072616E05
:1016F000676520282D00290A0020746F20003F58BC
:10170000206F7574206F662072616E676520282DCA
:101710000050726F6265204F6666736574205800D2
:1017200043616E6E6F74206F70656E2073756264B6
:10173000697220002569730025696D202569730091
:101740002569682025696D20256973002569642055
:101750002569682025696D20256973002569792030
:10176000256964202569682025696D202569730035
:101770003D3D4477696E20496E697420436F6D70FA
:101780006C6574653D3D002A2A2A4E6F7A7A6C6535
:1017900054656D705374617475735B325D203D00E8
:1017A0003D3D48656174696E6720446F6E652043F6
:1017B00068616E67652046696C616D656E743D3D5C
:1017C000002020737461727470726F677265737336
:1017D00020003D3D7761697477617920353D3D009A
:1017E0003D3D7761697477617920343D3D003D3D31
:1017F0007761697477617920333D3D003D3D7761C4
:10180000697477617920313D3D003D3D6F6E5072C6
:10181000696E7454696D657253746F707065643D60
:101820003D003D3D6F6E466163746F727952657322
:1018300065743D3D00270A0A000027202700202765
:10184000002D006E6F74696669636174696F6E2044
:101850000063616E63656C005072696E7420416252
:101860006F72746564004469736D697373005549E0
:101870002041626F7274656400726573756D6500F6
:101880004D3234002A2A2A43506C617920546F6EFD
:10189000652A2A2A003D3D6F6E5072696E74546944
:1018A0006D65725061757365643D3D00486F6D698B
:1018B0006E67204661696C6564006F70656E0054E8
:1018C0005249474745524544003A200066696C61D9
:1018D0006D656E74007A5F6D696E00795F6D696E1B
:1018E00000785F6D696E005265706F7274696E6723
:1018F00020656E6473746F70207374617475730AFD
:101900000020746F6F206C6F6E672065787472753D
:1019100073696F6E2070726576656E7465640A0017
:1019200020636F6C6420657874727573696F6E20C4
:1019300070726576656E7465640A00486F6D652027
:10194000257325732573204669727374005761727D
:101950006E696E673A20486F6D696E672042756DDB
:10196000702044697669736F72203C20310A00024E
:101970000204000000000000000000000000000061
:10198000E1430000E1430000EB43000000410000A0
:10199000004100000040FFFFFF00000001000000C8
:1019A00001000080005555550000004000333333DE
:1019B00000AAAA2A004992240000002000C7711C36
:1019C0000099991900D1451700555515003BB113E1
:1019D000002449120011111100000010000F0F0F18
:1019E00000E3380E0043790D00CCCC0C00C3300C62
:1019F00000E8A20B0064210B00AAAA0A00703D0AAD
:101A0000009DD80900427B090092240900DCD3081C
:101A100000888808001042080000000800F0C10794
:101A2000008787070075500700711C07003EEB0612
:101A300000A1BC06006990060066660600703E06BE
:101A4000006118060017F4050074D105005BB005AD
:101A500000B2900500627205005555050078390501
:101A600000B81E0500050505004EEC040087D404EF
:101A700000A1BD040090A7040049920400C17D04A8
:101A800000EE690400C7560400444404005C3204BC
:101A9000000821040041100400000004003FF0038E
:101AA00000F8E0030026D20300C3C30300CCB50353
:101AB000003AA803000A9B0300388E0300C081038C
:101AC000009F750300D0690300505E03001D53039F
:101AD0000034480300913D0300333303001629030B
:101AE00000381F030097150300300C0300030303A5
:101AF000000BFA020049F10200BAE802005CE002C1
:101B0000002DD802002DD0020059C80200B0C0023A
:101B10000031B90200DAB10200AAAA0200A0A302B1
:101B200000BC9C0200FA9502005C8F0200DF880274
:101B30000082820200457C020027760200277002A4
:101B400000436A02007C640200D05E02003F59023A
:101B500000C8530200FFFDFCFAF8F6F4F2F0EEECD8
:101B6000EAE9E7E5E3E1E0DEDCDAD9D7D5D4D2D0A3
:101B7000CFCDCBCAC8C7C5C3C2C0BFBDBCBAB9B739
:101B8000B6B4B3B2B0AFADACAAA9A8A6A5A4A2A1A1
:101B9000A09E9D9C9A99989795949392908F8E8DE4
:101BA0008B8A8988878684838281807F7E7D7B7A09
:101BB000797877767574737271706F6E6D6C6B6A0D
:101BC000696867666564636261605F5E5D5C5B5AFD
:101BD0005958585756555453525150504F4E4D4CDA
:101BE0004B4A4A4948474646454443424241403FA2
:101BF0003E3E3D3C3B3B3A39383837363535343359
:101C000032323130302F2E2E2D2C2B2B2A29292801
:101C1000272726252524232322212120201F1E1E9D
:101C20001D1C1C1B1B1A191918181716161515142C
:101C3000131312121111100F0F0E0E0D0D0C0C0BB1
:101C40000A0A09090808070706060505040403032C
:101C500002020100003D3D6F6E5072696E7454695E
:101C60006D6572537461727465643D3D000000E1FE
:101C7000430000E1430000EB4300000000000000CF
:101C800000000000003D3D6F6E53746F7265536538
:101C90007474696E67733D3D003D3D6F6E436F6EBA
:101CA00066696775726174696F6E53746F72655798
:101CB00072697474656E3D3D0053657474696E6736
:101CC000732053746F726564000A20696E69742012
:101CD0007A70726F62655F7A6F6666736574203DB5
:101CE00020003D3D6F6E436F6E666967757261746B
:101CF000696F6E53746F7265526561643D3D004556
:101D00004550524F4D20496E697469616C697A651E
:101D1000640A003B20003A0A0020204D3630332070
:101D20000020440020204D34313220530046696C9D
:101D3000616D656E742072756E6F75742073656E5B
:101D4000736F723A002055004C0046696C616D65F6
:101D50006E74206C6F61642F756E6C6F6164206CA3
:101D6000656E677468733A0020204D38353120580D
:101D7000005A2D50726F6265204F6666736574005D
:101D800020204D343133205300506F7765722D4C35
:101D90006F7373205265636F766572793A002044E1
:101DA0000020490020204D333034205000204400D2
:101DB00020490020204D333031205000504944202C
:101DC00073657474696E67733A00204A0020204777
:101DD0003239205720490020204D34323020530022
:101DE0004175746F20426564204C6576656C696E40
:101DF000673A0020204D323036205800486F6D651C
:101E0000206F66667365743A0020580020530020E6
:101E1000204D323035204200416476616E63656446
:101E20003A20423C6D696E5F7365676D656E745FE5
:101E300074696D655F75733E20533C6D696E5F66B6
:101E4000656564726174653E20543C6D696E5F74B3
:101E5000726176656C5F66656564726174653E206B
:101E6000583C6D61785F785F6A65726B3E20593CC3
:101E70006D61785F795F6A65726B3E205A3C6D6177
:101E8000785F7A5F6A65726B3E20453C6D61785F72
:101E9000655F6A65726B3E0020540020520020206E
:101EA0004D323034205000416363656C657261745B
:101EB000696F6E2028756E6974732F7332293A200A
:101EC000503C7072696E745F616363656C3E205252
:101ED0003C726574726163745F616363656C3E201C
:101EE000543C74726176656C5F616363656C3E003F
:101EF00020204D3230312058004D6178696D756D6C
:101F000020416363656C65726174696F6E2028752A
:101F10006E6974732F7332293A0020204D323033AA
:101F20002058004D6178696D756D20666565647235
:101F3000617465732028756E6974732F73293A0074
:101F400053746570732070657220756E69743A0001
:101F500020440020204D323030205300204469734B
:101F600061626C65640A0046696C616D656E74201F
:101F700073657474696E67733A0020286D6D29006B
:101F80002020473231202020203B20556E69747379
:101F900020696E206D6D003D3D6F6E4C6F61645326
:101FA000657474696E67733D3D000000FA4300007C
:101FB000C84300007041000096420000A0420000AB
:101FC000A0420000C8430080CF43E8030000BC02E9
:101FD0000000640000004B00000024F4D43050C323
:101FE0008E20C2A24017828B7011127A910D816CE3
:101FF000D90AA861E108C7586607615143061E4B1C
:102000005D05C145A7041A411104093D98037139C2
:1020100031034036DB0265339102D4305402802E06
:102020001D02632CEE01752AC501B028A0011027FE
:1020300081018F2564012B244B01E0223401AC2166
:102040001F018D200D01801FFC00841EED00971DD7
:10205000DF00B81CD200E61BC600201BBC00641ABF
:10206000B200B219A8000A19A0006A189900D11785
:10207000910040178B00B516840031167E00B31511
:1020800079003A157300C7146F0058146A00EE13F4
:1020900066008813630025135E00C7125B006C1294
:1020A000570015125400C111510070114F00211139
:1020B0004B00D61049008D10470046104400021016
:1020C0004200C00F4000800F3E00420F3C00060F50
:1020D0003B00CB0E3800930E37005C0E3500270E08
:1020E0003400F30D3200C10D3100900D3000600D51
:1020F0002E00320D2D00050D2C00D90C2B00AE0C3E
:102100002900850C29005C0C2700350C27000E0CDB
:102110002600E80B2400C40B2400A00B23007D0B39
:1021200023005A0B2100390B2100180B2000F80A5C
:102130001F00D90A1E00BB0A1E009D0A1D00800A4E
:102140001D00630A1C00470A1B002C0A1B00110A11
:102150001A00F7091A00DD091900C4091900AB09B2
:102160001900920917007B091800630917004C0930
:10217000160036091600200916000A091500F50890
:102180001500E0081400CC081400B8081400A408D6
:102190001400900813007D0812006B081300580803
:1021A000120046081200340811002308110012081A
:1021B000110001081100F0071000E0071000D0071F
:1021C0001000C0071000B0070F00A1071000910712
:1021D0000E0083070F0074070F0065070E005707F6
:1021E0000E0049070E003B070D002E070E002007CA
:1021F0000D0013070D0006070D00F9060C00ED0693
:102200000D00E0060C00D4060C00C8060C00BC064D
:102210000C00B0060C00A4060B0099060C008D06FD
:102220000B0082060B0077060B006C060B006106A4
:102230000A0057060B004C060A0042060A00380640
:102240000A002E060A0024060A001A060A001006D2
:10225000090007060A00FD050900F4050900EB0561
:102260000900E2050900D9050900D0050900C705E4
:102270000900BE050900B5050800AD050800A50563
:1022800009009C050800940508008C0508008405D9
:1022900008007C050800740508006C05070065054A
:1022A00008005D050700560508004E0507004705B4
:1022B00007004005080038050700310507002A051A
:1022C0000700230507001C050600160507000F057B
:1022D00007000805060002050700FB040600F504D8
:1022E0000700EE040600E8040600E2040700DB0431
:1022F0000600D5040600CF040600C9040600C30486
:102300000600BD040600B7040600B1040500AC04D5
:102310000600A6040600A00405009B040600950420
:102320000500900406008A04050085040500800469
:1023300006007A04050075040500700405006B04AE
:10234000050066040500610405005C0405005704EF
:102350000500520405004D0405004804050043042F
:1023600005003E0404003A0405003504050030046D
:1023700004002C04050027040400230405001E04A7
:1023800004001A04040016040500110404000D04DE
:102390000400090405000404040000040400FC0314
:1023A0000400F8030400F4030400F0030400EC0349
:1023B0000400E8030400E4030400E0030400DC0379
:1023C0000400D8030400D4030400D0030400CC03A9
:1023D0000400C8030300C503030024F404D9201B30
:1023E000C40C5C0E9804C4095F0265077101F40512
:1023F000F900FB04B30048048700C10369005803D7
:10240000550003034500BE023A0084023100530226
:102410002A002902250004022000E4011C00C80152
:102420001900AF0117009801140084011300710115
:1024300010006101100051010E0043010D00360132
:102440000B002B010B0020010B00150109000C01F2
:10245000090003010800FB000800F3000800EB007E
:102460000700E4000600DE000600D8000600D200E7
:102470000600CC000500C7000500C2000500BD0035
:102480000400B9000400B5000400B1000400AD0070
:102490000400A9000400A5000300A20003009F009F
:1024A00004009B00030098000300950002009300C5
:1024B0000300900003008D0002008B0003008800E1
:1024C00002008600020084000300810002007F00F9
:1024D00002007D0002007B0002007900020077000C
:1024E0000100760002007400020072000100710019
:1024F00002006F0002006D0001006C0002006A0023
:10250000010069000200670001006600010065002B
:10251000010064000200620001006100010060002F
:1025200001005F0002005D0001005C0001005B0033
:1025300001005A0001005900010058000100570035
:102540000100560001005500010054000100530035
:102550000000530001005200010051000100500032
:1025600001004F0001004E0000004E0001004D0030
:1025700001004C0001004B0000004B0001004A002C
:102580000100490001004800000048000100470028
:102590000100460000004600010045000000450023
:1025A000010044000100430000004300010042001C
:1025B0000000420001004100000041000100400015
:1025C00001003F0000003F0001003E0000003E000F
:1025D00001003D0000003D0001003C0000003C0007
:1025E00000003C0001003B0000003B0001003A00FD
:1025F00000003A00010039000000390001003800F5
:1026000000003800000038000100370000003700EB
:1026100001003600000036000000360001003500E1
:1026200000003500000035000100340000003400D7
:1026300000003400010033000000330000003300CC
:1026400001003200000032000000320001003100C1
:1026500000003100000031000100300000003000B7
:102660000000300001002F0000002F0000002F00AC
:1026700000002F0001002E0000002E0000002E00A0
:1026800001002D0000002D0000002D0000002D0095
:1026900001002C0000002C0000002C0000002C0089
:1026A00001002B0000002B0000002B0000002B007D
:1026B00001002A0000002A0000002A0000002A0071
:1026C0000100290000002900000029000000290065
:1026D0000000290001002800000028000000280058
:1026E000000028000000280001002700000027004B
:1026F000000027000000270000002700010026003E
:102700000000260000002600000026000000260031
:102710000100250000002500000025000000250024
:102720000000250000002500010024000000240016
:102730000000240000002400000024000100230009
:1027400000002300000023000000230000002300FD
:1027500000002300000023000100220000002200EE
:1027600000002200000022000000220000002200E1
:1027700001002100000021000000210000002100D4
:1027800000002100000021000000210001002000C5
:1027900000002000000020000000200000002000B9
:1027A00000002000000020000000200001001F00A9
:1027B00000001F0000001F0000001F0000001F009D
:1027C00000001F0000001F0001001E0000001E008E
:1027D00000001E0000001E000000393000003325FC
:1027E000000087190000B00F0000DB080000BD04E6
:1027F0000000740200003F01000020436F756E74FA
:1028000020583A0023646566696E65204445464158
:10281000554C545F0000626564004B6420004B69B6
:1028200020004B702000504944204175746F74752E
:102830006E652066696E69736865642120507574E1
:1028400020746865206C617374204B702C204B6978
:1028500020616E64204B6420636F6E7374616E74CC
:10286000732066726F6D2062656C6F7720696E747D
:102870006F20436F6E66696775726174696F6E2E43
:10288000680A00504944204175746F74756E652064
:102890006661696C6564212074696D656F75740A81
:1028A00000504944204175746F74756E65206661EF
:1028B000696C6564212054656D7065726174757210
:1028C0006520746F6F20686967680A00204B643A5E
:1028D0002000204B693A2000204B703A2000204312
:1028E0006C617373696320504944200A00204E6F65
:1028F000206F76657273686F6F740A002054753AA2
:102900002000204B753A2000206D61783A2000208D
:102910006D696E3A200020643A200020626961737C
:102920003A2000504944204175746F74756E6520DB
:1029300073746172740A00504944204175746F7455
:10294000756E65206661696C6564212054656D70E3
:102950006572617475726520746F6F20686967684D
:102960000A0042656400453100626564002C2073F2
:10297000797374656D2073746F707065642120487D
:1029800065617465725F49443A2000486561746905
:102990006E67204661696C65640048656174696EA4
:1029A00067206661696C6564004D3131322053687F
:1029B0007574646F776E001000C90210012C01401D
:1029C00001220170011801B0010E01F00104015053
:1029D00002FA00B002F0003003E600D003DC009001
:1029E00004D2007005C800A006BE000008B400B004
:1029F00009AA00D00BA000600E960060118C0000A8
:102A000015820020197800C01D6E00A0226400B05D
:102A1000275A00902C500000314600E0343C001052
:102A2000383200903A2800603C1E00A03D1400801F
:102A30003E0A00203F0000544845524D414C205270
:102A4000554E4157415900546865726D616C205272
:102A5000756E61776179004572723A204D41585424
:102A6000454D50004D415854454D50207472696792
:102A70006765726564004572723A204D494E54454F
:102A80004D50004D494E54454D5020747269676752
:102A90006572656400202F002042403A0020403AD1
:102AA0000020573A0020573A00496E76616C6964FD
:102AB0002065787472756465720A007C3C3E5E2BFA
:102AC0003D3F2F5B5D3B2C2A225C0043616E6E6FA5
:102AD00074206F70656E2073756264697220005394
:102AE0004420496E6974204661696C005344206338
:102AF000617264206F6B0A006F70656E526F6F7445
:102B0000206661696C65640A00766F6C756D652E70
:102B1000696E6974206661696C65640A004E6F2095
:102B2000534420636172640A000A4D3234004D320E
:102B300033202573002E0A006F70656E2066616970
:102B40006C65642C2046696C653A200046696C65AA
:102B50002073656C65637465640A002053697A6547
:102B60003A200046696C65206F70656E65643A2096
:102B700000454E4420535542524F5554494E450A44
:102B8000002220706F73002220706172656E743AAB
:102B90002200535542524F5554494E452043414C13
:102BA0004C207461726765743A22005375626361E8
:102BB0006C6C204F766572666C6F77004578636544
:102BC00065646564206D617820535542524F5554B9
:102BD000494E452064657074683A002E0A004465C9
:102BE0006C6574696F6E206661696C65642C204643
:102BF000696C653A200046696C652064656C657493
:102C000065643A005344207072696E74696E67207F
:102C10006279746520004E6F74205344207072698D
:102C20006E74696E670A0057726974696E67207402
:102C30006F2066696C653A2000667265736800648F
:102C40006F696E67002066696C653A20004E6F7789
:102C500020002F6175746F25632E67002020506C53
:102C6000616E6E65724275666665724279746573EF
:102C70003A20002046726565204D656D6F72793A85
:102C80002000436F6D70696C65643A20417072205A
:102C9000323420323032310A00204C6173742055B6
:102CA0007064617465643A20323032312D30342DD5
:102CB0003138207C20417574686F723A20426F6E03
:102CC0006474656368202F20496E73616E6974793E
:102CD0004175746F6D6174696F6E0A00322E302E0B
:102CE000375F4457372E330A004D61726C696E00AE
:102CF00020536F6674776172652052657365740A3C
:102D000000205761746368646F672052657365744F
:102D10000A002042726F776E206F757420526573BF
:102D200065740A002045787465726E616C20526586
:102D30007365740A00506F77657255700A0073747A
:102D40006172740A004732385859004D31303031C1
:102D5000006572726F722077726974696E67207491
:102D60006F2066696C650A00446F6E65207361763A
:102D7000696E672066696C652E0A004D3239004520
:102D80006E6473746F707300255320256320256370
:102D900020256320256300205A3A0020593A00205C
:102DA000583A00656E6473746F7073206869743A82
:102DB00020006001F4017001EA019001E001B0011E
:102DC000D601D001CC010002C2013002B80160027C
:102DD000AE019002A401D0029A0120039001700379
:102DE0008601C0037C0130047201A0046801200543
:102DF0005E01B005540160064A0120074001F0075A
:102E00003601F0082C01100A2201500B1801C00CE9
:102E10000E01500E04013010FA002012F000501480
:102E2000E600C016DC007019D200501CC800501F0C
:102E3000BE007022B400B025AA00F028A000202C0B
:102E40009600302F8C0010328200A0347800F036CB
:102E50006E00E0386400803A5A00403B5500E03B89
:102E60005000F03C4600C03D3C00603E3200E03E79
:102E70002800303F1E00503F1900703F1400A03F53
:102E80000A00C03F0000D03FF6FFE03FECFF00002B
:102E90000A0B02090C0D0E080703040100000000D4
:102EA0000000000000000000000000000000000022
:102EB00000000000000000000000121110000000DF
:102EC0000000000000000000000000000000000002
:102ED0000000000050726F62696E67204661696C85
:102EE000656400205A3A200020593A200042656467
:102EF00020583A20003D3D6F6E55736572436F6EEA
:102F00006669726D52657175697265643D3D002236
:102F10000A00556E6B6E6F776E20636F6D6D616E1C
:102F2000643A2022002042002050006F6B002045B0
:102F300000205A00205900204D39322058002045E9
:102F40003A00205A3A0020593A00583A0020746F4B
:102F50006F206C6F6E6720657874727573696F6E21
:102F60002070726576656E7465640A0020636F6C0C
:102F70006420657874727573696F6E2070726576FF
:102F8000656E7465640A0043616E6E6F7420656ED1
:102F9000746572207375626469723A20004D32352F
:102FA00020500A4D323400526573756D65005549E5
:102FB000205061757365004E6F204D617463682009
:102FC0003A0050675570005067446F776E00497340
:102FD0002046696C652000497320446972200047CF
:102FE0006F557044697200486173204D6564696172
:102FF0000046696C656E616D652053656C65637430
:103000006564004D3130303043004D313030300098
:1030100046696C616D656E74205374617420302054
:103020002D20330046696C616D656E7420537461A8
:10303000742030202D20320046696C616D656E74FD
:1030400020537461742030202D2031002046696C9B
:10305000616D656E7420526573706F6E7365204E7E
:103060006F00526573756D652059657320647572C4
:10307000696E67207072696E74000A204E6F204678
:10308000696C616D656E7400496E76616C6964206F
:103090004F7074696F6E004D3530300053746F722D
:1030A000652053657474696E6773004265642050CF
:1030B00049442053746172746564004D3939390A8A
:1030C0004D32383050305331363000424C546F75E9
:1030D0006368205265736574004D3530320A4D3592
:1030E000303000496E697420454550524F4D0048BC
:1030F0006F74656E64205049442053746172746526
:103100006400456E676C69736820416C7265616428
:103110007920536574004368696E657365204E6F4E
:103120007420537570706F7274656400496E4C61E1
:103130006E6743686F696365000A202A2A2A7265F0
:10314000636461742E646174615B305D203D00478F
:1031500032380A4731204631303030205A31300081
:10316000556E737570706F72746564204F707469FA
:103170006F6E2053656C6563746564004732365228
:10318000323535004D3139305335350A4732380A3A
:103190004732390A4D3430300A4D313034533231F0
:1031A000350A4732380A4D313039533231350A4DFC
:1031B00034323053310A47315831303059313030A0
:1031C00046353030300A47315A300A4D3530300AF2
:1031D0004D31313720536574205A204F6666736530
:1031E00074004731204631303030205A302E3000C4
:1031F0004732380A4731204631303030205A302E9D
:1032000030004D353030005A204F666673657420AB
:103210003A202573004D353030005A204F666673D2
:103220006574203A202573004732380A4731463109
:103230003530305A302E30004732385A0A4731463E
:10324000313530305A302E30004D38340047314659
:10325000313030305A302E30004732380A4731464C
:10326000313030305A302E30004D616E75616C5304
:10327000657454656D70005A204F666673657420DE
:103280003A2025730053746F702054726967676524
:103290007265640053746F70204E6F0053746F70CA
:1032A0005072696E740048616E646C65204461748C
:1032B000612041646A7573742032205365747469A7
:1032C0006E672053637265656E200048616E646CA2
:1032D000652044617461205072696E7446696C6542
:1032E00020332053657474696E672053637265657B
:1032F0006E200048616E646C6520446174612050EA
:1033000072696E7446696C65203220536574746905
:103310006E672053637265656E20004D3834004837
:10332000616E646C652044617461205072696E74D2
:1033300046696C6520506F73740048616E646C65FB
:103340002044617461205072696E7446696C652016
:1033500050726500426567696E53776974636800EF
:103360003D3D20436865636B6B65793D3D0072654B
:10337000636461742E61646472203D3D0072656314
:103380006461742E646174615B305D203D3D007743
:10339000616974776179203D3D0020202A2A2A2A1C
:1033A0002A2A2A5254535F48616E646C65446174E2
:1033B000612A2A2A2A2A2A2A2A2000526573656E3F
:1033C000643A200000002200250028002B002E0077
:1033D0003100340002010000050108010B0100006A
:1033E0002100240027002A002D00300033000101B5
:1033F0000000040107010A01050505050705080885
:103400000808020202020A0A08080404040401016E
:103410000101010101010303030303030303040783
:1034200007070C0C0C0C0C0C0C0C0202020206061A
:103430000606060606060B0B0B0B0B0B0B0B01020D
:1034400010202008081020401020408002010201B6
:10345000080402010102040810204080804020106E
:1034600008040201800402018040201008040201C7
:10347000080402010102040810204080010204082F
:1034800010204080444458204D617820526561648A
:10349000792E005072696E74696E672E2E2E005060
:1034A00072696E7420506175736564006E6F746923
:1034B0006669636174696F6E2000504944205475D9
:1034C0006E652046696E697368656400CA00FC0019
:1034D00011241FBECFEFD1E2DEBFCDBF00E00CBF95
:1034E00014E0A0E0B2E0EEE2F0E602E00BBF02C0C2
:1034F00007900D92A030B107D9F726E1A0E0B4E023
:1035000001C01D92AC32B207E1F71AE1C7E6DAE179
:1035100000E006C021970109802FFE010F94442C82
:10352000C636D10780E00807A9F70F94BB190D94A0
:1035300005300C9400009F92AF92BF92CF92DF9221
:10354000EF92FF920F931F93CF93DF9300D01F92C0
:103550001F92CDB7DEB7E5E5FBE10027BB27462F7D
:10356000572FA82FAA2341F4A52F542FB85FAA23C1
:1035700019F4A52F5527B85FA03138F45295A295BC
:10358000452F4F70507FA42BBC5FA03428F4550FFB
:10359000AA1F550FAA1FBE5FA03818F4550FAA1F07
:1035A000B395550FAA1FEA0FF01F449151E0AA27C7
:1035B000B85081F1C8F0B0FF02C0440F551FB1FFF1
:1035C00004C0440F551F440F551FB2FF06C052954B
:1035D0004295142F1F70407F512BB3FF1BC0A52FA6
:1035E000542F44270C940A1BB195B0FF02C0559587
:1035F0004795B1FF04C05595479555954795B2FF3E
:1036000005C05295407F4295452B5F70B3FF02C0C5
:10361000452F5527DD24CC24BB24B2E0649FD0186D
:10362000C108B00AB00B749FC018B108B00B849FDA
:10363000B018B109659FC018B108B00B759FB018DC
:10364000B109859FB0196A9FB018B1097A9FB01966
:103650004D9DA12C99243327992722275D9DA00CED
:10366000911C301F901F201FAD9D900C311D901F8D
:10367000201F4C9DA00C911C301F901F201F5C9D93
:10368000900C311D901F201FAC9D300D911D201FEF
:103690004B9D900C311D901F201F5B9D300D911D87
:1036A000201FAB9D900D211D4B9F300D911D201FA4
:1036B0005B9F900D211DAB9F200DB1E0BB24CC245E
:1036C000DD24639FD018C108B00AB00B739FC018E7
:1036D000B108B00B839FB018B109699FC018B10839
:1036E000B00B799FB018B109899FB019629FB018CB
:1036F000B109729FB019D61AC70AB80A20F0B1E012
:103700003B0F901F201F1124792F632F90E0822FF1
:103710000F900F900F900F900F90DF91CF911F910E
:103720000F91FF90EF90DF90CF90BF90AF909F9060
:103730000895AF92BF92CF92DF92EF92FF920F93D4
:103740001F93CF93DF93CAE3DCE009EE18E08AE42D
:10375000A82E8CE0B82EC12CD12C7601C39469918F
:103760007991899199910F948225288939894A897B
:103770005B890F94E3250F94C02DF8016193719339
:10378000819391938F01C616D706E806F90610F4C7
:103790006B017C01AC16BD0611F76FEF7FEFCB011B
:1037A000A70196010F94C12B2093F9083093FA08D2
:1037B0004093FB085093FC08DF91CF911F910F912C
:1037C000FF90EF90DF90CF90BF90AF900895CF9291
:1037D000DF92EF92FF928091F507882309F457C09A
:1037E000C090F107D090F207E090F307F090F40753
:1037F00020E030E0A901C701B6010F947D258823A0
:1038000009F445C020E030E040E05FE3C701B601C5
:103810000F94E3259B01AC010F94E3252BED3FE0D2
:1038200049E450E40F94E3259B01AC0160E070E0B3
:1038300080E89FE30F94472D6B017C01C092360C0A
:10384000D092370CE092380CF092390C60916502FE
:1038500070916602072E000C880B990B0F9484253B
:103860002AE037ED43E25CE30F94E325A7019601DC
:103870000F94E32560936102709362028093630268
:1038800090936402FF90EF90DF90CF900895C12C49
:10389000D12C80E8E82E8FE3F82ED0CF0F931F9322
:1038A000CF93DF9350E0FC01E40FF51F8081440FBC
:1038B000551F440F551F45565A4FEA01882329F1D9
:1038C00088819981AA81BB81EB01088119812A81B4
:1038D0003B810097A105B10569F40C591F4F2F4F8B
:1038E0003F4FDA010D931D932D933C9313978FEF68
:1038F000808306C0081B190B2A0B3B0B37FDF7CF43
:10390000DF91CF911F910F910895188219821A8229
:103910001B82F6CFCF93DF9324E0829FC001112456
:10392000EC01C453D74FFC01EE5FF74F8A50984F1C
:10393000DC012D913D914D915C916081718182817D
:1039400093810F944D2C688379838A839B83DF91C5
:10395000CF9108958091960590919705A091980533
:10396000B09199058093410290934202A093430243
:10397000B0934402809194059091950590936802CC
:103980008093670208958091410290914202A09134
:103990004302B09144028093960590939705A093BB
:1039A0009805B09399058091670290916802909371
:1039B00095058093940584E690E090936802809347
:1039C000670208958091851290918612891B8770F5
:1039D00089F480918D0D81110DC08091820C9091A0
:1039E000830C892B39F481E09091A406911103C0D6
:1039F00080E0089581E00895CF93DF93DB01F90122
:103A00009C919130C1F0943080F094509C93883018
:103A1000D1F480819181009771F001979183808327
:103A2000480F591FEA01188206C08C3539F49C5F93
:103A30009C93943041F4DF91CF9108958B3339F703
:103A400081E08C93F8CF20813181B9016F5F7F4F86
:103A500071836083420F531FEA01888380819181C3
:103A60008F3591056CF7E7CF0F931F9381E000919D
:103A7000291410912A1420912B1430912C14409168
:103A8000251450912614609127147091281404175E
:103A900015072607370708F480E01F910F91089556
:103AA00090E080E00895282F9091F007833021F472
:103AB00095FD0FC094FD0FC0892F90E0B0E0A0E00D
:103AC00004C0B695A795979587952A95D2F78170EA
:103AD000089581E0089580E00895FC016591759155
:103AE0008591949108958F929F92AF92BF92CF92B9
:103AF000DF92EF92FF92CF93DF93EC018090C808A2
:103B00009090C908A090CA08B090CB0820E030E09F
:103B1000A901C501B4010F947D25882309F454C07F
:103B2000C880D980EA80FB80A7019601C501B40155
:103B30000F947D2518160CF04CC02091C0083091D0
:103B4000C1084091C2085091C308C701B6010F9443
:103B50007D25882331F1C092C008D092C108E0923F
:103B6000C208F092C3082091C4083091C508409162
:103B7000C6085091C708688179818A819B810F941A
:103B8000E3259B01AC0160E070E080E89FE30F94C7
:103B90004C2C60930F02709310028093110290934B
:103BA000120260910F0270911002809111029091A7
:103BB0001202DF91CF91FF90EF90DF90CF90BF90F6
:103BC000AF909F908F90089560E070E080E89FE351
:103BD000F0CF60E070E0CB01ECCFCF92DF92EF92BC
:103BE000FF92CF93DF93EC01CC80DD80EE80FF80ED
:103BF00027E137EB41ED58EBC701B6010F94AD2E2D
:103C000087FD23C023E030E041EE53E4C701B60155
:103C10000F947D251816CCF0C880D980EA80FB80EF
:103C200027E137EB41ED58EBC701B6010F94AD2EFC
:103C300087FD0BC0C1E023E030E041EE53E4C70153
:103C4000B6010F947D2518160CF4C0E08C2FDF917F
:103C5000CF91FF90EF90DF90CF9008952FEB280F3A
:103C60002A3108F047C0E22FF0E0809133059091AF
:103C70003405A0913505B091360504C0B695A795D9
:103C8000979587952A95D2F780FD02C08170089597
:103C9000EB5EFA4FE081EE2341F180918207909133
:103CA0008307E80FF92FF11D808190ED980F9A306E
:103CB00030F08E3251F4818180538A3098F4F09341
:103CC0000405E093030581E008958D3211F08B32F5
:103CD00049F4818190ED980F9A3088F38E3211F477
:103CE0008281EACFF0E0E0E0EACF10920405109282
:103CF0000305E9CF80E008950E942E1E882341F03D
:103D000081E02091030530910405232B09F480E024
:103D100008958F929F92AF92BF92CF92DF92EF92CF
:103D2000FF92C090D205D090D305E090D405F090DA
:103D3000D50520E030E0A901C701B6010F947D252B
:103D40008823E1F1A701960160E070E080E89FE33D
:103D50000F94472D6B017C018090D6059090D7057C
:103D6000A090D805B090D90520E030E0A901C501A8
:103D7000B4010F947D25882329F1A501940160E009
:103D800070E080E89FE30F94472DC092DC04D0924E
:103D9000DD04E092DE04F092DF046093E0047093AF
:103DA000E1048093E2049093E304FF90EF90DF90AE
:103DB000CF90BF90AF909F908F900895C12CD12C41
:103DC0007601CACF60E070E0CB01DFCF129A089590
:103DD0005F9A8091340C8E7F8093340C8A9A809104
:103DE000340C8D7F8093340C809108018095817014
:103DF000809306018091340C8B7F8093340C0C945B
:103E0000E61E269A2E9A0895833B21E0920714F02D
:103E100083EB91E09093EA118093E9110C9463FD98
:103E2000EEE0F6E0108211821282138214820C946A
:103E300063FD4F925F926F927F928F929F92AF92AB
:103E4000BF92CF92DF92EF92FF920F931F93CF9387
:103E5000DF93EC012091CA053091CB054091CC0550
:103E60005091CD05688179818A819B810F944C2C7A
:103E70006B017C012091CE053091CF054091D0059A
:103E80005091D1056C817D818E819F810F944C2C46
:103E90004B015C01A701960160910302709104023D
:103EA00080910502909106020F947D25882309F4E4
:103EB00050C0C0920302D0920402E0920502F09238
:103EC00006022091DC043091DD044091DE04509123
:103ED000DF04C701B6010F94E3252B013C010F94C9
:103EE000EF2D6B017C0120E030E0A9010F947D25CE
:103EF00087FD70C020E030E040E450E4C701B60127
:103F00000F94AD2E18162CF4C12CD12CC0E4EC2E3D
:103F1000FE2CA7019601C301B2010F944C2C6093B3
:103F2000D4047093D5048093D6049093D704C7012A
:103F3000B6010F94B92D6093D204062E000C770BB6
:103F40006F5F7F4F6430710514F064E070E0609340
:103F5000D004D09101021091D204A5019401609186
:103F60000702709108028091090290910A020F9451
:103F70007D25811133C0D11381C02091B8043091C7
:103F8000B9044091BA045091BB046091D40470917B
:103F9000D5048091D6049091D7040F94E325209105
:103FA000BC043091BD044091BE045091BF040F94F5
:103FB0004D2CDF91CF911F910F91FF90EF90DF90EB
:103FC000CF90BF90AF909F908F907F906F905F90B9
:103FD0004F900895C12CD12C76019BCF809207027F
:103FE00090920802A0920902B0920A022091E00485
:103FF0003091E1044091E2045091E304C501B40121
:104000000F94E3254B015C010F94EF2D6B017C01B4
:1040100020E030E0A9010F947D2587FDF3C020E06A
:1040200030E040E450E4C701B6010F94AD2E1816FD
:104030002CF4C12CD12CB0E4EB2EFE2CA701960160
:10404000C501B4010F944C2C6093D8047093D9042B
:104050008093DA049093DB04C701B6010F94B92D65
:104060006093D304062E000C770B6F5F7F4F643094
:10407000710514F064E070E06093D104C091D30442
:10408000D11305C0809102028C1709F470C0809191
:10409000D2049091D30490930202809301020C2EDB
:1040A000000CDD0B25E01203C0011124FC01EC0F14
:1040B000FD1FEE0FFF1FEE0FFF1FE457F84F20818B
:1040C0003181428153812093CC043093CD044093BD
:1040D000CE045093CF040091D104002E000C110B9C
:1040E000FC01E00FF11FEE0FFF1FEE0FFF1FE45763
:1040F000F84F60817181828193810F944C2C609381
:10410000C8047093C9048093CA049093CB0420918F
:10411000D00435E02303F0011124CE0FDF1FCC0FB4
:10412000DD1FCC0FDD1FC457D84F288139814A814C
:104130005B812093C4043093C5044093C60450931C
:10414000C704E00FF11FEE0FFF1FEE0FFF1FE45734
:10415000F84F60817181828193810F944C2C609320
:10416000C0047093C1048093C2049093C3048090F0
:10417000D8049090D904A090DA04B090DB04209188
:10418000C8043091C9044091CA045091CB04C501C0
:10419000B4010F94E3252091CC043091CD044091DB
:1041A000CE045091CF040F944D2C6B017C01C09232
:1041B000BC04D092BD04E092BE04F092BF042091F2
:1041C000C0043091C1044091C2045091C304C501A0
:1041D000B4010F94E3252091C4043091C5044091AB
:1041E000C6045091C7040F944D2CA70196010F945B
:1041F0004C2C6093B8047093B9048093BA049093E4
:10420000BB04BBCEC12CD12C760118CFCF92DF924C
:10421000EF92FF92CF93DF93EC0108960E94731DFB
:104220006B017C0120E030E0A9010F947D2520E0A6
:1042300030E0A901882359F0CE010E94191F9B018B
:10424000AC01C701B6010F94E3259B01AC01688561
:1042500079858A859B850F944C2C688779878A8716
:104260009B87DF91CF91FF90EF90DF90CF900895E3
:104270002F923F924F925F926F927F928F929F9276
:10428000AF92BF92CF92DF92EF92FF920F931F9364
:10429000CF93DF93D62FC72FFC0180809180A2801F
:1042A000B380C501B40120E831E541E050E00F944E
:1042B000C12BC9016DE671E00F94302C6B017C01BC
:1042C000C501B40120E13EE040E050E00F94C12B75
:1042D000CA01B90128E130E040E050E00F94C12B61
:1042E000362E272E062F172F8CE3482E512C612CAB
:1042F000712CC501B401A30192010F94C12BB62EFC
:10430000A72ECA01B901A30192010F94C12BCB01C1
:10431000C114D10479F1AF92BF927F936F932F9222
:104320003F92FF92EF92DF92CF928CE597E19F93BD
:104330008F93CF93DF930F9414258DB79EB70E966E
:104340000FB6F8949EBF0FBE8DBF8D2F9C2FDF91AF
:10435000CF911F910F91FF90EF90DF90CF90BF9082
:10436000AF909F908F907F906F905F904F903F9015
:104370002F900895E114F104C9F0AF92BF927F939A
:104380006F932F923F92FF92EF928CE497E19F936D
:104390008F93CF93DF930F941425EDB7FEB73C9620
:1043A0000FB6F894FEBF0FBEEDBFCFCF012BB9F013
:1043B000AF92BF927F936F932F923F9280E497E1E9
:1043C0009F938F93CF93DF930F9414258DB79EB750
:1043D0000A960FB6F8949EBF0FBE8DBFB6CF892B3D
:1043E000A9F0AF92BF927F936F9388E397E19F9379
:1043F0008F93CF93DF930F941425EDB7FEB73896C4
:104400000FB6F894FEBF0FBEEDBF9FCFAF92BF9225
:1044100084E397E19F938F93CF93DF930F941425B9
:104420000F900F900F900F900F900F908ECFEF92F4
:10443000FF920F931F93CF93DF93CDB7DEB78C011D
:10444000EDB6FEB60F94CA2401962DB73EB7281BD1
:10445000390B0FB6F8943EBF0FBE2DBF8DB79EB778
:104460000196B8010F94C3240E9486F90FB6F89400
:10447000FEBE0FBEEDBEDF91CF911F910F91FF9059
:10448000EF9008958C38910514F08CE890E09093AB
:104490007F1180937E110C947BBEAB01BC014093D5
:1044A000291450932A1460932B1470932C1481E9CF
:1044B00095E10C9433AF2F923F924F925F926F929F
:1044C0007F928F929F92AF92BF92CF92DF92EF92A4
:1044D000FF920F931F93CF93DF93CDB7DEB7609713
:1044E0000FB6F894DEBF0FBECDBF8B876C87042F4D
:1044F000122F282F30E03E872D87462F50E05A8715
:10450000498785E0982E929EC001939E900D1124BC
:10451000988B8F87FA01E80FF91FEE0FFF1FEE0F40
:10452000FF1FE457F84F60817181828193819B0165
:10453000AC010F943F2F882309F445C14B85400FF0
:104540006C85610F949EC0011124E985FA85E80FFE
:10455000F91FEE0FFF1FEE0FFF1FE457F84FC0804B
:10456000D180E280F380040F909EA0011124E985A0
:10457000FA85E40FF51FEE0FFF1FEE0FFF1FE45744
:10458000F84F0081918082807380262F30E0EF8584
:10459000F889E20FF31FEE0FFF1FEE0FFF1FE45726
:1045A000F84F20807181798372817A8373817B8354
:1045B000610F70E0EF85F889E60FF71FEE0FFF1F20
:1045C000EE0FFF1FE457F84FF88BEF87F081FC8365
:1045D000EF85F889F181FD83EF85F889F281FE830B
:1045E000EF85F889F381FF83FC01E20FF31FEE0FE3
:1045F000FF1FEE0FFF1FE457F84F20812887A1808F
:10460000B2806380FA01E60FF71FEE0FFF1FEE0F77
:10461000FF1FE457F84F4080518032801381202FD4
:10462000392D482D572D602F792D882D972D0F94DA
:104630003F2F882321F000E0912C812C712C9601D2
:10464000A701B601C7010F943F2F882321F0C02E88
:10465000D92CE82CF72C2C813D814E815F816C8117
:104660007D818E819F810F943F2F882321F01C82B2
:104670001D821E821F82222D39814A815B81622D1B
:1046800079818A819B810F943F2F882339F02C8078
:104690003D8139834E814A835F815B839201432D43
:1046A000512FB201832D912F0F943F2F882321F09A
:1046B000412C512C312C10E028853A2D4B2D562DB4
:1046C00068857A2D8B2D962D0F943F2F882321F00E
:1046D0004886A52CB32C612E85E02D853E85829FD2
:1046E000F001839FF00D112449855A85E40FF51FD1
:1046F000EE0FFF1FEE0FFF1FE457F84FFA87E98711
:104700009601A701B601C7010F944D2C202F392D1A
:10471000482D572D0F944C2C6B017C01222D398193
:104720004A815B81622D79818A819B810F944D2C16
:104730002C813D814E815F810F944C2C9B01AC01FB
:10474000C701B6010F944D2C6B017C0128853A2DD1
:104750004B2D562D68857A2D8B2D962D0F944D2C33
:104760009201432D512F0F944C2C9B01AC01C7019A
:10477000B6010F944D2C20E030E040E450E40F945B
:10478000472DE985FA8560837183828393836C85E5
:104790008B8560960FB6F894DEBF0FBECDBFDF915C
:1047A000CF911F910F91FF90EF90DF90CF90BF902E
:1047B000AF909F908F907F906F905F904F903F90C1
:1047C0002F900C9419F860960FB6F894DEBF0FBEC8
:1047D000CDBFDF91CF911F910F91FF90EF90DF90B0
:1047E000CF90BF90AF909F908F907F906F905F9091
:1047F0004F903F902F90089580910305909104056C
:10480000009731F04AE050E070E060E00D949823AA
:1048100060E070E0CB01089580910305909104055C
:10482000009731F04AE050E070E060E00D946A22B9
:1048300060E070E0CB010895CF93DF93EB010E941D
:104840007C1E882319F00E940C24EB01CE01DF911D
:10485000CF9108950E940C2497FD0CC00E940C2457
:104860006F3F71058105910509F034F40E940C2415
:10487000862F089580E008958FEF0895CF93C62F77
:104880000E947C1E882319F0CF910C942A248C2F2F
:10489000CF9108958091030590910405892B41F0F3
:1048A0000E942A2491E0811101C090E0892F08958F
:1048B00091E0FCCFCF93DF93C82FD62F0E947C1EB0
:1048C000882321F0DF91CF910C944A248C2F0E94F1
:1048D0002E1E811101C08D2FDF91CF9108950E946E
:1048E0000C24CB010895CF93DF93EB010E947C1E33
:1048F000882321F0DF91CF910C946F24CE01DF91BA
:10490000CF9108950F931F93CF93809103059091BA
:1049100004050097E9F0FC018F01C1912C2F2F7D38
:1049200081F0C53411F0C536B9F7F801108270E096
:1049300060E00F940C21F801C083CF911F910F917B
:10494000089570E060E0CF911F910F910D940C21BC
:1049500060E070E0CB01F1CFCF92DF92EF92FF9257
:104960006A017B010E947C1E882331F0FF90EF904A
:10497000DF90CF900C948224C701B601FF90EF9096
:10498000DF90CF9008954F925F926F927F928F92B7
:104990009F92AF92BF92CF92DF92EF92FF921F93BE
:1049A000CF93DF9300D01F92CDB7DEB719821A8262
:1049B0001B821C82CE0101964C0180E7C82E87E045
:1049C000D82E94E2E92E9CE0F92E2CECA22E28E0C1
:1049D000B22E10E088E5810F0E947C1EF4018193C5
:1049E0004F01882309F4E0C00E9482242B013C017E
:1049F000812F0E94531D882309F4CCC0F701208128
:104A0000318142815381C301B2010F944D2CF601D3
:104A100060837183828393831F5FF4E0CF0ED11C88
:104A200084E0E80EF11C94E0A90EB11C133091F65D
:104A300085E40E947C1E8C83882309F4C0C00E94F8
:104A400082246B017C0183E00E94531D882371F056
:104A50002091300C3091310C4091320C5091330C3C
:104A6000C701B6010F944D2C6B017C01C0927C07ED
:104A7000D0927D07E0927E07F0927F078091C90572
:104A8000882359F180912D1482FF27C08C818823BF
:104A900021F18981811103C08A818823F1F02DECF5
:104AA0003CEC4CE45DE3609117087091180880912C
:104AB000190890911A080F944D2C9B01AC0160913C
:104AC0002C0C70912D0C80912E0C90912F0C0F942A
:104AD000AD2E181614F40E945FF740E050E0BA01C2
:104AE00086E40E94AC2420E030E0A9010F94AD2EB2
:104AF000181684F40E94822420E030E040E752E45B
:104B00000F94472D609341027093420280934302B9
:104B1000909344028091E20B83FD28C080918F0620
:104B2000882321F12091300C3091310C4091320CCE
:104B30005091330C60917C0770917D0780917E07C6
:104B400090917F070F944C2C20919C0630919D06EC
:104B500040919E0650919F060F944D2C60939C06A9
:104B600070939D0680939E0690939F060F900F90E2
:104B70000F900F90DF91CF911F91FF90EF90DF90FA
:104B8000CF90BF90AF909F908F907F906F905F90ED
:104B90004F900895F5012081318142815381C301F5
:104BA000B2010F944C2C33CFF70180819181A28107
:104BB000B381F60180839183A283B3832DCF80914B
:104BC000300C9091310CA091320CB091330C809349
:104BD0007C0790937D07A0937E07B0937F074ECF0D
:104BE000CF92DF92EF92FF926B017C0183E3C816B4
:104BF000D104E104F10470F082E3C81AD108E1089D
:104C0000F10862E370E080E090E00E9424FD0E94E1
:104C1000F5C1ECCFC701B6010E9424FDFF90EF90D3
:104C2000DF90CF900C94F5C1CF92DF92EF92FF927C
:104C30000F931F93CF93DF936B017A01EC01C8565A
:104C4000DB4F28813CE0389F8001399F100D1124F3
:104C500027FF24C0FB011182108288818F5F888327
:104C600088819801280F311D87FD3A95C90120914F
:104C70007012F6012817190629F024F088818C306B
:104C80000CF43CC080819181049680349C4908F4E6
:104C900075C0F60180819181049672C08881980167
:104CA000280F311D87FD3A95C901209170122817F0
:104CB000190699F294F28881A801480F511D87FDC9
:104CC0005A95FA01EE0FFF1FE40FF51FE85DFD4E48
:104CD000808187FFC2CF8881F801E80FF11D87FD31
:104CE000FA95CF01EE0FFF1FE80FF91FE85DFD4EAB
:104CF000808160E08F770E94C2FBAFCF808191817D
:104D00002881A801420F511D27FD5A959A01FA01E9
:104D1000EE0FFF1FE20FF31FE85DFD4E2181328190
:104D2000820F931FF7019183808388819801280F58
:104D3000311D87FD3A95F901EE0FFF1FE20FF31FBA
:104D4000E85DFD4E808187FF20C08881080F111D1E
:104D500087FD1A95F801EE0FFF1FE00FF11FE85DC8
:104D6000FD4E808161E08F77DF91CF911F910F9190
:104D7000FF90EF90DF90CF900C94C2FB80E49CE911
:104D8000F701918380838FEF8883DF91CF911F910B
:104D90000F91FF90EF90DF90CF9008950F931F93A6
:104DA000CF93DF930EE41CE0C2E6D1E1F80121913C
:104DB0003191419151918F0160E070E080E89FE373
:104DC0000F94472D6993799389939993F1E1C237B1
:104DD000DF0761F70E949EF5DF91CF911F910F9140
:104DE0000C94991BCF92DF92EF92FF92CF93DF93B7
:104DF0002091350C222329F1EC0108960E94731DA5
:104E00006B017C0120E030E0A9010F947D2520E0BA
:104E100030E0A901882359F0CE010E94191F9B019F
:104E2000AC01C701B6010F94E3259B01AC01688575
:104E300079858A859B850F944D2C688779878A8729
:104E40009B87DF91CF91FF90EF90DF90CF900895F7
:104E50002F923F924F925F926F927F928F929F928A
:104E6000AF92BF92CF92DF92EF92FF920F931F9378
:104E7000CF93DF93CDB7DEB76C970FB6F894DEBF54
:104E80000FBECDBF8C015B015A834983FC01EA5BF5
:104E9000FF4F208131814281538129873A874B8797
:104EA0005C87CA01B9010F9482256B017C01D50191
:104EB0002D913D914D915C910F94E3250F942B2DF5
:104EC0002B013C01E981FA812081318142815381AA
:104ED000C701B6010F94E3250F942B2D4B015C0104
:104EE000C301B2010F94C02D698B7A8B8B8B9C8B85
:104EF000683771058105910540F428E730E040E00E
:104F000050E0298B3A8B4B8B5C8BC501B4010F941D
:104F1000C02D6D877E878F87988B683771058105D7
:104F2000910540F448E750E060E070E04D875E870F
:104F30006F87788BF801EE5AFF4F40805180628076
:104F40007380C301B2010F94842569837A838B83B4
:104F50009C8369897A898B899C890F9482256D8BC2
:104F60007E8B8F8B988F20E030E0A90169817A8158
:104F70008B819C810F947D25882309F4E1C1A701D1
:104F80009601C701B6010F94E3254B015C012D8901
:104F90003E894F89588DCA01B9010F94E3259B01C1
:104FA000AC01C501B4010F944C2C4B015C0129816B
:104FB0003A814B815C81CA01B9010F944D2C9B0150
:104FC000AC01C501B4010F94472D0F942B2D0F9404
:104FD000C02D6D837E838F83988766277727CB01CB
:104FE00064197509860997090F9484254B015C01A2
:104FF0006D857E858F8598890F9482252B013C01D4
:1050000020E030E0A901C501B4010F947D2588237B
:1050100009F49AC1A3019201C301B2010F94E325DF
:10502000698F7A8F8B8F9C8FA7019601C701B6017C
:105030000F94E3259B01AC01698D7A8D8B8D9C8D3E
:105040000F944C2C6B017C01A5019401C501B401A6
:105050000F944D2C9B01AC01C701B6010F94472D55
:105060000F94EF2DD80195968D909D90AD90BC90AA
:105070009897750164012D813E814F815885C21A30
:10508000D30AE40AF50A0F94C02DC61AD70AE80A13
:10509000F90AF7FE8EC02D893E894F89588DCA01C5
:1050A000B9010F94E3256B017C0129813A814B8181
:1050B0005C81CA01B9010F944D2C69877A878B876F
:1050C0009C8720E030E0A90169817A818B819C81F5
:1050D0000F947D25882309F43BC1C501B4010F94C9
:1050E000822529853A854B855C850F94E325A701A8
:1050F00096010F944C2C6D837E838F839887A30138
:105100009201C301B2010F94E3259B01AC016D81B3
:105110007E818F8198850F944D2C2B013C0120E0DE
:1051200030E040E850E469817A818B819C810F9462
:10513000E3259B01AC01C301B2010F94472D0F94ED
:105140002B2D2B013C0120E030E0A9010F94AD2E66
:1051500018161CF0412C512C3201C301B2010F94DE
:10516000C02D6D837E838F83988786169706A80649
:10517000B90620F48D829E82AF82B8866D817E81D1
:105180008F8198850F94822529853A854B855C858A
:105190000F94E325A70196010F944D2C0F94FB2E3D
:1051A0000F94C02D69877A878B879C87C12CD12C5F
:1051B000760169857A858B859C8529893A894B8911
:1051C0005C89621B730B840B950B0F9482252981DC
:1051D0003A814B815C810F94472D20E034E244EF0B
:1051E00059E40F94E3250F94C02D4B015C016985B0
:1051F0007A858B859C852D853E854F855889621BD8
:10520000730B840B950B0F94822529813A814B8176
:105210005C810F94472D20E034E244EF59E40F9471
:10522000E3250F94C02D2B013C013FE6831691042A
:10523000A104B10408F090C0F401EE0FFF1FEE0FBF
:10524000FF1FE756F64E85919591A591B4918983FC
:10525000292E3A2EBD8B4FE6441651046104710489
:1052600008F083C0F201EE0FFF1FEE0FFF1FE7569D
:10527000F64E45915591659174919A01CB014D81FE
:105280005E816F817885D80199964D935D936D937A
:105290007C939C974C0D5D1D6E1D7F1DF80145A7ED
:1052A00056A767A770ABE65BFF4F49895A896B89A0
:1052B0007C894083518362837383D5968D929D92BE
:1052C000AD92BC92D897F80141AE52AE63AE74AEC7
:1052D000FD9649814083218232825D8953833496D1
:1052E000208331838283938369857A858B859C852E
:1052F000D1966D937D938D939C93D4973D962D85F8
:105300003E854F85588920833183428353836C9631
:105310000FB6F894DEBF0FBECDBFDF91CF911F91C6
:105320000F91FF90EF90DF90CF90BF90AF909F9044
:105330008F907F906F905F904F903F902F90089547
:1053400060E070E0CB0141CE60E070E0CB0188CE40
:1053500060E070E0CB01F3CEC501B4010E949B1A5E
:105360006983272E382E9D8B76CFC301B2010E9410
:105370009B1A9B0184CF8091851290918612891B84
:10538000877019F490E080E008959091821299233B
:1053900051F0833030F48FEF890F19F0809382122F
:1053A000F1CF10928212809186122CE5829FC0016B
:1053B00011248E5F964FFC01208120FDE3CF2091C8
:1053C00086122F5F277020938312309186122091CE
:1053D0008412321304C02091831220938412089502
:1053E00090916F0081E091FD02C080E0089590915E
:1053F0006F009D7F90936F00089580FF04C090918F
:105400009A0590FD8E7F81FF05C090919A05969533
:1054100090FD8D7F82FF06C090919A059695969596
:1054200090FD8B7F08958F929F92AF92BF92CF9203
:10543000DF92EF92FF92CF93DF93209145022223D8
:1054400009F49EC0EC0180919A05C82ED12CF12C54
:10545000E12C80FF2CC08090470290904802A090E1
:105460004902B0904A02288139814A815B81C50195
:10547000B4010F94AD2E181624F488829982AA8262
:10548000BB828090530290905402A0905502B0903D
:105490005602288139814A815B81C501B4010F948C
:1054A0007D2587FF04C088829982AA82BB82D701AA
:1054B000C601B695A7959795879580FF2CC08090DB
:1054C0004B0290904C02A0904D02B0904E022C8165
:1054D0003D814E815F81C501B4010F94AD2E181638
:1054E00024F48C829D82AE82BF828090570290907D
:1054F0005802A0905902B0905A022C813D814E81F1
:105500005F81C501B4010F947D2587FF04C08C82A3
:105510009D82AE82BF8282E0F694E794D794C794CE
:105520008A95D1F7C0FE2CC0C0904F02D090500297
:10553000E0905102F0905202288539854A855B85BA
:10554000C701B6010F94AD2E181624F4C886D9866B
:10555000EA86FB86C0905B02D0905C02E0905D0220
:10556000F0905E02288539854A855B85C701B601C2
:105570000F947D2587FF04C0C886D986EA86FB86FE
:10558000DF91CF91FF90EF90DF90CF90BF90AF90E1
:105590009F908F900895CF92DF92EF92FF920F939A
:1055A0001F93C12CD12C76018C0120E33CE04CE20E
:1055B0005CE068E27CE084E29CE00E949AF41F9147
:1055C0000F91FF90EF90DF90CF9008950C949EF58F
:1055D0008091A106811105C080918007882309F47C
:1055E00063C080918705659B59C081608093870562
:1055F000909103018091870591FF52C08260809352
:105600008705809187054A9B4DC0846080938705FC
:105610008091EE0580FF10C08091A20680FF0CC033
:105620008091870580FF08C08091E40681608093A7
:10563000E40680E00E9455C68091EE05869580FFC5
:1056400011C08091A206869580FF0CC080918705CD
:1056500081FF08C08091E40682608093E40681E0C7
:105660000E9455C68091EE058695869580FF1CC0E8
:105670008091A2068695869580FF16C0809180074E
:10568000882391F08091870582FF0EC08091E40607
:1056900084608093E40682E00C9455C68E7FA6CF8A
:1056A0008D7FADCF8B7FB2CF08958091A106811100
:1056B00004C080918007882331F062E070E080E0D0
:1056C00090E00C94F02508950F931F938091201182
:1056D000813019F50E9457FD0091A3051091A40592
:1056E0002091A5053091A605601B710B820B930BD1
:1056F00028EE33E040E050E00F94C12B6091A70505
:105700007091A8058091A9059091AA05620F731F59
:10571000841F951F1F910F9108956091AB057091A3
:10572000AC058091AD059091AE05D6CF10922011B9
:105730001092A3051092A4051092A5051092A6053B
:105740001092AB051092AC051092AD051092AE050B
:105750001092A7051092A8051092A9051092AA050B
:105760000895CF92DF92EF92FF92CF93DF93C62FEF
:10577000FC01C080D180E280F38020E030E0A9010C
:10578000C701B6010F947D2520E030E0A90187FD17
:1057900014C020E030E048EC52E4C701B6010F9499
:1057A000AD2E24E630E040E050E0181634F0C7019A
:1057B000B6010F94B92D9B01AC01C230A0F4D0E02A
:1057C000C350D74FAFEFB0E00F94022C24E630E087
:1057D00040E050E00F94E32B2F3F310519F010F01B
:1057E0002FEF30E02883DF91CF91FF90EF90DF9093
:1057F000CF9008958091090180FD06C080912D14FD
:1058000083FB882780F9089580E00895CF92DF9286
:10581000EF92FF92FC01C080D180E280F38066307D
:1058200019F5109213061092140610921506109294
:105830001606109217060E947BBE20E030E0A901F8
:10584000C701B6010F947D2587FF1DC0C12CD12C47
:105850007601C701B6010F94BA2ECB01FF90EF90ED
:10586000DF90CF900C9442220E94101F20E030E085
:10587000A901C701B6010F947D2587FF15C0C12C72
:10588000D12C760122C020E030E04CE053E4C70187
:10589000B6010F94AD2E1816E4F6C12CD12C9CE065
:1058A000E92E93E4F92ED5CF20E030E849ED53E41A
:1058B000C701B6010F94AD2E18163CF4C12C80E838
:1058C000D82E89EDE82E83E4F82EC701B6010F9497
:1058D000BA2ECB01FF90EF90DF90CF900C94041F75
:1058E0009091340C977081E0973009F080E0089532
:1058F0002091850520FF14C020E83EE3629FA001AF
:10590000639F500D729F500D1124CA019695879583
:1059100096958795009731F08A950000E9F70895EC
:105920000C94F0250895CF93DF931092E30B10921F
:10593000860C1092880C1092870C1092840510929D
:105940008305CFEFDFEF80912D1485FD07C00E9406
:1059500094AAD093AC12C093AB12F5CF8FEF9FEF08
:105960009093AC128093AB12DF91CF9108958F92F8
:105970009F92AF92BF92CF92DF92EF92FF920F93DE
:105980001F93CF93DF9310923805109237052FE3C2
:1059900020933205109231051092300510922F0598
:1059A0001092330510923405109235051092360589
:1059B0009C01F90190812F5F3F4F9032D1F39E34CB
:1059C000C9F4818190ED980F9A3020F08D3211F05A
:1059D0008B3281F432969F012F5F3F4F808180533D
:1059E0008A3008F47BC09F012F5F3F4F8081803257
:1059F00009F476C0F0938307E09382078F010F5F6D
:105A00001F4FC0816AE270E0C8010F949B2F00977E
:105A100031F0FC01319780818032E1F31182CD3485
:105A200029F0C43519F0C73409F04BC0F801808162
:105A30000F5F1F4F8032D1F380538A3008F041C08E
:105A4000C093320530E020E04AE0DF011196429F2A
:105A5000C001439F900D11249C0120533109808186
:105A6000280F311D87FD3A95818190ED980F9A306E
:105A7000C8F130933105209330058E3261F43296AF
:105A800090E04AE0DF0131968C9150ED580F5A308A
:105A900058F190932F05CD01DC0101964C914032D5
:105AA000D9F3CD3489F52E31310539F018F5273188
:105AB000310519F02C31310539F5B0933805A09333
:105AC0003705DF91CF911F910F91FF90EF90DF90FD
:105AD000CF90BF90AF909F908F900895F9017BCFAA
:105AE000F90181CFFD01B1CF949F800D112490ED7C
:105AF000980FC8CF2537310538F027373105E8F240
:105B0000203A83E03807C9F2D091820740E050E0A4
:105B1000BA0110E000E0C12CD12C7601C394FD0144
:105B200031968C91882309F47FC08132E1F4CD3421
:105B3000D1F420323105B9F4409333055093340544
:105B40006093350570933605F0933805E09337057B
:105B500063E270E0CF010F949B2F009709F4B1CF5F
:105B6000FC011082AECF81548A3108F058C0DF01A9
:105B70009D91903291F0A0EDA90FAA30E8F09E32ED
:105B800071F4918190539A30B8F00115110519F410
:105B90008F010150110990E013C0FD01E8CF9D3243
:105BA00011F09B3291F79181A0EDA90FAA3020F05E
:105BB0009E3259F79281E6CF9E2F9D1B309759F365
:105BC000A82FB0E04601570104C0880C991CAA1CFC
:105BD000BB1C8A95D2F7482959296A297B29AB5ED3
:105BE000BA4F9C9380818154DF018A3108F497CFAA
:105BF000DF018191882309F492CF90ED980F9A30BC
:105C0000B8F393ED980F923098F38B3289F3CD016E
:105C10000196EC91E03209F082CFDC01F8CF01155A
:105C2000110501F78D01DECF10933805009337057C
:105C300040933305509334056093350570933605D2
:105C400040CF4F925F926F927F928F929F92AF92CE
:105C5000BF92CF92DF92EF92FF92CF93DF9300D06B
:105C600000D01F921F92CDB7DEB75C01DB01CD9053
:105C7000DD90ED90FC90E0918012F0918112FE8316
:105C8000ED8384819581A681B78189839A83AB83D3
:105C9000BC839C01AD01C701B6010F944C2C2B01B4
:105CA0003C01F50180809180A280B380AD81BE81EE
:105CB0008D919D910D90BC91A02D8D839E83AF837E
:105CC000B88727E137EB41ED58EBC301B2010F94E0
:105CD000AD2E87FDD1C023E030E041EE53E4C30197
:105CE000B2010F947D2518160CF4C6C02D813E819B
:105CF0004F815885C501B4010F944C2C2B013C01F8
:105D000027E137EB41ED58EB0F94AD2E87FDB4C082
:105D100023E030E041EE53E4C301B2010F947D254E
:105D200018160CF4A9C020E030E0A9016D817E8135
:105D30008F8198850F944D2C2B013C0120E030E0A1
:105D400040E450E40F947D2587FF05C0412C512C81
:105D500030E4632E762C27E137EB41ED58E3C301A5
:105D6000B2010F944C2C9B01AC01C501B4010F94FE
:105D7000AD2E87FD81C020E030E041EE53E46D811F
:105D80007E818F8198850F944D2C2B013C0120E062
:105D900030E84FED53E40F94AD2E18163CF4412C2F
:105DA00020E8522E2FED622E23E4722E27E137EBEE
:105DB00041ED58E3C301B2010F944D2C9B01AC019E
:105DC000C501B4010F947D2518160CF455C020E0D0
:105DD00030E0A90169817A818B819C810F944D2CDF
:105DE0004B015C0120E030E040E951E40F947D2557
:105DF00087FF06C0812C912C90E9A92E91E4B92E41
:105E000027E137EB41ED58E3C501B4010F944C2C69
:105E10009B01AC01C701B6010F94AD2E87FD2CC0CC
:105E200020E030E041EE53E469817A818B819C81EE
:105E30000F944D2C4B015C0120E030E048ED53E421
:105E40000F94AD2E181634F4812C912C88EDA82EC9
:105E500083E4B82E27E137EB41ED58E3C501B401E7
:105E60000F944D2C9B01AC01B1E0B983C701B60181
:105E70000F947D2518160CF41982898128960FB687
:105E8000F894DEBF0FBECDBFDF91CF91FF90EF90B2
:105E9000DF90CF90BF90AF909F908F907F906F904A
:105EA0005F904F900895EEE0F8E082EBDF011D92E5
:105EB0008A95E9F708958091C905811104C00E946F
:105EC000532F0C94F5B780912D1482FD0C945FF73D
:105ED000089580910E08882361F09091BF0889137E
:105EE00008C080912D1483FF04C08CE498E00C94CA
:105EF000BFB680E00895FC01238121110C94F4B217
:105F00000895EFE6F0E08081826080830895CF926B
:105F1000DF92EF92FF92CF93DF93C82F0E94F02978
:105F200094E0C99FE0011124FE01E450FA4FC080C3
:105F3000D180E280F38081110E94812FCE59DE4E04
:105F4000C701B6010F948425288139814A815B817C
:105F50000F94E325DF91CF91FF90EF90DF90CF90EA
:105F600008958F929F92AF92BF92CF92DF92EF925D
:105F7000FF921F93CF93DF93CDB7DEB760970FB635
:105F8000F894DEBF0FBECDBF182F80E00E94872F90
:105F90004B015C018092880590928905A0928A0548
:105FA000B0928B0581E00E94872F6B017C01C0922B
:105FB0008C05D0928D05E0928E05F0928F0582E0DF
:105FC0000E94872F609390057093910580939205AE
:105FD000909393051D861E861F86188A89829A8251
:105FE000AB82BC82CD82DE82EF82F88669877A87B7
:105FF0008B879C8783E00E94872F6D877E878F87A2
:10600000988B8091350C882321F0CE0101960E9457
:1060100006211E3FD9F480E1FE013196A4E2BCE0E6
:1060200001900D928A95E1F760960FB6F894DEBF65
:106030000FBECDBFDF91CF911F91FF90EF90DF900A
:10604000CF90BF90AF909F908F90089584E0189F5D
:10605000F0011124DF01AC5DB34F81E090E08C0FC3
:106060009D1FE80FF91F40815181628173814D931B
:106070005D936D937C931397D7CFCF92DF92EF927E
:10608000FF92CF93DF93C82F0E94F02994E0C99F1D
:10609000E0011124FE01E051FA4FC080D180E2807E
:1060A000F38081110E94812FCE59DE4EC701B601C7
:1060B0000F948425288139814A815B810F94E325DF
:1060C000DF91CF91FF90EF90DF90CF9008950E94E5
:1060D000F029909186129093851290938412909358
:1060E000831294E69093821220ED33E030930109FD
:1060F0002093000981110E94812F81E08093EF0598
:106100000895CF93DF93CDB7DEB72C970FB6F894F1
:10611000DEBF0FBECDBF0E947CF60E94F0299CE03E
:10612000ECEFF5E0DE01119601900D929A95E1F702
:1061300081110E94812FCE0101960E9435C62C96B6
:106140000FB6F894DEBF0FBECDBFDF91CF9108959B
:106150002F923F924F925F926F927F928F929F9277
:10616000AF92BF92CF92DF92EF92FF920F931F9365
:10617000CF93DF9300D0CDB7DEB78090240C909002
:10618000250CA090260CB090270C4090280C509025
:10619000290C60902A0C70902B0CC0902C0CD09085
:1061A0002D0CE0902E0CF0902F0C0E94991B0E9459
:1061B000E71B09E71CE187E492E09B838A838DE675
:1061C000282E8CE1382E198289810E948A1CC801F0
:1061D0000E946D1DEA81FB8161937193819391937C
:1061E000FB83EA83C1010E946D1DEA81FB81608708
:1061F000718782879387F981FF5FF9830C5F1F4F57
:1062000084E0280E311CF330F9F68AED95E00E9407
:10621000E1F60E94891E0E94CE26A501940160919C
:10622000240C7091250C8091260C9091270C0F94D2
:106230007D2581111CC0A30192016091280C7091F1
:10624000290C80912A0C90912B0C0F947D258111A3
:106250000EC020912C0C30912D0C40912E0C5091A1
:106260002F0CC701B6010F947D258823B9F00F903C
:106270000F900F90DF91CF911F910F91FF90EF90B2
:10628000DF90CF90BF90AF909F908F907F906F9056
:106290005F904F903F902F900C9481300F900F9013
:1062A0000F90DF91CF911F910F91FF90EF90DF90B2
:1062B000CF90BF90AF909F908F907F906F905F90A6
:1062C0004F903F902F900895809176119091771183
:1062D000892B79F48091761190917711892B49F46B
:1062E000209176113091771181E0232B19F480E011
:1062F000089581E008951092E9048091220290911E
:106300002302A0912402B09125028093E605909388
:10631000E705A093E805B093E905089590918D11E4
:1063200010928D11923071F0943079F0913099F48F
:10633000813089F48091E904882369F01092260263
:106340000C947B311092230C089580E898E190938F
:10635000830C8093820C089590912D1493FB8827D1
:1063600080F993FF06C081E090919415911101C0CE
:1063700080E00895CF93C0918605CF7739F50E94CC
:10638000AC31882319F18091251490912614A091A5
:106390002714B09128140097A105B105B9F0BC01EC
:1063A000CD016D597F4F8F4F9F4F24E630E040E085
:1063B00050E00F94C12B6091291470912A148091A0
:1063C0002B1490912C140F94C12BC22F8C2FCF9192
:1063D0000895EDEFF8E010821182089581E00895AC
:1063E000DC01EC918E2F90E0FC01EE0FFF1FE80F17
:1063F000F91FE85DFD4E80818F77808308958F922D
:106400009F92AF92BF92CF92DF92EF92FF920F9343
:10641000CF93DF931F92CDB7DEB75C017B014901BB
:106420006B01C40ED51EF501808191810F949B2BC9
:106430008983002311F0F7018083BE016F5F7F4FD6
:10644000C4010E94FFE0F501808191810196918352
:106450008083FFEFEF1AFF0AEC14FD0421F780E0C0
:106460000F90DF91CF910F91FF90EF90DF90CF9041
:10647000BF90AF909F908F9008950F93AB010091C4
:10648000DE0521E002272FED35E0BC018FEB95E022
:106490000E94FF310F910895009781F410929000AF
:1064A00082E0809391001092950010929400C19A1E
:1064B000809171008260809371000895019761F46A
:1064C0001092A00082E08093A1001092A50010928B
:1064D000A40089BB8093720008957F928F929F924F
:1064E000AF92BF92CF92DF92EF92FF920F931F93E2
:1064F000CF93DF93EC017B018881883108F0C3C022
:1065000090E0FC01EE0FFF1FE80FF91FE85DFD4E64
:1065100080818F770E9447E719821A8288812CE058
:10652000622F0F94242C829FB001112430E020E0D0
:10653000AB01420F531FFA01EE0FFF1FE40FF51FCF
:10654000E85DFD4E908197FD08C02F5F3F4F2C30D6
:10655000310571F790E00E944C327880072D10E0F1
:106560006801CC0CDD1CF601E00FF11FE85DFD4E6B
:1065700080818068808377FC86C080E2E81682E0B4
:10658000F8060CF03FC08A8128E532E0281B31096B
:1065900087FD3395220F331F220F331F032E000C6C
:1065A000440B550B898178E8872E912C881A910825
:1065B00087FD9394880C991C880C991C092C000C5D
:1065C000AA08BB0860E070E0CB01F7FC0AC0B70185
:1065D000653B710514F064EB70E0072E000C880B2E
:1065E000990B281939094A095B090F94B12B24EB3F
:1065F00030E040E050E00F94E32B820E931EA41E87
:10660000B51E740187E18715D8F0298188E890E0EC
:10661000821B910927FD9395880F991F880F991F59
:10662000E816F90604F502972FB7F894E601C00FB3
:10663000D11FC85DDD4E880F991F9A8389832FBFB4
:1066400062E370E080E090E0DF91CF911F910F91C5
:10665000FF90EF90DF90CF90BF90AF909F908F9082
:106660007F900C94F0252A8188E592E0821B9109A5
:1066700027FD9395880F991F880F991FE816F90633
:1066800094F6C701D0CFDF91CF911F910F91FF906A
:10669000EF90DF90CF90BF90AF909F908F907F90C2
:1066A0000895CF93DF93EB01682F70E081E792E1CB
:1066B0000E946D32688179818A819B81643F21E0EB
:1066C00072078105910520F464EF71E080E090E0AD
:1066D0000E94F02589B182FB882780F9DF91CF9154
:1066E0000895CF93DF9300D01F92CDB7DEB78EEE23
:1066F00092E0A0E0B0E089839A83AB83BC83BE01C3
:106700006F5F7F4F8AE50E9451330F900F900F907B
:106710000F90DF91CF910895CF93DF9300D01F9218
:10672000CDB7DEB78EEE92E0A0E0B0E089839A8329
:10673000AB83BC83BE016F5F7F4F8AE00E94513301
:106740000F900F900F900F90DF91CF910895CF93FE
:10675000DF9300D01F92CDB7DEB784EF91E0A0E0C9
:10676000B0E089839A83AB83BC83BE016F5F7F4FA8
:1067700080EA0E9451330F900F900F900F90DF919D
:10678000CF9108951F920F920FB60F9211240BB65E
:106790000F922F933F934F935F936F937F938F93BA
:1067A0009F93AF93BF93EF93FF9348EA50E064EA5F
:1067B00070E081E090E00E941426FF91EF91BF917C
:1067C000AF919F918F917F916F915F914F913F9189
:1067D0002F910F900BBE0F900FBE0F901F9018952A
:1067E0001F920F920FB60F9211240BB60F922F9398
:1067F0003F934F935F936F937F938F939F93AF9349
:10680000BF93EF93FF9348E950E064E970E090E0B4
:1068100080E00E941426FF91EF91BF91AF919F916C
:106820008F917F916F915F914F913F912F910F9039
:106830000BBE0F900FBE0F901F9018959091D10036
:1068400095FD0CC09091D00095FF08C08093D600B4
:106850008091D00080648093D00008952091160428
:106860002F5F2F770FB607FC27C090911704921364
:1068700028C09091D00095FF1EC0909117044091C0
:106880001604941306C09091D1009F7D9093D1007F
:1068900012C0E92FF0E0EA5EFB4F32819F5F9F77E5
:1068A0003093D600909317043091D0003064309329
:1068B000D000491741F3D9CF90911704921301C02A
:1068C000FBCFE0911604F0E0EA5EFB4F8283209359
:1068D00016048091D10080628093D10008958F9238
:1068E0009F92AF92BF92CF92DF92EF92FF920F935F
:1068F0001F93CF93DF937C0121E5E20EF11CD701BA
:106900004C914A3509F0A4C06C01B2E5CB0ED11C04
:10691000F6013081353A09F09BC0EC01C05BDF4FD6
:106920002881233008F494C08C0100561F4FD801F1
:106930004C93E15BFF4F308331962083EF54F10994
:106940003081E05BFF4F30833038B1F43196AC5486
:10695000B1093C913083E854F109AF5ABF4F50E080
:1069600040E02250330B42175307CCF4808132961B
:106970008D934F5F5F4FF7CF233031F5313809F0FA
:1069800074C0FC01EC55FF4FDC01AC5ABF4F2C9199
:1069900020833196885A9F4FDC018C918083480177
:1069A000B12CA12C888190E002968A159B050CF4ED
:1069B0003FC0F40181914F010E941E340E9415E1F5
:1069C000FFEFAF1ABF0AEECF323821F5FC01EC5AC7
:1069D000FF4F30814181E05BFF4F40833196308330
:1069E000DC01AA55BF4F50E040E02350330B421763
:1069F0005307ACF6FA01EE7FE45AFF4FE80FF91F98
:106A0000608171817C9311966C9311974E5F5F4FFB
:106A10001296EDCF243019F6333809F6FC01EC5A02
:106A2000FF4F20813181E05BFF4F30833196B0CF43
:106A300080E5DE011D928A95E9F78AE1F80111925D
:106A40008A95E9F78AE5D7018C9385EAF601808378
:106A5000DF91CF911F910F91FF90EF90DF90CF903A
:106A6000BF90AF909F908F900895323809F097CFE4
:106A7000ADCFAF92BF92CF92DF92EF92FF920F9382
:106A80001F93CF93DF93EC0184E6C82E80E2D82ECB
:106A9000E12CF12C02E8A12C90E2B92E15E0009334
:106AA000BA13C092BB13D092BC13E092BD13F09204
:106AB000BE13B092C413A092C3131093B71387E60A
:106AC00093E10E946F348FEFC81AD80AE80AF80AD7
:106AD00088E7C81680E2D806E104F10401F724E64D
:106AE00030E240E050E0BE0187E693E1DF91CF91D4
:106AF0001F910F91FF90EF90DF90CF90BF90AF90DC
:106B00000C941AE1CF92DF92EF92FF920F931F93B2
:106B1000CF93DF93CDB7DEB77C01CDB6DEB60F9451
:106B2000CA2401962DB73EB7281B390B0FB6F8942F
:106B30003EBF0FBE2DBF0DB71EB70F5F1F4FB70172
:106B4000C8010F94C324F80101900020E9F73197A0
:106B5000E01BF10B759720F08BE792E0F801848B36
:106B6000C8010E9439350FB6F894DEBE0FBECDBE07
:106B7000DF91CF911F910F91FF90EF90DF90CF9019
:106B800008958F929F92AF92BF92CF92DF92EF9231
:106B9000FF920F931F93CF93DF930E94932C3AE0C1
:106BA000C32E30E2D32EE12CF12C15E002E8460191
:106BB0005701CAE0D0E01092C4131092C31310938F
:106BC000B7130093BA138092BB139092BC13A09298
:106BD000BD13B092BE1387E693E10E946F342197F4
:106BE0008FEF881A980AA80AB80A209721F78AE036
:106BF000C80ED11CE11CF11C82EDC81680E2D8063B
:106C0000E104F104A1F6C12C20E2D22EE12CF12CFA
:106C1000D5E0C2E81092C4131092C313D093B713F7
:106C2000C093BA13C092BB13D092BC13E092BD13B1
:106C3000F092BE1387E693E10E946F341092C41362
:106C40001092C313D093B713C093BA13D701C601E0
:106C50008C529F4FAF4FBF4F8093BB139093BC1389
:106C6000A093BD13B093BE1387E693E10E946F34E7
:106C70008FEFC81AD80AE80AF80A8AE0C81680E234
:106C8000D806E104F10431F69EEDC92E90E2D92E2A
:106C9000E12CF12CD5E0C2E81092C4131092C3137A
:106CA000D093B713C093BA13C092BB13D092BC1346
:106CB000E092BD13F092BE1387E693E10E946F3419
:106CC0008FEFC81AD80AE80AF80A86EEC81680E2DA
:106CD000D806E104F10401F7CC24C39482E1D82E54
:106CE000E12CF12C0AE010E0D5E0C2E81093C413C7
:106CF0000093C313D093B713C093BA13C092BB13BE
:106D0000D092BC13E092BD13F092BE1387E693E1DC
:106D10000E946F341093C4130093C313D093B7131E
:106D2000C093BA13D701C6018096A11DB11D8093EF
:106D3000BB139093BC13A093BD13B093BE1387E60F
:106D400093E10E946F348FEFC81AD80AE80AF80A54
:106D500085E1C81682E1D806E104F10439F682E142
:106D600090E09093C4138093C313D093B713C09350
:106D7000BA1384E190E1A0E0B0E08093BB1390935C
:106D8000BC13A093BD13B093BE1387E693E1DF91CC
:106D9000CF911F910F91FF90EF90DF90CF90BF9018
:106DA000AF909F908F900C946F341F920F920FB6FC
:106DB0000F9211240BB60F922F938F939F93EF9303
:106DC000FF938091170420911604821306C08091CE
:106DD000D1008F7D8093D10012C0E82FF0E0EA5EF1
:106DE000FB4F92818F5F8F779093D600809317042B
:106DF0009091D00090649093D000281741F3FF91B8
:106E0000EF919F918F912F910F900BBE0F900FBE1E
:106E10000F901F9018951F920F920FB60F9211248A
:106E20000BB60F920F931F932F933F934F935F9344
:106E30006F937F938F939F93AF93BF93CF93DF9382
:106E4000EF93FF93C091D60000913A05D091390598
:106E500011E01D0F1F7390911504913108F09FC030
:106E6000E92FF0E08827E85CF84C8F4F0D94442C14
:106E700049377837873796379D37CF37A137CF37A0
:106E8000A537A937CF37AD37B137B537BC37CF378F
:106E9000C737C03229F028F5CA3011F0CD3031F5AE
:106EA000011731F0ED2FF0E0E75CFA4FC283D12FEC
:106EB000D0933905FF91EF91DF91CF91BF91AF91C1
:106EC0009F918F917F916F915F914F913F912F9102
:106ED0001F910F910F900BBE0F900FBE0F901F9040
:106EE0001895CD3481F081E0CE3471F080E10CC092
:106EF000CA3338F4C033A0F6C03291F2CD32B1F7C4
:106F0000CFCFCD3499F782E080931504C9CFC13338
:106F100059F018F4C03221F2E9CF88E0C433A1F36C
:106F20008BE0C83389F3E2CF83E0EECF84E0C03357
:106F300059F386E0C13341F3D9CF85E0C833B1F6C8
:106F4000E3CF87E0C23391F6DFCF89E0C13371F63A
:106F5000DBCF8AE0C03351F6D7CF8CE0C73331F6B0
:106F6000D3CF8DE0C63311F6CFCFC03209F498CF1E
:106F70008EE0C33549F2BACF80ED8C0F8A3008F02D
:106F80008FCF9FE0909315048093140489CFCA306B
:106F900019F0CD3009F084CF1092150481CFCA309A
:106FA00019F0CD3009F07CCF809121148823A1F312
:106FB000973089F038F4953079F710923C021092AE
:106FC000230CEACF9A3059F09F3031F780911404A6
:106FD0000E948E31E1CF81E080930D06DDCF81E00C
:106FE00080930C06D9CF9091C00095FFFCCF809381
:106FF000C6000895CF93DF93EC018991882319F09F
:107000000E94F337FACF8DE00E94F3378AE0DF91D8
:10701000CF910C94F337CF92DF92EF92FF92CF9300
:107020006B017C01C42F4A3069F4F7FE0BC0F09469
:10703000E094D094C094C11CD11CE11CF11C8DE2E1
:107040000E94F3374C2FC701B601CF91FF90EF900C
:10705000DF90CF900C942DAACF93DF93EC01FE012B
:1070600084912196882319F00E94F337F8CFDF919D
:10707000CF910895CF93DF93D091201185E59CE1C6
:107080000E942C388AE00E94F33780919F0C873051
:1070900009F449C083E080939D0C81E080936E02E7
:1070A00080E190E09093C4138093C31385E08093B4
:1070B000B713C2E8C093BA1384E190E1A0E0B0E056
:1070C0008093BB139093BC13A093BD13B093BE13D6
:1070D00087E693E10E946F3461E070E080E090E029
:1070E0000E94782C81E09AE59093C4138093C31397
:1070F00085E390E09093C6138093C51387E0809357
:10710000B713C093BA1384E890E0A0E0B0E0809396
:10711000BB139093BC13A093BD13B093BE1387E62B
:1071200093E10E946F3480912011813089F1823087
:1071300061F50E94642B6093A7057093A805809366
:10714000A9059093AA0581E0809320110E9457FD24
:107150006093A3057093A4058093A5059093A6055D
:10716000D23089F08091900690919106019690938B
:107170009106809390061092AF051092B005109280
:10718000B1051092B20581E004C00E94962BDBCFBE
:1071900080E0DF91CF910895CF93C82FCB010E945B
:1071A0002C3889EC98E10E942C388AEB98E1CC23AA
:1071B00011F08FEB98E10E942C388AE0CF910C946B
:1071C000F337CF93DF9300D01F92CDB7DEB784EFB4
:1071D00091E0A0E0B0E089839A83AB83BC83BE01D9
:1071E0006F5F7F4F8CE30E94513387EE98E10E94DE
:1071F0002C388CB161EE78E185FB882780F90E94FC
:10720000CC38809103016BED78E1869581700E9406
:10721000CC3889B165ED78E182FB882780F90E943E
:10722000CC388CB16CEC78E1829581700E94CC38BE
:107230004A9909C00E948C330F900F900F900F90C5
:10724000DF91CF9108950E9471330F900F900F90AE
:107250000F90DF91CF910895809120118130C1F579
:1072600085E998E10E942C388AE00E94F33781E09A
:107270009AE59093C4138093C31387E590E09093AD
:10728000C6138093C51387E08093B71382E8809379
:10729000BA1384E890E0A0E0B0E08093BB13909331
:1072A000BC13A093BD13B093BE1387E693E10E9475
:1072B0006F3482E0809320110E9457FD6093AB05EC
:1072C0007093AC058093AD059093AE0581E0089571
:1072D00080E008950F931F930E9457FD00918B0645
:1072E00010918C0620918D0630918E0601151105A6
:1072F0002105310509F067C020919912222309F474
:107300005FC0E091971221502093991221E02E0F37
:107310002093971230919A12231302C01092971261
:1073200024E0E29FF0011124E556FD4E0081118119
:107330002281338100938706109388062093890663
:1073400030938A06600F711F811D911D60938B061B
:1073500070938C0680938D0690938E06809189069B
:1073600090918A06892B61F11FB7F89484E898E11F
:107370000E942C388AE00E94F33784E096E09093D4
:10738000C4138093C31380EA90E89093C61380934C
:10739000C51387E08093B71382E88093BA1380EA1D
:1073A00090E0A0E0B0E08093BB139093BC13A09357
:1073B000BD13B093BE1387E693E10E946F341FBFE5
:1073C0001F910F910895601B710B820B930B97FD1A
:1073D000F7CF409810928B0610928C0610928D0673
:1073E00010928E06EDCF0F931F93CF93DF938C01F6
:1073F000EB019091991220919A12921305C00E946C
:107400006A390E94F5C1F5CF8091981234E0839FCC
:10741000F0011124E556FD4E11830083D383C2830E
:107420009F5F909399128F5F281739F0809398127D
:10743000DF91CF911F910F91089510929812F8CF7C
:10744000CF92DF92EF92FF921F93CF93DF93182F8B
:10745000662351F01092E8041092E4041092E504BF
:107460001092E6041092E7040E9457FD6B017C0124
:107470008091E4049091E504A091E604B091E704C2
:10748000A7019601281B390B4A0B5B0BDA01C901D6
:10749000B7FD3DC02091E80417FD13C0412F012E18
:1074A000000C550B4C5F5F4F822F022E000C990B86
:1074B0004817590764F184EF91E0A0E0B0E021178C
:1074C00024F488EE93E0A0E0B0E08C0D9D1DAE1D8D
:1074D000BF1D8093E4049093E504A093E604B09369
:1074E000E7042170C22F30E0D32F84E28C9FB001DB
:1074F0008D9F700D7C1B112460597C4F82E390E0BE
:107500000E94F3398091E8048F5F8093E804DF9153
:10751000CF911F91FF90EF90DF90CF900895CF9380
:10752000DF9300D01F92CDB7DEB78AE098E10E94CA
:107530002C388AE00E94F33780919F0C8330D9F178
:1075400019821A821B821C8260E0CE0101960E9481
:10755000B12B19821A821B821C8261E0CE01019636
:107560000E94B12B81E080936D0210929C0C80935D
:107570006E0281E09AE59093C4138093C31383E372
:1075800090E09093C6138093C51387E08093B71360
:1075900082E88093BA1384E890E0A0E0B0E08093A2
:1075A000BB139093BC13A093BD13B093BE1387E697
:1075B00093E10E946F340F900F900F900F90DF9126
:1075C000CF9108956F927F928F929F92AF92BF92C8
:1075D000CF92DF92EF92FF920F931F93CF93DF939F
:1075E000CDB7DEB764970FB6F894DEBF0FBECDBF40
:1075F0001092D0008091D00082608093D0001092D1
:10760000D50080E18093D4008091D1008061809387
:10761000D1008091D10088608093D1008091D10009
:1076200080688093D1008091D1008F7D8093D100BC
:107630008AE58093B8138093681385EA8093B91321
:1076400080936913E7E0F4E18AE1DF011D928A95F6
:10765000E9F780919B0C882309F473C283E090E0E2
:107660009093C4138093C31385E08093B71382E88B
:107670008093BA138FE190E1A0E0B0E08093BB1358
:107680009093BC13A093BD13B093BE1387E693E110
:107690000E946F3484E690E09093C4138093C313E8
:1076A00005E00093B71312E81093BA1386E090E157
:1076B000A0E0B0E08093BB139093BC13A093BD13E4
:1076C000B093BE1387E693E10E946F348BE090E0A5
:1076D0009093C4138093C3130093B7131093BA13FA
:1076E00080E092E1A0E0B0E08093BB139093BC13E4
:1076F000A093BD13B093BE1387E693E10E946F344D
:107700001092C4131092C3130093B7131093BA13BB
:1077100084E390E1A0E0B0E08093BB139093BC13AE
:10772000A093BD13B093BE1387E693E10E946F341C
:107730001092C4131092C3130093B7131093BA138B
:107740008AE390E1A0E0B0E08093BB139093BC1378
:10775000A093BD13B093BE1387E693E10E946F34EC
:107760008091E7119091E8119093C4138093C31313
:107770000093B7131093BA1386E390E1A0E0B0E052
:107780008093BB139093BC13A093BD13B093BE130F
:1077900087E693E10E946F3480917C1190917D1176
:1077A0009093C4138093C3130093B7131093BA1329
:1077B0008CE390E1A0E0B0E08093BB139093BC1306
:1077C000A093BD13B093BE1387E693E10E946F347C
:1077D00082E090E09093C4138093C3130093B71397
:1077E0001093BA138EE190E1A0E0B0E08093BB1358
:1077F0009093BC13A093BD13B093BE1387E693E19F
:107800000E946F3481E080936D0270E6C72E70E1B4
:10781000D72EE12CF12C1092C4131092C3130093B5
:10782000B7131093BA13C092BB13D092BC13E0925B
:10783000BD13F092BE1387E693E10E946F34BFEF51
:10784000CB1ADB0AEB0AFB0AE4E7CE16E0E1DE0620
:10785000E104F10401F7CE0101967C0184E1D70136
:107860001D928A95E9F781E08F9396ED9F938F9310
:1078700092EC9F938F939F9389E993E09F938F93CB
:10788000FF92EF920F94D52F20E630E140E050E0D8
:1078900066EA73E087E693E10E941AE12AE630E1A6
:1078A00040E050E06EEA73E087E693E10E941AE15F
:1078B00024E730E140E050E0B70187E693E10E9421
:1078C0001AE12EE730E140E050E06AEB73E087E632
:1078D00093E10E941AE11092C4131092C313009313
:1078E000B7131093BA138EE090E1A0E0B0E080935C
:1078F000BB139093BC13A093BD13B093BE1387E644
:1079000093E10E946F341092C4131092C31300933A
:10791000B7131093BA138FE090E1A0E0B0E080932A
:10792000BB139093BC13A093BD13B093BE1387E613
:1079300093E10E946F340FB6F894DEBF0FBECDBF47
:107940004AE0C42E40E2D42EE12CF12C55E0752EF5
:1079500062E8662E460157010AE010E01092C41357
:107960001092C3137092B7136092BA138092BB1334
:107970009092BC13A092BD13B092BE1387E693E120
:107980000E946F3401501109FFEF8F1A9F0AAF0A4E
:10799000BF0A0115110511F78AE0C80ED11CE11CC0
:1079A000F11C92EDC91690E2D906E104F10491F6BA
:1079B000C12C30E2D32EE12CF12C05E012E810921C
:1079C000C4131092C3130093B7131093BA13C09249
:1079D000BB13D092BC13E092BD13F092BE1387E6A6
:1079E00093E10E946F341092C4131092C31300935A
:1079F000B7131093BA13D701C6018C529F4FAF4FE4
:107A0000BF4F8093BB139093BC13A093BD13B0934F
:107A1000BE1387E693E10E946F34AFEFCA1ADA0A09
:107A2000EA0AFA0ABAE0CB16B0E2DB06E104F10496
:107A300031F62EEDC22E20E2D22EE12CF12C05E003
:107A400012E81092C4131092C3130093B71310934B
:107A5000BA13C092BB13D092BC13E092BD13F09244
:107A6000BE1387E693E10E946F34EFEFCE1ADE0A71
:107A7000EE0AFE0AF6EECF16F0E2DF06E104F104AC
:107A800001F7CC24C39482E1D82EE12CF12C9AE0AA
:107A9000A92EB12C05E012E8B092C413A092C31332
:107AA0000093B7131093BA13C092BB13D092BC13B8
:107AB000E092BD13F092BE1387E693E10E946F340B
:107AC000B092C413A092C3130093B7131093BA13C8
:107AD000D701C6018096A11DB11D8093BB13909361
:107AE000BC13A093BD13B093BE1387E693E10E942D
:107AF0006F348FEFC81AD80AE80AF80A95E1C91658
:107B000092E1D906E104F10439F680E797E10E9499
:107B10002C388AE00E94F33764960FB6F894DEBFE3
:107B20000FBECDBFDF91CF911F910F91FF90EF90CE
:107B3000DF90CF90BF90AF909F908F907F906F908D
:107B4000089582E090E08CCD0E94E23A1092820586
:107B500081E080936E0282E298E10E942C388AE0F4
:107B60000C94F3370F931F93CF938C01C62F8FE1A3
:107B700094E10E942C38C8010E942C388AE30E94AC
:107B8000F33780E38C0F0E94F3378AE0CF911F9187
:107B90000F910C94F33782EA95E10E942C3860E053
:107BA00082E995E10E94B23D60E08DE795E10E9497
:107BB000B23D61E086E795E10E94B23D61E08BE66F
:107BC00095E10E94B23D61E08BE595E10E94B23DF6
:107BD00060E082E595E10E94B23D61E088E495E1D4
:107BE0000E94B23D61E08EE395E10E94B23D61E00A
:107BF00087E395E10E94B23D61E08FE295E10E944A
:107C0000B23D61E081E295E10E94B23D61E083E135
:107C100095E10E94B23D60E084E095E10E94B23DB2
:107C200060E086EF94E10E94B23D60E080EE94E176
:107C30000E94B23D61E08FEC94E10E94B23D61E0B0
:107C400080EC94E10E94B23D61E089EB94E10E94F6
:107C5000B23D60E082EB94E10E94B23D61E089EACE
:107C600094E10E94B23D61E084E994E10E94B23D5A
:107C700061E086E894E10E94B23D61E083E794E12F
:107C80000E94B23D60E086E694E10E94B23D61E070
:107C900081E694E10E94B23D61E084E594E10E94B6
:107CA000B23D60E080E494E10E94B23D60E08DE28C
:107CB00094E10E94B23D60E080E394E10E94501D97
:107CC000682F617084E294E10C94B23D8091330599
:107CD000827149F4809135058C7829F480913605BC
:107CE000837009F475C082E40E942E1E882351F02F
:107CF0000E94FC2360934A0C70934B0C80934C0CB5
:107D000090934D0C83E50E942E1E882351F00E9413
:107D1000822460937A0C70937B0C80937C0C9093FC
:107D20007D0C84E50E942E1E882351F00E9482243F
:107D300060937E0C70937F0C8093800C9093810CE9
:107D400088E50E942E1E882351F00E9482246093B1
:107D5000D9087093DA088093DB089093DC0889E5F2
:107D60000E942E1E882351F00E9482246093DD0819
:107D70007093DE088093DF089093E0088AE50E9404
:107D80002E1E8823B1F00E9482246093E108709334
:107D9000E2088093E3089093E4082DEC3CEC4CEC73
:107DA0005DE30F947D25181624F088E99EE00E947B
:107DB0002C3885E40E942E1E882351F00E948224D4
:107DC0006093E5087093E6088093E7089093E808CD
:107DD0000895AF92BF92CF92DF92EF920F931F93CD
:107DE000CF93DF935B01EA016901882309F463C043
:107DF00081E99EE00E942C38F501608171818281C9
:107E0000938146E00E9435BAE1100BC088E89EE0FD
:107E10000E942C38688179818A819B8146E00E948A
:107E200035BA81E89EE00E942C38F60160817181AC
:107E30008281938143E00E9435BA8AE79EE00E94E6
:107E40002C38F801608171818281938143E00E9426
:107E500035BA81E79EE00E942C38F60120813181FD
:107E600042815381F80160817181828193810F94F5
:107E70004C2C43E00E9435BAEE20F9F08AE00E94D3
:107E8000F3378CE59EE00E942C38688179818A81E5
:107E90009B8146E00E9435BA8AE00E94F3378AE06F
:107EA000DF91CF911F910F91EF90DF90CF90BF9016
:107EB000AF900C94F337E110E4CFDF91CF911F9195
:107EC0000F91EF90DF90CF90BF90AF9008950F93F8
:107ED0001F93CF938C01C62F89E798E00E942C381E
:107EE000C8010E942C38CC2331F08AE0CF911F9139
:107EF0000F910C94F337CF911F910F9108950E9429
:107F0000AFE41092230C10923C020E94AC31882303
:107F100051F080912D1482FD06C080E898E1909385
:107F2000830C8093820C61E089E798E10E94673FAF
:107F30000C943A380F931F93CF93DF938C016F3FCC
:107F400019F41092611160E020916111862F062EC4
:107F5000000C990B2817190609F08CF56093611134
:107F600060E083E498E10E94673FC8010E942C38DA
:107F70008AE00E94F337C8010F94CA24800F911F32
:107F8000EC01C01BD10BC034D1053CF00197FC01C2
:107F90002491207C2038D1F3F3CFDD27AE01B80146
:107FA00081E291E10F94EB24CF5DDE4E188281E2F5
:107FB00091E1DF91CF911F910F910C943935DF91B1
:107FC000CF911F910F9108951092230C10923C02B3
:107FD00080912D14806480932D1461E081E598E1F7
:107FE0000E94673F46E658E16EE678E185E00E9430
:107FF00034E360E088E598E10C949A3F0F931F9377
:10800000CF938C01C62F60E083E898E00E94673F21
:10801000C8010E942C38CC2331F08AE0CF911F9107
:108020000F910C94F337CF911F910F91089561E058
:108030008BE898E00C94FE3FEF92FF920F931F9312
:10804000CF937C018B01C42F60E083E898E00E940D
:10805000673FC7010E942C3880E20E94F337C801B5
:108060000E942C38CC2319F08C2F0E94F3378AE021
:10807000CF911F910F91FF90EF900C94F337DF9207
:10808000EF92FF920F931F93CF93DF93D82E7B0134
:108090008A01E9010E941740D0928D1140E0B7019A
:1080A00084E799E00E941C400115110531F040E081
:1080B000B8018DE699E00E941C40209731F040E025
:1080C000BE018DE699E00E941C4061E088E699E0DF
:1080D000DF91CF911F910F91FF90EF90DF900C9463
:1080E000FE3FAF92BF92CF92DF92EF92FF920F933B
:1080F0001F93CF93DF9386EE97E00E942C38C0E069
:10810000D7E0D15021F080E20E94F337FACF8C2FD4
:108110000E946DE1CF5FC53099F78AE00E94F33786
:108120000CE817E0C0E080E20E94F3378C2F0E9439
:108130006DE15801D5E080E20E94F337F501C0807F
:10814000D180E280F380A7019601C701B6010F94A8
:108150003F2F882369F180E20E94F3378DE30E946C
:10816000F3378DE30E94F3378DE30E94F3378DE3FD
:108170000E94F3378DE30E94F337D150F4E1AF0E44
:10818000B11CD111D8CF8AE00E94F337CF5F0C5FCA
:108190001F4FC53041F68AE0DF91CF911F910F91BB
:1081A000FF90EF90DF90CF90BF90AF900C94F3379B
:1081B00020E030E0A901C701B6010F94AD2E87FD84
:1081C00003C08BE20E94F33743E0C701B6010E946F
:1081D00035BAD3CF811107C08AEC9EE00E942C38BB
:1081E0008AE00C94F3378EEC9EE0F8CFCF93DF93C8
:1081F000EB010E942C38CE01DF91CF910C942BE241
:10820000CF93C62F0E942C388C2FCF910C946DE108
:10821000CF92DF92EF92FF926A017B010E942C388D
:1082200042E0C701B601FF90EF90DF90CF900C9431
:1082300035BACF92DF92EF92FF926A017B010E94E2
:108240002C384AE0C701B601FF90EF90DF90CF9045
:108250000C940B38CF93DF93EB010E942C38CE01A6
:10826000DF91CF910C9474E14F925F926F927F9265
:108270008F929F92AF92BF92CF92DF92EF92FF9236
:108280000F931F93CF93DF9300D000D01F921F92C4
:10829000CDB7DEB78091810581110AC480917F0539
:1082A000909180059C012F5F3F4F30938005209374
:1082B0007F058E3E924008F4FBC38091E7119091B8
:1082C000E8119093C4138093C31305E00093B71390
:1082D00012E81093BA1386E390E1A0E0B0E0809337
:1082E000BB139093BC13A093BD13B093BE1387E64A
:1082F00093E10E946F3480917C1190917D11909355
:10830000C4138093C3130093B7131093BA138CE371
:1083100090E1A0E0B0E08093BB139093BC13A093D6
:10832000BD13B093BE1387E693E10E946F34809132
:10833000E9119091EA119093C4138093C3130093B1
:10834000B7131093BA1384E390E1A0E0B0E08093F8
:10835000BB139093BC13A093BD13B093BE1387E6D9
:1083600093E10E946F3480917E1190917F119093E0
:10837000C4138093C3130093B7131093BA138AE303
:1083800090E1A0E0B0E08093BB139093BC13A09366
:10839000BD13B093BE1387E693E10E946F3481E072
:1083A000809381051092800510927F0580919F0C2B
:1083B000882339F10E94E21C811123C080917E053F
:1083C0008F5F80937E0580917E05853620F0109228
:1083D0007E0510929F0CE0919F0CE150E73008F071
:1083E0006AC00E2E000CFF0B8827E650FE4B8F4F05
:1083F0000D94442C044253421F444B448C44C444C7
:10840000574210927E05DFCF0E94702C882309F41A
:1084100052C081E080936E028CEF97E10E942C386D
:108420008AE00E94F33780E190E09093C413809338
:10843000C31385E08093B71312E81093BA1384E155
:1084400090E1A0E0B0E08093BB139093BC13A093A5
:10845000BD13B093BE1387E693E10E946F3481E0B1
:108460009AE59093C4138093C31386E390E09093AE
:10847000C6138093C51387E08093B7131093BA1384
:1084800084E890E0A0E0B0E08093BB139093BC132D
:10849000A093BD13B093BE1387E693E10E946F349F
:1084A00010929F0C08C00E94702C882321F00E941B
:1084B000E21C8823A9F380916E02882309F433C754
:1084C000809182058111C0C284E096E09093C4132C
:1084D0008093C31380EA90E89093C6138093C513EA
:1084E00017E01093B71302E80093BA1380EA90E004
:1084F000A0E0B0E08093BB139093BC13A093BD1396
:10850000B093BE1387E693E10E946F3480916902B5
:1085100090916A02A0916B02B0916C020097A10544
:10852000B10509F03FC21092C4131092C31315E0B5
:108530001093B7130093BA138AE890E1A0E0B0E07B
:108540008093BB139093BC13A093BD13B093BE1341
:1085500087E693E10E946F3489E090E09093C41322
:108560008093C3131093B7130093BA138CE890E170
:10857000A0E0B0E08093BB139093BC13A093BD1315
:10858000B093BE1387E693E10E946F348091690235
:1085900090916A02A0916B02B0916C020097F1E099
:1085A000AF07B10508F441C2B093C413A093C3133D
:1085B0009093C6138093C51387E08093B71382E826
:1085C0008093BA1388E890E1A0E0B0E08093BB13F9
:1085D0009093BC13A093BD13B093BE1387E693E1B1
:1085E0000E946F348091690290916A02A0916B029F
:1085F000B0916C02BA2FA92F982F8827009721E0FD
:10860000A207B10508F417C2B093C413A093C31313
:108610009093C6138093C51387E08093B71312E835
:108620001093BA1381EA90E0A0E0B0E08093BB130E
:108630009093BC13A093BD13B093BE1387E693E150
:108640000E946F348091350C882309F4FAC183E0CD
:1086500090E09093C4138093C31385E08093B71385
:108660001093BA1385E490E1A0E0B0E08093BB13CF
:108670009093BC13A093BD13B093BE1387E693E110
:108680000E946F3480918205875E809382052091DD
:108690008205822F90E0253608F021C29093C41302
:1086A0008093C31385E08093B71382E88093BA1355
:1086B00080E090E1A0E0B0E08093BB139093BC1306
:1086C000A093BD13B093BE1387E693E10E946F346D
:1086D0000E94E21C811114C20E94AC31811105C0BC
:1086E0009091850591FD0E94E21C9091850580FB8B
:1086F00091F99093850591FD03C280912D1482FD1F
:10870000FFC1809120118150823008F4F9C160913D
:108710007E1170917F11072E000C880B990B0F941E
:1087200084256B017C0120E030E0A9010F947D25B8
:10873000882309F4BBC660917C1170917D11072ECE
:10874000000C880B990B0F9484252B013C0120E031
:1087500030E040E850E4C701B6010F944C2CA3016F
:1087600092010F94AD2E18160CF4C2C66091E71159
:108770007091E811072E000C880B990B0F9484253B
:108780006D837E838F8398876091E9117091EA11E0
:10879000072E000C880B990B0F9484254B015C016C
:1087A00020E030E040E251E40F944C2C2D813E81DA
:1087B0004F8158850F94AD2E18160CF499C620E001
:1087C00030E040E850E4C701B6010F944D2CA301FE
:1087D00092010F947D2587FD10C020E030E040E23B
:1087E00051E4C501B4010F944D2C2D813E814F8180
:1087F00058850F947D2587FF6AC684E190E09093A9
:10880000C4138093C31385E08093B71382E88093E9
:10881000BA1384E190E1A0E0B0E08093BB139093A1
:10882000BC13A093BD13B093BE1387E693E10E94DF
:108830006F3480919D0C81117CC682E07AC68EEEE9
:1088400097E10E942C388AE00E94F33781E09AE594
:108850009093C4138093C31380E490E09093C61365
:108860008093C51317E01093B71382E88093BA136F
:1088700084E890E0A0E0B0E08093BB139093BC1339
:10888000A093BD13B093BE1387E693E10E946F34AB
:1088900010939F0C10CE80918C0C882309F40BCE82
:1088A0000E94702C882309F406CE0E94E21C8111DC
:1088B00002CE80EE97E10E942C388AE00E94F337C6
:1088C00080918D0C90E0B0E0A0E0895B9F4FAE4FAF
:1088D000B54A21E03AE53093C4132093C313909333
:1088E000C6138093C51387E08093B71382E8809303
:1088F000BA1384E890E0A0E0B0E08093BB139093BB
:10890000BC13A093BD13B093BE1387E693E10E94FE
:108910006F3410928C0CC4CD0E94702C882309F403
:10892000CACD0E94E21C8111C6CD81E080936E0207
:1089300010929F0C82ED97E10E942C388AE00E94F1
:10894000F33781E09AE59093C4138093C3138EE4C8
:1089500090E09093C6138093C51387E08093B7137C
:1089600082E88093BA1384E890E0A0E0B0E08093BE
:10897000BB139093BC13A093BD13B093BE1387E6B3
:1089800093E10E946F3497CD0E94E21C811193CD38
:1089900019821A821B821C8262E0CE0101960E941B
:1089A000FCF47ECD0196A11DB11D35E0B695A795CD
:1089B000979587953A95D1F70197A109B109009745
:1089C000E1E0AE07B10548F1B093C413A093C3131F
:1089D0009093C6138093C5131093B71312E81093A6
:1089E000BA138AE890E1A0E0B0E08093BB139093C3
:1089F000BC13A093BD13B093BE1387E693E10E940E
:108A00006F3488E090E09093C4138093C31385E0A3
:108A10008093B7131093BA13A9CD9093C413809386
:108A2000C31385E08093B713D9CF9093C413809379
:108A3000C31385E0C2CD9093C4138093C31385E024
:108A4000ECCD82E090E005CE8A3F08F020CE8EEF9C
:108A50008093820581EC97E10E942C388AE00E9485
:108A6000F33781E080936E0281E09AE59093C4131E
:108A70008093C3138DE290E09093C6138093C51347
:108A800087E08093B71382E88093BA1384E890E07C
:108A9000A0E0B0E08093BB139093BC13A093BD13F0
:108AA000B093BE1387E693E10E946F341092810564
:108AB00028960FB6F894DEBF0FBECDBFDF91CF91E1
:108AC0001F910F91FF90EF90DF90CF90BF90AF90EC
:108AD0009F908F907F906F905F904F9008958456F5
:108AE00091099093C4138093C31385E08093B713C7
:108AF00082E88093BA1381E090E1A0E0B0E0DCCDA1
:108B00008CE090E09093C4138093C31315E010930E
:108B1000B71382E88093BA1384E190E1A0E0B0E05B
:108B20008093BB139093BC13A093BD13B093BE135B
:108B300087E693E10E946F340E94642B20E13EE0BF
:108B400040E050E00F94C12B2115310581E048072A
:108B5000510508F470C05093C4134093C31330936D
:108B6000C6132093C51387E08093B71312E81093C0
:108B7000BA1380E190E1A0E0B0E08093BB13909342
:108B8000BC13A093BD13B093BE1387E693E10E947C
:108B90006F340E94642B20E13EE040E050E00F94EF
:108BA000C12B2CE330E040E050E00F94C12B309318
:108BB000C4132093C31305E00093B7131093BA13A3
:108BC00082E190E1A0E0B0E08093BB139093BC13EE
:108BD000A093BD13B093BE1387E693E10E946F3458
:108BE0000E94BA31882309F45CC48F5F80937D05AD
:108BF000E82EF12C833330F5EE0CFF1CF092C413F9
:108C0000E092C3130093B7131093BA138EE090E170
:108C1000A0E0B0E08093BB139093BC13A093BD136E
:108C2000B093BE1387E693E10E946F341092C41391
:108C30001092C3132BC03093C4132093C31310930B
:108C4000B71394CF84E690E09093C4138093C3133A
:108C50000093B7131093BA138EE090E1A0E0B0E058
:108C60008093BB139093BC13A093BD13B093BE131A
:108C700087E693E10E946F34A2E3EA1AA0E8FA0AB9
:108C8000EE0CFF1CF092C413E092C3130093B713D1
:108C90001093BA138FE090E1A0E0B0E08093BB1393
:108CA0009093BC13A093BD13B093BE1387E693E1DA
:108CB0000E946F340E94BA3190E09093C413809365
:108CC000C31385E08093B71382E88093BA1386E1DB
:108CD00090E1A0E0B0E08093BB139093BC13A0930D
:108CE000BD13B093BE1387E693E10E946F3420E07A
:108CF00030E0A90160917C1270917D1280917E120A
:108D000090917F120F944D2C20E030E048EC52E41B
:108D10000F94E3250F94B92D7093C4136093C3137C
:108D200005E00093B71312E81093BA1386E290E1BE
:108D3000A0E0B0E08093BB139093BC13A093BD134D
:108D4000B093BE1387E693E10E946F348091650271
:108D5000909166029093C4138093C3130093B7134A
:108D60001093BA1380E093E1A0E0B0E08093BB13CE
:108D70009093BC13A093BD13B093BE1387E693E109
:108D80000E946F3420E030E040E251E460914E0CEC
:108D900070914F0C8091500C9091510C0F94E325E1
:108DA0000F94C02D7093C4136093C3130093B71333
:108DB0001093BA1382E492E1A0E0B0E08093BB1379
:108DC0009093BC13A093BD13B093BE1387E693E1B9
:108DD0000E946F3420E030E040E251E46091520C98
:108DE0007091530C8091540C9091550C0F94E32585
:108DF0000F94C02D7093C4136093C3130093B713E3
:108E00001093BA1386E492E1A0E0B0E08093BB1324
:108E10009093BC13A093BD13B093BE1387E693E168
:108E20000E946F3420E030E040E251E46091560C43
:108E30007091570C8091580C9091590C0F94E32528
:108E40000F94C02D7093C4136093C3130093B71392
:108E50001093BA138AE492E1A0E0B0E08093BB13D0
:108E60009093BC13A093BD13B093BE1387E693E118
:108E70000E946F3420E030E040E251E460915A0CEF
:108E800070915B0C80915C0C90915D0C0F94E325CC
:108E90000F94C02D7093C4136093C3130093B71342
:108EA0001093BA138EE492E1A0E0B0E08093BB137C
:108EB0009093BC13A093BD13B093BE1387E693E1C8
:108EC0000E946F3420E030E048EC52E4609174126C
:108ED0007091751280917612909177120F94E3251C
:108EE0000F94B92D7093C4136093C3130093B713F9
:108EF0001093BA1386E392E1A0E0B0E08093BB1335
:108F00009093BC13A093BD13B093BE1387E693E177
:108F10000E946F3420E030E048EC52E46091781217
:108F20007091791280917A1290917B120F94E325BF
:108F30000F94B92D7093C4136093C3130093B713A8
:108F40001093BA138AE392E1A0E0B0E08093BB13E0
:108F50009093BC13A093BD13B093BE1387E693E127
:108F60000E946F3480917502909176029093C413A1
:108F70008093C3130093B7131093BA1382E592E161
:108F8000A0E0B0E08093BB139093BC13A093BD13FB
:108F9000B093BE1387E693E10E946F348091730211
:108FA000909174029093C4138093C3130093B713EA
:108FB0001093BA1384E592E1A0E0B0E08093BB1374
:108FC0009093BC13A093BD13B093BE1387E693E1B7
:108FD0000E946F3420E030E040E251E46091EC11F7
:108FE0007091ED118091EE119091EF110F94E325A6
:108FF0000F94C02D7093C4136093C3130093B713E1
:109000001093BA1386E592E1A0E0B0E08093BB1321
:109010009093BC13A093BD13B093BE1387E693E166
:109020000E946F342CEA35EC47E25EE36091F01168
:109030007091F1118091F2119091F3110F94472DDD
:1090400020E030E040E251E40F94E3250F94C02D7E
:109050007093C4136093C3130093B7131093BA13A0
:109060008AE592E1A0E0B0E08093BB139093BC133B
:10907000A093BD13B093BE1387E693E10E946F34B3
:109080002CEA35EC47E25EE36091F4117091F51142
:109090008091F6119091F7110F94E32520E030E0D4
:1090A00040E251E40F94E3250F94C02D7093C41354
:1090B0006093C3130093B7131093BA138EE592E134
:1090C000A0E0B0E08093BB139093BC13A093BD13BA
:1090D000B093BE1387E693E10E946F3420E030E046
:1090E00040E251E46091811170918211809183116D
:1090F000909184110F94E3250F94C02D7093C413A5
:109100006093C3130093B7131093BA1382E692E1EE
:10911000A0E0B0E08093BB139093BC13A093BD1369
:10912000B093BE1387E693E10E946F342CEA35ECCE
:1091300047E25EE3609185117091861180918711FD
:10914000909188110F94472D20E030E040E251E4E7
:109150000F94E3250F94C02D7093C4136093C31331
:109160000093B7131093BA1386E692E1A0E0B0E043
:109170008093BB139093BC13A093BD13B093BE1305
:1091800087E693E10E946F342CEA35EC47E25EE318
:109190006091891170918A1180918B1190918C113D
:1091A0000F94E32520E030E040E251E40F94E32502
:1091B0000F94C02D7093C4136093C3130093B7131F
:1091C0001093BA138AE692E1A0E0B0E08093BB135B
:1091D0009093BC13A093BD13B093BE1387E693E1A5
:1091E0000E946F348091960C811105C08091980C7B
:1091F000882309F46DC06091E7117091E811072E82
:10920000000C880B990B0F94842520E030E048EC8B
:1092100052E40F94E3256B017C016091E911709198
:10922000EA11072E000C880B990B0F9484259B01E3
:10923000AC01C701B6010F94472D0F94C02D6536C0
:10924000710510F064E670E07093C4136093C3136B
:1092500005E00093B71312E81093BA1384E290E18B
:10926000A0E0B0E08093BB139093BC13A093BD1318
:10927000B093BE1387E693E10E946F346091E711CB
:109280007091E811072E000C880B990B0F94842520
:109290006B017C0120E030E04AE253E40F94AD2EF4
:1092A000181624F48091960C811146C16091E91141
:1092B0007091EA11072E000C880B990B0F948425EE
:1092C0009B01AC01C701B6010F94AD2E87FFAFC162
:1092D00080918C0C882339F180918B0C91E0980F50
:1092E00090938B0C90E09093C4138093C31385E00C
:1092F0008093B71382E88093BA1382E490E1A0E0F0
:10930000B0E08093BB139093BC13A093BD13B093B4
:10931000BE1387E693E10E946F3480918B0C8A30F4
:1093200010F010928B0C0E94FA2B882309F4B5C11F
:109330006091840C7091850CEE24E394F12C6115FE
:109340007105A9F090E080E00F94822520E030E0E4
:1093500040E85EE30F94E3250F942B2D20E030E0EE
:1093600040E85FE30F944D2C0F94C02D7B0101E08A
:1093700010E08091860C811102C010E000E0809125
:10938000AB129091AC128F3F980711F40E948AB3F0
:109390009093AC128093AB12080F191FB80190E0A4
:1093A00080E00F94822520E030E040E85EE30F94F7
:1093B000E3250F942B2D4B015C01F092C413E09236
:1093C000C31305E00093B71312E81093BA1380E1BA
:1093D00093E1A0E0B0E08093BB139093BC13A09303
:1093E000BD13B093BE1387E693E10E946F34C501AD
:1093F000B4010F94C02D7093C4136093C3130093F2
:10940000B7131093BA1382E193E1A0E0B0E0809328
:10941000BB139093BC13A093BD13B093BE1387E608
:1094200093E10E946F3407E014E1AAE1FA2E8091E3
:10943000390590913A0520917B0530917C05891B77
:109440008F7309F449C12A3131050CF0DBC19091C9
:10945000390580913A054FEF5FEF981749F0E82FF3
:10946000F0E0E75CFA4F42818F5F8F7380933A059B
:10947000F901E95FFB4E4083809107148A3509F0BA
:10948000B3C162E070E080E090E00E94782C8091AF
:109490007B0590917C05019690937C0580937B05DC
:1094A000C6CF1092C4131092C313ACCB6091E911D4
:1094B0007091EA11072E000C880B990B0F948425EC
:1094C00020E030E0A9010F947D25811134C98CE0A2
:1094D00090E09093C4138093C31385E08093B713F7
:1094E00082E88093BA1384E190E1A0E0B0E0F3CB8E
:1094F0008DE090E09093C4138093C31385E0809334
:10950000B71382E88093BA1384E190E1A0E0B0E061
:109510008093BB139093BC13A093BD13B093BE1361
:1095200087E693E10E946F3480919D0C811101C008
:1095300081E080939D0CDBCB1092960C20E030E014
:1095400040E251E460918E0C70918F0C8091900CF0
:109550009091910C0F94E3250F94B92D7093C4133F
:109560006093C3130093B7131093BA1384E590E18B
:10957000A0E0B0E08093BB139093BC13A093BD1305
:10958000B093BE1387E693E10E946F3420E030E091
:1095900040E251E46091920C7091930C8091940C94
:1095A0009091950C0F94E3250F94B92D7093C413EB
:1095B0006093C3130093B7131093BA1388E590E137
:1095C000A0E0B0E08093BB139093BC13A093BD13B5
:1095D000B093BE1387E693E10E946F3480EA97E16F
:1095E0000E942C388AE00E94F33781E09AE590933C
:1095F000C4138093C31381E490E09093C6138093C7
:10960000C51387E08093B7131093BA1384E890E0F2
:10961000A0E0B0E08093BB139093BC13A093BD1364
:10962000B093BE1387E693E10E946F3451CE6091F0
:10963000980C662309F44CCE062E000C770B87E8B5
:1096400097E10E942A418AE00E94F3371092980C19
:1096500084E090E09093C4138093C31385E08093DB
:10966000B71312E81093BA138EE890E1A0E0B0E0CF
:109670008093BB139093BC13A093BD13B093BE1300
:1096800087E693E10E946F3481E09AE59093C413DA
:109690008093C31383E590E0B0CF1092C41310926F
:1096A000C31305E00093B71312E81093BA1380E1D7
:1096B00093E1A0E0B0E08093BB139093BC13A09320
:1096C000BD13B093BE1387E693E10E946F341092EE
:1096D000C4131092C31393CE121613060CF492C047
:1096E00080916B1390916C13A0916D13B0916E13D8
:1096F0008C34E0E19E07A105B10509F4D7C98A348D
:109700009041A105B10509F4D1C920E030E040E263
:1097100051E46091240C7091250C8091260C90915D
:10972000270C0F94E3250F94B92D7093C413609305
:10973000C31305E00093B71312E81093BA1388E43B
:1097400090E1A0E0B0E08093BB139093BC13A09392
:10975000BD13B093BE1387E693E10E946F3420E0FF
:1097600030E040E251E46091280C7091290C809126
:109770002A0C90912B0C0F94E3250F94B92D709324
:10978000C4136093C3130093B7131093BA138AE4FE
:1097900090E1A0E0B0E08093BB139093BC13A09342
:1097A000BD13B093BE1387E693E10E946F3420E0AF
:1097B00030E040E251E460912C0C70912D0C8091CE
:1097C0002E0C90912F0C0F94E3250F94B92D7093CC
:1097D000C4136093C3130093B7131093BA138CE4AC
:1097E00090E1A0E0B0E056C9121613060CF01FCEAF
:1097F000F8012F2D11922A95E9F710927C0510920D
:109800007B0515CE9091681380910714981321C0A1
:10981000909169138091081498131BC0233031056F
:10982000C4F0909109149093671380910A14809367
:109830006A139330D1F4982F9D7F9038B1F49091B2
:109840000B149F3409F059C090910C149B3409F00B
:1098500054C0E7E0F4E18AE1DF011D928A95E9F75F
:1098600010927C0510927B053BCF833809F045C0F0
:1098700080910B1490910C14982789279827B0E0B9
:10988000A0E080936B1390936C13A0936D13B0932F
:109890006E13C0900D14D12CF12CE12CC0926F13DB
:1098A000D0927013E0927113F09272132EE034E1B3
:1098B00040E050E0BA014C155D056E057F0508F0EB
:1098C0004AC0DB01CA01B695A7959795879506967C
:1098D000880F991FFC01E959FC4ED9018C91119612
:1098E0009C91892798278927918380834E5F5F4FBA
:1098F0006F4F7F4F2E5F3F4FDECF813861F58091F4
:109900000B1490E0B0E0A0E080936B1390936C1385
:10991000A0936D13B0936E1380910C14482F50E0F8
:1099200070E060E040936F13509370136093711375
:1099300070937213ADE0B4E1E3E7F3E190E030E05F
:1099400020E08217930739F04D9150E041935193F5
:109950002F5F3F4FF6CFE7E0F4E18AE1DF011D9290
:109960008A95E9F710927C0510927B050E9407FE0C
:10997000B7CE3F924F925F926F927F928F929F925B
:10998000AF92BF92CF92DF92EF92FF920F931F930D
:10999000CF93DF938091350587FD38C080913605E0
:1099A0008370A1F5C0918012D091811248815981B4
:1099B0006A817B8181E197E10E9408414C815D8150
:1099C0006E817F8184E39FE20E94084140917C1276
:1099D00050917D1260917E1270917F1281E39FE21F
:1099E0000E9408418AE0DF91CF911F910F91FF9073
:1099F000EF90DF90CF90BF90AF909F908F907F902F
:109A00006F905F904F903F900C94F337609074127A
:109A1000709075128090761290907712A0907812C4
:109A2000B090791200917A1210917B12C0907C1242
:109A3000D0907D12E0907E12F0907F1288E50E9417
:109A40007C1EC82F882309F49AC00E948224362ED7
:109A5000472E582ED92F20E030E041EE53EC0F94E2
:109A6000AD2E87FD0DC020E030E041EE53E4632DC4
:109A7000742D852D9D2F0F947D2518160CF081C017
:109A800062EC71E08EEF96E10E942A4162EC71E097
:109A900089EF96E10E942A4186EF96E10E942C38D8
:109AA000C0E089E50E947C1E882361F10E94822427
:109AB000362E472E582ED92F20E030E041EE53ECC1
:109AC0000F94AD2E87FD0DC020E030E041EE53E451
:109AD000632D742D852D9D2F0F947D2518160CF068
:109AE00055C062EC71E083EE96E10E942A4162EC7F
:109AF00071E08EED96E10E942A418BED96E10E9485
:109B00002C38C0E08AE50E947C1E882309F443C0FB
:109B10000E9482246B017C0120E030E040E151ECA6
:109B20000F94AD2E87FD0AC020E030E040E151E403
:109B3000C701B6010F947D2518166CF567EF7FEF0E
:109B400089EC96E10E942A4169E070E084EC96E19C
:109B50000E942A4181EC96E1DF91CF911F910F91F4
:109B6000FF90EF90DF90CF90BF90AF909F908F903D
:109B70007F906F905F904F903F900C942C38C1E095
:109B800090CF632C742C852C9D2E8BCFA32CB42CC2
:109B9000052D1D2FB7CFCC23E1F0C301D401809355
:109BA000741290937512A0937612B0937712C50138
:109BB000D8018093781290937912A0937A12B0937F
:109BC0007B12C0927C12D0927D12E0927E12F092B3
:109BD0007F12DF91CF911F910F91FF90EF90DF9057
:109BE000CF90BF90AF909F908F907F906F905F903D
:109BF0004F903F9008958FED97E00C942C3889EDAD
:109C000097E00C942C3884E690E09093C005809304
:109C1000BF051092E0051092DF050C94DEDBEF9299
:109C2000FF920F931F93CF93DF93CDB7DEB7629769
:109C30000FB6F894DEBF0FBECDBF0E94FD2988236A
:109C400009F43FC046EE53E082FF02C04AEC53E005
:109C500026EE33E081FF02C02CEC33E080FD2EC005
:109C600086EE93E05F934F933F932F939F938F9351
:109C70008BE399E19F938F938E010F5F1F4F1F938B
:109C80000F930F9414250E94FF4DC8010E94FA37CC
:109C9000C8010E9477E40FB6F894DEBF0FBECDBFB7
:109CA00081E062960FB6F894DEBF0FBECDBFDF91A4
:109CB000CF911F910F91FF90EF9008958EEC93E05C
:109CC000D1CF80E0EECFCF92DF92EF92FF928AE584
:109CD0000E947C1E882309F45AC00E94822420E03E
:109CE00030E040E050EC0F947D25C12CD12CE12CCC
:109CF00090ECF92E87FD0FC00E94822420E030E016
:109D000040E050E40F94AD2E18160CF462C00E948F
:109D100082246B017C012091560C3091570C4091AC
:109D2000580C5091590CC701B6010F94E3250F94BC
:109D3000B92DCB010E9490FD80E50E942E1E81115D
:109D40004EC0A701960160917C1270917D128091A6
:109D50007E1290917F120F944D2C60937C12709321
:109D60007D1280937E1290937F120E94FF4D40914E
:109D70007C1250917D1260917E1270917F1282EB65
:109D800096E10E9408418AE00E94F33705C083E50E
:109D90000E947C1E8111A1CF8091350587FD24C0D2
:109DA00080913605837001F50E94FF4D40917C1231
:109DB00050917D1260917E1270917F1283EA96E13C
:109DC0000E9408418AE0FF90EF90DF90CF900C94C2
:109DD000F337C12CD12CE12C80E4F82E9CCF0E94CB
:109DE0004A248111AECFD8CF82E50E942E1E811168
:109DF000DBCFFF90EF90DF90CF900895CF9384E575
:109E00000E947C1EC0E08823D9F00E942A24C82F1B
:109E10001816B4F40E94FF4D8DE40E94F337809130
:109E20003005909131050E942BE26C2FCC0F770BFF
:109E300088EA9FE00E942A418AE00E94F337CFEF30
:109E40008C2FCF9108954F925F926F927F928F9255
:109E50009F92AF92BF92CF92DF92EF92FF92CF93F9
:109E6000DF93CDB7DEB72C970FB6F894DEBF0FBEE9
:109E7000CDBF4090CC085090CD086090CE08709037
:109E8000CF082091470230914802409149025091F9
:109E90004A02C301B2010F944D2C69837A838B83EC
:109EA0009C838090D0089090D108A090D208B09068
:109EB000D30820914B0230914C0240914D025091B9
:109EC0004E02C501B4010F944D2C6D837E838F83A8
:109ED0009887C090D408D090D508E090D608F0902C
:109EE000D70820914F023091500240915102509179
:109EF0005202C701B6010F944D2C69877A878B8770
:109F00009C87209153023091540240915502509108
:109F10005602C301B2010F944D2C2B013C0120913C
:109F20005702309158024091590250915A02C5018E
:109F3000B4010F944D2C4B015C0120915B023091D8
:109F40005C0240915D0250915E02C701B6010F9420
:109F50004D2C6B017C010E94FF4D83EE9EE00E9420
:109F60002C3883E50E942E1E882321F00E944A246B
:109F70008093450280914502811151C08AEC9EE098
:109F80000E942C388BED9EE00E942C3849815A812A
:109F90006B817C8189E09EE10E9408414D815E8158
:109FA0006F81788584E39FE20E94084149855A8544
:109FB0006B857C8581E39FE20E94084189ED9EE0EC
:109FC0000E942C3881ED9EE00E942C38B301A20142
:109FD00089E09EE10E940841B501A40184E39FE26B
:109FE0000E940841B701A60181E39FE20E94084157
:109FF0008AE02C960FB6F894DEBF0FBECDBFDF917E
:10A00000CF91FF90EF90DF90CF90BF90AF909F9057
:10A010008F907F906F905F904F900C94F3378EEC01
:10A020009EE0AECF5F926F927F928F929F92AF929F
:10A03000BF92CF92DF92EF92FF920F931F93CF9335
:10A04000DF931F92CDB7DEB77C0139018B015B0135
:10A05000A40EB51ED12CC12CA016B10609F450C017
:10A06000F70180809180F80151908F015982C401DD
:10A070000F949B2B5816B9F1652DC4010F94A32B97
:10A08000FFEFCF1ADF0AC6018F779927892B21F1BD
:10A0900062E070E080E090E00E9424FDC4010F9433
:10A0A0009B2B99818917F9F00E94FF4D8FE694E070
:10A0B0000E942C3881E00F90DF91CF911F910F917A
:10A0C000FF90EF90DF90CF90BF90AF909F908F90D8
:10A0D0007F906F905F90089562E070E080E090E084
:10A0E0000E94F025DBCFBE016F5F7F4FC3010E944E
:10A0F000FFE0F70180819181019691838083ACCF4D
:10A1000080E0D9CFDF92EF92FF920F931F93CF930E
:10A11000DF93CDB7DEB7CA5AD1090FB6F894DEBFC8
:10A120000FBECDBFCF55DF4F188219821A821B8216
:10A13000C15AD0408091D0039091D103A091D20315
:10A14000B091D303CB55DF4F88839983AA83BB8318
:10A15000C55AD04084E690E09093C0058093BF0537
:10A160001092E0051092DF051092E1052FED35E029
:10A1700044E050E0BE016B557F4F8FEB95E00E94AD
:10A1800012508091BF059091C00502969093C00532
:10A190008093BF051092E0051092DF0581E0C6555F
:10A1A000DF4F8883CA5AD040CE0186559F4F0E9408
:10A1B000A1D12FED35E048E450E06AE37CE08FEB7D
:10A1C00095E00E9412502FED35E040E150E069ED3E
:10A1D00078E08FEB95E00E9412508AE097EDA3EAB9
:10A1E000BCE3CF55DF4F88839983AA83BB83C15AD1
:10A1F000D040CE018F559F4F0E9498D182E098E0C9
:10A200000E94B3D186E292E00E94AAD182E292E05B
:10A210000E9498D18091C8089091C908A091CA085D
:10A22000B091CB0889839A83AB83BC838E010F5F87
:10A230001F4FC8010E9498D1CF55DF4F1882198255
:10A240001A821B82C15AD0407E018DE6E80EF11CB5
:10A2500083E0D7018C938983CE018F559F4F0E9455
:10A2600098D1C7010E94A1D1C8010E94A1D14AE0A2
:10A27000D42EDA94DD2031F0CE018F559F4F0E940D
:10A2800098D1F7CF84E792E10E94B3D1CF55DF4F49
:10A29000188219821A821B82C15AD0403AE0D32E0A
:10A2A000DA94DD2031F0CE018F559F4F0E9498D176
:10A2B000F7CF85E0D82ED982F701D082C8010E945D
:10A2C000A1D1C7010E94A1D12FED35E048E050E0B7
:10A2D00062ED75E08FEB95E00E9412502FED35E0B6
:10A2E00048E050E06AEC75E08FEB95E00E94125078
:10A2F0002FED35E044E650E06CE877E08FEB95E039
:10A300000E94125019828FEFD7018C93C8010E94CE
:10A31000AAD1C7010E94A1D12FED35E044E050E061
:10A3200066EE72E08FEB95E00E9412508091A306DA
:10A330008983C8010E94AAD1198A1A8A1B8A1C8A99
:10A3400080E090E0A0E8BFE38D879E87AF87B88B61
:10A350008091EC119091ED11A091EE11B091EF115F
:10A3600089839A83AB83BC832CEA35EC47E25EE3B6
:10A370006091F0117091F1118091F2119091F311AF
:10A380000F94472D6D837E838F8398872CEA35EC5D
:10A3900047E25EE36091F4117091F5118091F6113E
:10A3A0009091F7110F94E32569877A878B879C87B3
:10A3B0002FED35E044E150E0B8018FEB95E00E94CD
:10A3C000125084E190E09A838983C8010E9486D16B
:10A3D0008091811190918211A0918311B09184118B
:10A3E00089839A83AB83BC832CEA35EC47E25EE336
:10A3F00060918511709186118091871190918811DB
:10A400000F94472D6D837E838F8398872CEA35ECDC
:10A4100047E25EE36091891170918A1180918B11FE
:10A4200090918C110F94E32569877A878B879C879D
:10A43000C8010E948FD18CE0EDE7F2E0D8010190D5
:10A440000D928A95E1F7C8010E948FD11982C80147
:10A450000E94A1D18FE790E09A838983C8010E946E
:10A4600086D1E9E8F2E0D80101900D92DA94E1F7A3
:10A470002FED35E045E050E0B8018FEB95E00E940C
:10A4800012508091C9058983C8010E94AAD180E237
:10A49000EEE8F2E0D80101900D928A95E1F72FEDF8
:10A4A00035E040E250E0B8018FEB95E00E94125099
:10A4B000F7011082C7010E94AAD185EF97E00E94A0
:10A4C000AAD181EF97E00E9498D1CF55DF4F188233
:10A4D00019821A821B82C15AD040CE018F559F4FDC
:10A4E0000E9498D180E2D8011D928A95E9F72FED5C
:10A4F00035E040E250E0B8018FEB95E00E94125049
:10A50000FE01F99688E0DF011D928A95E9F744E69D
:10A5100050E060E070E049835A836B837C834D8315
:10A520005E836F83788783E090E0A0E0B0E0898766
:10A530009A87AB87BC874D875E876F87788B498BFF
:10A540005A8B6B8B7C8B8D8B9E8BAF8BB88F898F4F
:10A550009A8FAB8FBC8F8D8F9E8FAF8FB8A38EE1FC
:10A5600090E0A0E0B0E089A39AA3ABA3BCA38DA325
:10A570009EA3AFA3B8A789A79AA7ABA7BCA78DA78F
:10A580009EA7AFA7B8AB89AB9AABABABBCAB8DAB5F
:10A590009EABAFABB8AF2FED35E040E450E0B80173
:10A5A0008FEB95E00E94125090E1D92EF8018D2D8D
:10A5B00011928A95E9F72FED35E040E150E0B801BE
:10A5C0008FEB95E00E941250D8011D92DA94E9F7C2
:10A5D0002FED35E040E150E0B8018FEB95E00E94AF
:10A5E0001250CF55DF4F188219821A821B82C15A2E
:10A5F000D040CE018F559F4F0E9498D12CE0D22E93
:10A60000F8018D2D11928A95E9F72FED35E04CE098
:10A6100050E0B8018FEB95E00E9412508CE6D80113
:10A620001D928A95E9F72FED35E04CE650E0B80130
:10A630008FEB95E00E94125083EB95E00E948FD142
:10A640002FED35E048E050E061EC75E08FEB95E0F0
:10A650000E941250F7011192DA94E9F7C755DF4FC3
:10A660001882C95AD04080E090E0A0E4B0E4C3561C
:10A67000DF4F88839983AA83BB83CD59D040C7011C
:10A680000E94B3D1CE0187559F4F0E94A1D1CE0128
:10A6900083569F4F0E9498D180E3D7011D928A95DF
:10A6A000E9F785E89CE10E942C388AE00E94F337A4
:10A6B0002FED35E040E350E0B7018FEB95E00E94CD
:10A6C00012508091E105811128C00091BF051091C1
:10A6D000C0058091DF059091E005F70191838083AB
:10A6E00084E690E09093C0058093BF052FED35E0A0
:10A6F00044E050E066EF72E08FEB95E00E9412506C
:10A70000C7010E9486D191E00536134009F490E01C
:10A710008091E105892B8093E1058091E10581110C
:10A7200005C060E089EB9CE10E949A3F89E99CE1C9
:10A730000E942C388AE00E94F3379091E10581E075
:10A740008927C655DF4F0FB6F894DEBF0FBECDBFC9
:10A75000DF91CF911F910F91FF90EF90DF900895BF
:10A76000CF93DF9300D01F92CDB7DEB780918F06D5
:10A770008823C1F083E390E09C838B831A82198243
:10A780009E012F5F3F4F40E150E060E976E0CE014F
:10A7900003960E94125089E99CE10E942C388AE0BD
:10A7A0000E94F3370F900F900F900F90DF91CF9191
:10A7B0000895CF92DF92EF92FF92CF93C82F8091AE
:10A7C00020118150823008F069C00E948F3A1092A7
:10A7D00020110E9457FD6093AB057093AC058093E8
:10A7E000AD059093AE05C090AF05D090B005E09058
:10A7F000B105F090B2050E94642BAB01BC014093FF
:10A80000AF055093B0056093B1057093B205809188
:10A81000940690919506A0919606B09197068C1992
:10A820009D09AE09BF09840F951FA61FB71F80930E
:10A83000940690939506A0939606B0939706C1113F
:10A840000AC0C1E00E94B0538C2FCF91FF90EF90CF
:10A85000DF90CF9008958091920690919306019693
:10A8600090939306809392060E94642BC090980662
:10A87000D0909906E0909A06F0909B06C616D706EF
:10A88000E806F906F0F60E94642B60939806709330
:10A89000990680939A0690939B06D3CFC0E0D2CFBF
:10A8A00081E00C94D9530E94A8BE0E94505480E0CD
:10A8B0000E9426F98091E5068130A1F40E94FB4DAB
:10A8C00082E697E00E942C3860E088E597E00E94DD
:10A8D0009A3F6EE571E080E090E00E94F02588E00C
:10A8E0008093E5060895CF92DF92EF92FF921F9337
:10A8F000CF93DF9300D01F92CDB7DEB78EEEC82E78
:10A9000082E0D82EE12CF12CC982DA82EB82FC8223
:10A91000BE016F5F7F4F8AE50E94513381110EC0E7
:10A9200010E0812F0F900F900F900F90DF91CF913B
:10A930001F91FF90EF90DF90CF9008950E94A73372
:10A94000C982DA82EB82FC82BE016F5F7F4F8AE5AB
:10A950000E945133182F882319F30E94FB4D8CE37A
:10A9600098E00E942C380E945354DBCFCF92DF92A4
:10A97000EF92FF921F93CF93DF9300D01F92CDB73A
:10A98000DEB78EEEC82E82E0D82EE12CF12CC982E3
:10A99000DA82EB82FC82BE016F5F7F4F8AE00E9409
:10A9A000513381110EC010E0812F0F900F900F9046
:10A9B0000F90DF91CF911F91FF90EF90DF90CF909C
:10A9C00008950E94A7330E9471330E948C330E9425
:10A9D0007133C982DA82EB82FC82BE016F5F7F4FE6
:10A9E0008AE00E945133182F8823E9F20E94FB4D20
:10A9F0008FEF97E00E942C380E945354D5CFCF930D
:10AA0000DF9300D01F921F92CDB7DEB781E0809315
:10AA10008F0680E1E0E9F6E0DF011D928A95E9F713
:10AA20000E94B05386E18D8382E390E09C838B8308
:10AA30001A8219829E012F5F3F4F41E050E0BE0114
:10AA40006B5F7F4FCE0103960E9412500F900F90C4
:10AA50000F900F900F90DF91CF910895CF93DF93D8
:10AA6000CDB7DEB7A8970FB6F894DEBF0FBECDBF47
:10AA70008C01F42E0E94A8BE0E94FB4D88E397E053
:10AA80000E942C380115110511F40FE217E0809196
:10AA9000850580FD79C08160809385058BE197E015
:10AAA0000E942C388AE00E94F337CC24C3948AE5B4
:10AAB000D82ED092C413C092C3138FE090E090932D
:10AAC000C6138093C51397E0792E7092B71322E8CE
:10AAD000E22EE092BA1334E8832E912CA12CB12CF3
:10AAE0008092BB139092BC13A092BD13B092BE1380
:10AAF00087E693E10E946F34D092C413C092C313CF
:10AB000088E590E09093C6138093C5137092B713B5
:10AB1000E092BA138092BB139092BC13A092BD1323
:10AB2000B092BE1387E693E10E946F348AE2898374
:10AB30008A838B838C83F801DE011596BE016F5FDB
:10AB40007F4FCD01861B970B2491319621110CC0AC
:10AB5000FB01E80FF91F8AE29F01261B370B283201
:10AB6000310524F48193F8CF2D93EBCF20E630E12B
:10AB700040E050E087E693E10E941AE16AE070E06D
:10AB800080E090E00E94782C61E086E297E00E94ED
:10AB9000673F89EE93E030E6019729F0232F2A954D
:10ABA0000000E9F7F9CFF89489EE93E038EE0197C9
:10ABB00029F0232F2A950000E9F7F9CF0E94A8BEBB
:10ABC000FF2031F00E94E81E0E94011FA895FECFD1
:10ABD0000E94E61EF9CF8091E406882319F01092B6
:10ABE000E406089540E070E060E08CEA98E10E949D
:10ABF0002E558091A00C9091A10C2FEF3FEF98174C
:10AC000051F0E92FF0E0E056F34F228130E09F5FF2
:10AC10009F779093A10CC90108951F920F920FB6D0
:10AC20000F9211240F900FBE0F901F9018951F9236
:10AC30000F920FB60F9211240BB60F920F931F9322
:10AC40002F933F934F935F936F937F938F939F9334
:10AC5000AF93BF93CF93DF93EF93FF93C091C60061
:10AC60000091A10CD091A00C11E01D0F1F779091C5
:10AC70001304913108F09FC0E92FF0E08827EC5BC6
:10AC8000F94A8F4F0D94442C555684569356A2562C
:10AC9000A956DB56AD56DB56B156B556DB56B956FE
:10ACA000BD56C156C856DB56D356C03229F028F5DA
:10ACB000CA3011F0CD3031F5011731F0ED2FF0E051
:10ACC000E056F34FC283D12FD093A00CFF91EF91A8
:10ACD000DF91CF91BF91AF919F918F917F916F91B4
:10ACE0005F914F913F912F911F910F910F900BBE4C
:10ACF0000F900FBE0F901F901895CD3481F081E01A
:10AD0000CE3471F080E10CC0CA3338F4C033A0F601
:10AD1000C03291F2CD32B1F7CFCFCD3499F782E086
:10AD200080931304C9CFC13359F018F4C03221F213
:10AD3000E9CF88E0C433A1F38BE0C83389F3E2CFD5
:10AD400083E0EECF84E0C03359F386E0C13341F3B2
:10AD5000D9CF85E0C833B1F6E3CF87E0C23391F6AF
:10AD6000DFCF89E0C13371F6DBCF8AE0C03351F623
:10AD7000D7CF8CE0C73331F6D3CF8DE0C63311F691
:10AD8000CFCFC03209F498CF8EE0C33549F2BACFA5
:10AD900080ED8C0F8A3008F08FCF9FE090931304E2
:10ADA0008093140489CFCA3019F0CD3009F084CFD4
:10ADB0001092130481CFCA3019F0CD3009F07CCF46
:10ADC000809121148823A1F3973089F038F49530CD
:10ADD00079F710923C021092230CEACF9A3059F086
:10ADE0009F3031F7809114040E948E31E1CF81E0D1
:10ADF00080930D06DDCF81E080930C06D9CF8EBD08
:10AE00000DB407FEFDCF08958FEF8EBD0DB407FE84
:10AE1000FDCF8EB50895909164009B7F9093640060
:10AE2000982F906A96959CBD80FD03C091E0863076
:10AE300009F490E09DBD0895CF93DF93EB010E944C
:10AE40002C38CE01DF91CF910C94F2AE2F923F922D
:10AE50004F925F926F927F928F929F92AF92BF922A
:10AE6000CF92DF92EF92FF920F931F93CF93DF93D6
:10AE7000009709F0AAC11092880C1092870C909349
:10AE8000840580938305BAE0CB2EB0E2DB2EE12C63
:10AE9000F12C15E002E846015701C4E1D0E0109220
:10AEA0000A13109209131093FD120093001380925D
:10AEB000011390920213A0920313B09204138DEA2F
:10AEC00092E10E946F3421972FEF821A920AA20A10
:10AED000B20A209721F744E1C40ED11CE11CF11CF9
:10AEE0008AE5C81680E2D806E104F104A1F6C12C77
:10AEF000A0E2DA2EE12CF12CD5E0C2E810920A1380
:10AF000010920913D093FD12C0930013C092011345
:10AF1000D0920213E0920313F09204138DEA92E1AF
:10AF20000E946F3410920A1310920913D093FD12ED
:10AF3000C0930013D701C6018C529F4FAF4FBF4F34
:10AF40008093011390930213A0930313B0930413FF
:10AF50008DEA92E10E946F34EFEFCE1ADE0AEE0A1C
:10AF6000FE0AFAE0CF16F0E2DF06E104F10431F662
:10AF7000FEEDCF2EF0E2DF2EE12CF12CD5E0C2E881
:10AF800010920A1310920913D093FD12C09300136C
:10AF9000C0920113D0920213E0920313F0920413B3
:10AFA0008DEA92E10E946F342FEFC21AD20AE20AB0
:10AFB000F20A46EEC41640E2D406E104F10401F7B9
:10AFC000CC24C394E2E1DE2EE12CF12C0AE010E067
:10AFD000D5E0C2E810930A1300930913D093FD1231
:10AFE000C0930013C0920113D0920213E092031396
:10AFF000F09204138DEA92E10E946F3410930A13C9
:10B0000000930913D093FD12C0930013D701C6011A
:10B010008096A11DB11D8093011390930213A093FC
:10B020000313B09304138DEA92E10E946F348FEF03
:10B03000C81AD80AE80AF80AE5E0CE16E2E1DE0608
:10B04000E104F10439F60091870C1091880C011588
:10B05000110509F0D6C08091860C882309F4E1C05F
:10B060002AE030E240E050E064ED73E08DEA92E1E6
:10B070000E941AE1C1E0D0E003E010E0E090870C0C
:10B08000F090880C35E0332E42E8242E44244A9474
:10B09000542C64E0662E712C7FE1C72E74E0D72E0D
:10B0A0008091870C9091880C800F911FE816F9060B
:10B0B00008F0D5C0C7010E9431E2882309F481C09D
:10B0C00080919B116EE871E1882311F06BE971E1C9
:10B0D000FB0101900020E9F7CF010197861B970B38
:10B0E000F4E1FC9F9001FD9F300D1124265F3F4D40
:10B0F00050E040E0459710F0FB01128A8DEA92E1A2
:10B100000E941AE1CE018F5F9D4EB0E0A0E0219633
:10B110004E0124E0880C991C2A95E1F7FDEF8F1A67
:10B12000FFE99F0AB12CA12C20912D1424FF7EC091
:10B1300070920A13609209133092FD12209200134C
:10B140008093011390930213A0930313B0930413FD
:10B150008DEA92E10E946F34D0920A13C0920913D3
:10B160003092FD12209200138092011390920213EC
:10B17000A0920313B09204138DEA92E10E946F34FF
:10B18000B70181E498E10E94F64080919B116BE940
:10B1900071E1811102C06EE871E18EE398E10E94D5
:10B1A0001C5763EE7BE08AE398E10E941C576EE82F
:10B1B00071E189E398E10E941C5785E398E10E94C0
:10B1C0002C382FEFE21AF20A6BCF2091870C3091C6
:10B1D000880CA90141505109609183057091840543
:10B1E0006817790738F42C5F3F4F3093880C209311
:10B1F000870C45CE4430510508F43DCE245031092A
:10B20000F4CF0430110569F48091860C882331F065
:10B2100083E090E09093880C8093870CD0E0C0E0AE
:10B220002DCFD0E0C0E004E010E028CF10920A1348
:10B23000109209133092FD12209200138093011393
:10B2400090930213A0930313B09304138DEA92E139
:10B250000E946F3450920A134092091381CFDF91FC
:10B26000CF911F910F91FF90EF90DF90CF90BF9003
:10B27000AF909F908F907F906F905F904F903F9096
:10B280002F900895AF92BF92CF92DF92EF92FF92EC
:10B290000F931F93CF93DF93CDB7DEB7E6970FB62B
:10B2A000F894DEBF0FBECDBF009137051091380571
:10B2B000F80101900020E9F731976F01C01AD10A17
:10B2C000F801CF01801B910B8C159D053CF48191F9
:10B2D0008F32B9F7DF0111971C92F3CF8BE1EDE4C8
:10B2E000F4E1DE015C9601900D928A95E1F7F12C74
:10B2F000E12CEC14FD040CF05DC0F801EE0DFF1D17
:10B300008081811103C08FEFE81AF80A5801AE0C52
:10B31000BF1CF5018081882309F44CC0FFEFEF1AB0
:10B32000FF0AF801EE0DFF1D7F01E01AF10A81917D
:10B330008111FACFCE014C960E9485B38BE1FE01BC
:10B340007C96DE01119601900D928A95E1F7B50188
:10B35000CE0101960E9493ABCE0101960E947B2FF5
:10B360008FE20E94F33780919B1181113BC081EEE7
:10B3700093E00E94F2AE80912D1484FF1BC01982CD
:10B380001C8221E0A501BE01645E7F4FCE010196C3
:10B390000E94C7B5811129C08AE00E94F3370E943C
:10B3A000FF4DB50180E297E10E941C57CE01019646
:10B3B0000E947B2F8AE00E94F337CE014C960E94B8
:10B3C0007B2FE6960FB6F894DEBF0FBECDBFDF91A0
:10B3D000CF911F910F91FF90EF90DF90CF90BF9092
:10B3E000AF9008958BE991E1C4CFCE014C960E94B5
:10B3F000F4B28BE1FE013196DE015C9601900D9274
:10B400008A95E1F7CE0101960E947B2F72CF2F9291
:10B410003F924F925F926F927F928F929F92AF92E4
:10B42000BF92CF92DF92EF92FF920F931F93CF9331
:10B43000DF9300D000D000D01F921F92CDB7DEB7AF
:10B44000B82E80918D0D843008F0D1C10E9457FD37
:10B450006B017C0180918D0D811108C08091A00C41
:10B460009091A10C891B8F7709F4A4C681E6A82EC0
:10B4700013C08A3019F08D3009F0F6C01092880D93
:10B480008091260D9091270DFC01EE5DF24F168202
:10B49000892BF1F40E94F5C180918D0D843008F064
:10B4A000ECC08091A00C9091A10C891B8F7709F4BE
:10B4B000E4C00E94F95597FFDCCF0E94FB4D85EB5D
:10B4C00095E00E942C388091A00C8093A10CE4CFD1
:10B4D0001092270D1092260D08E21DE0F8018191CF
:10B4E000803209F446C08E3409F0A9C060EB75E0E3
:10B4F000C8010F94FA244C01892B41F06EE470E0EE
:10B50000C80104960F949B2F009709F4C8014AE0E4
:10B5100050E070E060E001960F946A222B013C013C
:10B520008091220D9091230DA091240DB091250DB5
:10B530000196A11DB11D481659066A067B0629F021
:10B5400060E08DE795E0892851F16AE270E0C8017A
:10B550000F94CA2F9C01009729F1982F901B912CD2
:10B56000992349F09150F801E90FF11D8081982647
:10B57000F7CF8F01B3CF4AE050E070E060E0C9013F
:10B5800001960F946A22292D30E050E040E06217C6
:10B5900073078407950751F060E08EE595E00E94FF
:10B5A000ACE77ACF60E084E395E0F9CF4092220DDA
:10B5B0005092230D6092240D7092250D8091E50626
:10B5C0008130E1F067E470E0C8010F949B2F009791
:10B5D000A9F04AE050E070E060E001960F946A2222
:10B5E000643071058105910548F483E994E00E9477
:10B5F0002C3860E089E894E00E949A3FC09284076A
:10B60000D0928507E0928607F09287078091280DF7
:10B610008B3309F441CF80918D0D843008F03CCFFD
:10B6200080918F0D8A9DC001112468E27DE08057D2
:10B63000924F0F94A62F80E00E9466E72DCF809155
:10B640002D1480FFBBCF6BE77DE2C8010F94FA2475
:10B65000009731F0FC01838180538A3008F0AECF2F
:10B6600060E08AE095E09BCF26E23DE048E25DE0C5
:10B6700068E87DE00E94FC1C0FCF80912D1482FFB2
:10B68000B6C01A82198271E6F72EE0E1EE2EF9E6D5
:10B69000DF2E80918D0D843008F0A9C00E94341DEA
:10B6A0008111A5C041E050E0BE016B5F7F4F81E991
:10B6B00095E10E9447B10D8110E0019711F00FEF65
:10B6C0001FEF8091991590919A15A0919B15B091BB
:10B6D0009C158093291490932A14A0932B14B09353
:10B6E0002C140E94341D0F3F100749F4811107C02C
:10B6F0000E94FB4D83ED95E00E942C38CACF40910B
:10B700008F0D242F30E00A3061F00D3051F0882386
:10B7100009F45FC089819A81009719F001969A8394
:10B72000898310929A0489819A81F29EF001F39E96
:10B73000F00D1124E357F24FE80FF91F1382892B04
:10B7400069F50E94F5C10E94341D882309F4A1CF38
:10B750000E946B6181E995E10E94F4B2809124140A
:10B76000882391F18150809324148D9DC001112470
:10B7700062E0835E994F0E9449B8E091241424E06E
:10B78000E29FF0011124E75EF94F608171818281AF
:10B7900093810E944D220E94FCAA7BCF1A821982BB
:10B7A00081E00E9466E78091291490912A14A0916B
:10B7B0002B14B0912C148093890D90938A0DA09333
:10B7C0008B0DB0938C0DBFCF0E94FDB2E092E506C9
:10B7D00060CF4F9DA00111244057524F9E012F5F13
:10B7E0003F4F6AE974E0802F0E94FC1C52CF0E94F8
:10B7F00057FD6B017C01B11004C080911F1188239B
:10B8000051F0C0927211D0927311E0927411F092C3
:10B810007511BB24B39480910F0590911005A091F0
:10B820001105B09112050097A105B105B1F0409145
:10B830007211509173116091741170917511840F90
:10B84000951FA61FB71FA7019601281B390B4A0B8E
:10B850005B0BDA01C901B7FF92C18091130290918D
:10B860001402A0911502B0911602892B8A2B8B2B02
:10B8700009F099C10E9457FD4B015C018091230C96
:10B88000811108C0209185129091861281E02913C0
:10B8900001C080E02091E7113091E81191E0892703
:10B8A0002A3A31050CF480E091E040919F045091D8
:10B8B000A0046091A1047091A204452B462B472B54
:10B8C00009F490E0981789F0882309F4BDC1D501E7
:10B8D000C40180569444A24FBF4F80939F0490931D
:10B8E000A004A093A104B093A2044090300C509007
:10B8F000310C6090320C7090330C20919B0430918D
:10B900009C0440919D0450919E04C301B2010F9488
:10B910007D25882319F180919F049091A004A09126
:10B92000A104B091A20440929B0450929C046092A6
:10B930009D0470929E04892B8A2B8B2B09F449C09D
:10B94000D501C40180569444A24FBF4F80939F04F9
:10B950009093A004A093A104B093A20480919F04AB
:10B960009091A004A091A104B091A2040097A10518
:10B97000B10579F1881A990AAA0ABB0AB7FC29C04D
:10B9800010929F041092A0041092A1041092A2049D
:10B9900083E396E00E942C3860E08FE196E00E94FD
:10B9A0009A3F8091E9119091EA111816190624F432
:10B9B00090E080E00E94041F80917E1190917F11A1
:10B9C0001816190634F410927F1110927E110E94FD
:10B9D0007BBE8091A7049091A804A091A904B09186
:10B9E000AA0446015701881A990AAA0ABB0AD50176
:10B9F000C401B7FDB9C12091851290918612409182
:10BA00002D0280912C02291323C19091FD08899F5A
:10BA1000C0011124880F892F881F990B91958D8360
:10BA20008091FE08489FC0011124880F892F881F2C
:10BA3000990B91958E830E9457FD69837A838B833E
:10BA40009C8340E0BE016F5F7F4FCE0105960E9450
:10BA50004E1C6D8170E089E00E944EFC41E0BE0109
:10BA60006F5F7F4FCE0105960E944E1C6E8170E085
:10BA700087E00E944EFC80911806882309F467C174
:10BA80000091200210912102C80102972091E91132
:10BA90003091EA11281739070CF459C180908612A9
:10BAA0008F82188619861A861B86809185129F8040
:10BAB000891509F4E7C0892D90E03CE5A32EA89EE6
:10BAC000F001A99EF00D1124EE5FF64F45895689CD
:10BAD0006789708D452B462B472B81F4418D528D04
:10BAE000638D748D452B462B472B41F4458D568D28
:10BAF000678D70A1452B462B472BE1F12CE5B22E2B
:10BB0000B89E9001B99E300D1124A9014E5F564F89
:10BB10001A01FA0161817281838194810F94FB2E55
:10BB20004B015C01F10161A172A183A194A10F9469
:10BB300082252B013C01F10165A176A187A190A589
:10BB40000F9482259B01AC01C301B2010F94472DD4
:10BB5000A50194010F94E3254B015C0128853985EB
:10BB60004A855B850F94AD2E181624F48886998635
:10BB7000AA86BB868F818F5F87708F8396CF0E9446
:10BB8000FB4D609182077091830782EE95E00E94E1
:10BB90001C578AE00E94F33740E070E060E090E0DC
:10BBA00080E00E942E559091851280918612981700
:10BBB00049F0C0927211D0927311E0927411F09218
:10BBC000751158CEBB2019F01092AB0453CE0E94D1
:10BBD00057FD0091721110917311209174113091E1
:10BBE00075118090130290901402A0901502B090ED
:10BBF0001602080D191D2A1D3B1D601B710B820BBF
:10BC0000930B97FDE1CF8091AB04811133CE81E09E
:10BC10008093AB045F9A8091340C8E7F8093340CB8
:10BC20008A9A8091340C8D7F8093340C8091080126
:10BC300080958170809306018091340C8B7F809376
:10BC4000340C0E94E61E16CE80E090E0DC0145CE6A
:10BC5000209186125CE5259F900111242E5F364FBE
:10BC6000F901EA5AFF4F9081899FC0011124880F82
:10BC7000892F881F990B91958D83295A3F4FF90180
:10BC80008081D0CE20911A0230911B0240911C027B
:10BC900050911D02688579858A859B850F94E325DF
:10BCA0004B015C01B801012E000C880B990B0F941D
:10BCB00084259B01AC01C501B4010F944D2C69830F
:10BCC0007A838B839C8340911E0250911F02B8019E
:10BCD000CE0101960E94B3C189809A80AB80BC805E
:10BCE0004090A3045090A4046090A5047090A60412
:10BCF000A3019201C501B4010F947D2587FF16C0F1
:10BD000028E431EE4AE75FE3C301B2010F94E32573
:10BD100020E037ED43EA5CE30F944D2CA50194013C
:10BD20000F94E32569837A838B839C8369817A816D
:10BD30008B819C816093A3047093A4048093A504D9
:10BD40009093A6040F94B92DCB010E94041FF4E632
:10BD5000CF0ED11CE11CF11CC092A704D092A80404
:10BD6000E092A904F092AA040E94F5C18091E50630
:10BD7000882309F4E0C180912602882309F4A3C036
:10BD80008091E90481119FC080911F11811108C029
:10BD900080912011813021F080912D1482FF93C079
:10BDA000F894649B10C08091220290912302A0918C
:10BDB0002402B09125028093E6059093E705A093B5
:10BDC000E805B093E9056091E6057091E70580917B
:10BDD000E8059091E905789420E030E0A9010F94FE
:10BDE0007D2587FF70C001E00093E90480911F1159
:10BDF000811167C088E496E00E942C388AE00E9496
:10BE0000F33784E080939D0C82E08093890C81E07D
:10BE10009AE59093C4138093C3138EE490E09093BB
:10BE2000C6138093C51387E08093B71382E880938D
:10BE3000BA1384E890E0A0E0B0E08093BB13909345
:10BE4000BC13A093BD13B093BE1387E693E10E9489
:10BE50006F340E94174000938D1140E36CE876E048
:10BE600084E799E00E941C4061E088E699E00E9426
:10BE7000FE3F1091130560E010278CE399E069F410
:10BE80008AE796E00E94673F80E30E94F3378AE0EA
:10BE90000E94F33760E08DE596E00E94673F88E6F8
:10BEA00096E00E942C3880E30E94F3378AE00E94DB
:10BEB000F337112331F083E696E09093830C80935F
:10BEC000820C0E946B6190910901892F809581708D
:10BED000109100021817C9F020912D1420622093B0
:10BEE0002D148093000290FD3FC164EF71E080E06B
:10BEF00090E00E94F0250E941FB380912D1483FDD5
:10BF00007CC1111133C10E94C1350E9457FD6B01E4
:10BF10007C01109117021123F1F080911405882300
:10BF2000D1F04091AC045091AD046091AE04709199
:10BF3000AF0446015701841A950AA60AB70AB5014B
:10BF4000A40177FD1AC0833009F42FC10CF01EC183
:10BF500081300CF023C1212F30E0A8EEB3E00F9424
:10BF6000152CC60ED71EE81EF91EC092AC04D09246
:10BF7000AD04E092AE04F092AF04809120118130C4
:10BF800009F073C00E9457FD6B017C018091B404DD
:10BF90009091B504A091B604B091B704A7019601A1
:10BFA000281B390B4A0B5B0BDA01C901B7FD3AC0FC
:10BFB000D701C601805F984DAF4FBF4F8093B40447
:10BFC0009093B504A093B604B093B7048090AF05E6
:10BFD0009090B005A090B105B090B2050E94642B7E
:10BFE000AB01BC014093AF055093B0056093B10520
:10BFF0007093B2058091940690919506A091960653
:10C00000B091970688199909AA09BB09840F951F51
:10C01000A61FB71F8093940690939506A09396064B
:10C02000B09397068091B0049091B104A091B204AE
:10C03000B091B30446015701881A990AAA0ABB0AAB
:10C04000D501C401B7FD11C020E8C20E2EEED21EEC
:10C0500026E3E21EF11CC092B004D092B104E0923B
:10C06000B204F092B3040E94B0530E946A390E9455
:10C07000344180910E05882379F10E9457FD6B01B0
:10C080007C0180910A0590910B05A0910C05B0915F
:10C090000D0546015701881A990AAA0ABB0AD5015B
:10C0A000C401B7FD19C020910E0530E0A8EEB3E041
:10C0B0000F94152CC60ED71EE81EF91EC0920A0555
:10C0C000D0920B05E0920C05F0920D0580E00E94E5
:10C0D000D9BA8AE00E94F33780910905882359F183
:10C0E0000E9457FD6B017C0180910505909106052A
:10C0F000A0910705B0910805A7019601281B390BEF
:10C100004A0B5B0BDA01C901B7FD15C02091090587
:10C1100030E0A8EEB3E00F94152CC60ED71EE81E33
:10C12000F91EC0920505D0920605E0920705F0922F
:10C1300008050E94BAAA2B960FB6F894DEBF0FBE70
:10C14000CDBFDF91CF911F910F91FF90EF90DF90C6
:10C15000CF90BF90AF909F908F907F906F905F90A7
:10C160004F903F902F9008950E940EB3123008F028
:10C17000CCCE0E94C13560E085EC96E050C083EDE6
:10C1800096E09093830C8093820CBFCE843009F0AC
:10C19000E2CE0E94FF4D8AED96E004C00E94FF4D62
:10C1A00089E097E00E942C38D6CE0E94FF4D82EFA6
:10C1B00096E0F8CF8091840790918507A09186073B
:10C1C000B0918707A7019601281B390B4A0B5B0B1F
:10C1D000DA01C901885E9340A109B109B7FD46C9DA
:10C1E0008DEC95E00E942C38C0928407D092850790
:10C1F000E0928607F092870739C9123098F48DE9EA
:10C2000096E00E942C388AE00E94F3370E94932C1B
:10C2100090E080E00E94265760E086EB96E00E9466
:10C220009A3F73CE123009F070CE0E9479B78823FE
:10C2300079F081E00E944FB742EB50E06EE078E089
:10C2400082E394E10E9447B182E394E10E94F4B258
:10C250000E94692F811193CF0E94532F0E94F5B73E
:10C260000E944AB752CECF93DF938091851290916E
:10C270008612891B8095877019F40E94075AF5CFA2
:10C28000809185128F5F8770A09185129CE5A99F90
:10C29000D0011124FD01EE5FF64FEF0119929A953E
:10C2A000E9F798E09083A95EB64F90E1E7E8F2E104
:10C2B00001900D929A95E1F7209185129091861246
:10C2C000291303C094E69093821280938512DF9124
:10C2D000CF910C94812F90918512809186129813A2
:10C2E00006C08091000990910109892B21F080E01E
:10C2F0000E94075AF0CF0895FC01208131814281CC
:10C30000538160915A0C70915B0C80915C0C909100
:10C310005D0C0F94E3250F94BA2E609393127093E3
:10C320009412809395129093961290918512809119
:10C33000861298130C9433610E946B610E94F0295D
:10C3400040919312509194126091951270919612AF
:10C35000409308065093090660930A0670930B06F3
:10C3600081110C94812F08954F925F926F927F926A
:10C370008F929F92AF92BF92CF92DF92EF92FF92F5
:10C380000F931F93CF93DF93EC018B015A01F901B7
:10C3900020915A0C30915B0C40915C0C50915D0CDB
:10C3A00060817181828193810F94E3250F94BA2E6D
:10C3B0006B017C012091560C3091570C4091580C28
:10C3C0005091590CF50160817181828193810F94A4
:10C3D000E3250F94BA2E4B015C012091520C309151
:10C3E000530C4091540C5091550CF80160817181AF
:10C3F000828193810F94E3250F94BA2E2B013C0187
:10C4000020914E0C30914F0C4091500C5091510C9A
:10C41000688179818A819B810F94E3250F94BA2EDC
:10C4200060938712709388128093891290938A1276
:10C4300040928B1250928C1260928D1270928E12DA
:10C4400080928F1290929012A0929112B0929212BA
:10C45000C0929312D0929412E0929512F09296129A
:10C460009091851280918612981791F0DF91CF916B
:10C470001F910F91FF90EF90DF90CF90BF90AF9002
:10C480009F908F907F906F905F904F900C9433614E
:10C490000E946B610E94F02940918F12509190127E
:10C4A000609191127091921200918B1210918C12E6
:10C4B00020918D1230918E12C0908712D0908812E8
:10C4C000E0908912F0908A12C092FC05D092FD058E
:10C4D000E092FE05F092FF0500930006109301061E
:10C4E00020930206309303064093040650930506FA
:10C4F0006093060670930706409193125091941230
:10C500006091951270919612409308065093090617
:10C5100060930A0670930B06882391F0DF91CF9108
:10C520001F910F91FF90EF90DF90CF90BF90AF9051
:10C530009F908F907F906F905F904F900C94812F81
:10C54000DF91CF911F910F91FF90EF90DF90CF90EF
:10C55000BF90AF909F908F907F906F905F904F9023
:10C5600008953F924F925F926F927F928F929F9227
:10C57000AF92BF92CF92DF92EF92FF920F931F93F1
:10C58000CF93DF93CDB7DEB768970FB6F894DEBFD1
:10C590000FBECDBFD82E2A013B01480159013E2CC8
:10C5A00020E030E0A901C501B8010F947D2581117B
:10C5B00010C081E08D1508F0B6C060E070E080E743
:10C5C00093E420E030E040E752E40F94472D4B0124
:10C5D0005C018D8A9E8AAF8AB88E0D2D10E0F8011D
:10C5E000EA56F64EE491BB24B3941E160CF4B12C1B
:10C5F000CC24C39420E030E0A901C301B2010F9420
:10C60000AD2E18160CF0C12CBC1471F092E0D912AA
:10C610000BC0332049F081E00E9426F969E170E007
:10C6200080E090E00E94F02580E00E94872F6983DF
:10C630007A838B839C8381E00E94872F6D837E8326
:10C640008F83988782E00E94872F69877A878B87FC
:10C650009C8783E00E94872F6D877E878F87988BCA
:10C66000000F111F000F111FE1E0F0E0EC0FFD1FA4
:10C670000E0F1F1FF80110821182128213829E0179
:10C68000235F3F4FAE01475F5F4FBE016B5F7F4F40
:10C69000CE0101960E94B461F8014082518262820B
:10C6A0007382198A1A8A1B8A1C8A809100099091C8
:10C6B0000109892B91F4CE0141967C018E010B5E1C
:10C6C0001F4F9E01235F3F4FAE01475F5F4FBE018B
:10C6D0006B5F7F4F40970E94D0E70E946B61BC1454
:10C6E00051F092E0D91205C0332019F080E00E9489
:10C6F00026F90E94EB5568960FB6F894DEBF0FBE80
:10C70000CDBFDF91CF911F910F91FF90EF90DF9000
:10C71000CF90BF90AF909F908F907F906F905F90E1
:10C720004F903F90089560E070E88BE395E449CF27
:10C730004F925F926F927F928F929F92AF92BF9231
:10C74000CF92DF92EF92FF920F931F93CF93DF93DD
:10C75000CDB7DEB72C970FB6F894DEBF0FBECDBFB6
:10C760002B013C0129873A874B875C874701580199
:10C77000F601E080F1800281138120E030E0A90120
:10C78000B701C8010F947D25882309F488C05E2D68
:10C790004F2D302F212F852F942FA32FB22F898338
:10C7A0009A83AB83BC8320E030E0A901B701C801C4
:10C7B0000F947D25811108C0E0903D02F0903E026B
:10C7C00000913F0210914002C701D8018D839E83E2
:10C7D000AF83B887A501940160912C0C70912D0C4A
:10C7E00080912E0C90912F0C0F947D2587FF0CC00B
:10C7F00080922C0C90922D0CA0922E0CB0922F0CAB
:10C80000CE0101960E94CB2A4092240C5092250C16
:10C810006092260C7092270C89859A85AB85BC8521
:10C820008093280C9093290CA0932A0CB0932B0C86
:10C83000CE0105960E94CB2AA501940160912C0C93
:10C8400070912D0C80912E0C90912F0C0F94AD2E89
:10C85000181664F480922C0C90922D0CA0922E0C41
:10C86000B0922F0CCE0101960E94CB2A0E946B61E0
:10C870002C960FB6F894DEBF0FBECDBFDF91CF91DF
:10C880001F910F91FF90EF90DF90CF90BF90AF90EE
:10C890009F908F907F906F905F904F90089550E0A1
:10C8A00040E030E820E477CFCF92DF92EF92FF9222
:10C8B0000F931F936A01E0902C0CF0902D0C0091C7
:10C8C0002E0C10912F0CFB0120813181428153816C
:10C8D000FC0160817181828193810E9498631F9124
:10C8E0000F91FF90EF90DF90CF900895CF92DF925D
:10C8F000EF92FF920F931F936B01FC01E080F18098
:10C9000002811381E4E2FCE0248135814681578174
:10C9100060817181828193810E9498631F910F9140
:10C92000FF90EF90DF90CF9008950F931F93CF93D8
:10C93000DF93EC018B0181E00E9426F969E170E050
:10C9400080E090E00E94F025B801CE010E9476645C
:10C95000C091E40680E00E9426F91092E40682E08D
:10C960000E94B12F0E94E62AC2FBCC27C0F981E0C9
:10C970008C27DF91CF911F910F910895AF92BF92B5
:10C98000CF92DF92EF92FF920F931F93CF93DF939B
:10C9900000D01F92CDB7DEB7FC01E080F1800281AC
:10C9A0001381611112C0A0902C0CB0902D0CC0907E
:10C9B0002E0CD0902F0C9501A601B701C8010F9441
:10C9C0007D2587FF02C07501860120E030E04BEE37
:10C9D00053E4B701C8010F947D2587FD04C0E12C05
:10C9E000F12C0BEE13E4C701D80189839A83AB8342
:10C9F000BC8362EE72E0CE0101960E9476640F90D5
:10CA00000F900F900F90DF91CF911F910F91FF909A
:10CA1000EF90DF90CF90BF90AF9008953F924F92EC
:10CA20005F926F927F928F929F92AF92BF92CF92BE
:10CA3000DF92EF92FF920F931F93CF93DF9300D07B
:10CA40001F92CDB7DEB7382E80E090E0A0E2B1E4CF
:10CA500089839A83AB83BC83C0907C12D0907D1273
:10CA6000E0907E12F0907F1220E030E0A901C70133
:10CA7000B6010F947D2587FF0CC0A701960160E0E9
:10CA800070E080E291E40F944C2C69837A838B836D
:10CA90009C8360E0CE0101960E94BE644090240C0D
:10CAA0005090250C6090260C7090270C8090280CDC
:10CAB0009090290CA0902A0CB0902B0C332089F177
:10CAC0000E94B65419821A821B821C82E0902C0CA0
:10CAD000F0902D0C00912E0C10912F0CCE01019690
:10CAE0006C01A5019401C301B2010E9498633092C8
:10CAF00080070E94552B0F900F900F900F90DF91A1
:10CB0000CF911F910F91FF90EF90DF90CF90BF904A
:10CB1000AF909F908F907F906F905F904F903F90DD
:10CB200008950E947354CECF80918007882319F016
:10CB300080E00E940E6580E008952F923F924F9210
:10CB40005F926F927F928F929F92AF92BF92CF929D
:10CB5000DF92EF92FF920F931F93CF93DF93CDB7A6
:10CB6000DEB766970FB6F894DEBF0FBECDBFF82EC6
:10CB7000282E312CF101EA56F64ED49022E0821391
:10CB800035C080918007811103C081E00E940E654D
:10CB90000E94B654811139C182E999E10E946D1D4C
:10CBA00020E030E0A9010F947D258823F9F06D2D58
:10CBB000DD0C770B880B990B0F9484252B013C011E
:10CBC00082E999E10E946D1D4B015C0120E030E09B
:10CBD00040EA50E40F947D2511E087FF1CC0812CB2
:10CBE000912C90EAA92E90E4B92E15C06D2DDD0C84
:10CBF000770B880B990B0F9484252B013C01C10105
:10CC0000880F991F880F991F8657964E0E946D1D99
:10CC10004B015C0110E0A3019201C501B4010F9426
:10CC2000E3254B015C016101CC0CDD1CCC0CDD1C4F
:10CC3000C6018258964E0E946D1DEE24E394E126B3
:10CC400020E030E040EC5FE30F94E325A301920184
:10CC50000F94E325AB01BC0100E010E098018F2D9B
:10CC60000E94B16220E030E0A901C501B4010F9437
:10CC70007D25F601EE58F64EFA8BE98B882309F4F0
:10CC80004DC0F2E000E010E020E431E4FF1619F0BE
:10CC900000E010E09801B501A4017058E12C8F2D3F
:10CCA0000E94B162A5019401C501B4010F944D2CFD
:10CCB0006B8B7C8B8D8B9E8B22E0F216E9F0F10161
:10CCC000E159F64E6491611107C00E94FF4D8DE459
:10CCD00099E10E942C386AE070E090E080E00F94C7
:10CCE00082259B01AC0160E070E088E492E40F943F
:10CCF000472D8B019C0104C000E010E020EC30E4E3
:10CD0000EE24E3944B895C896D897E898F2D0E9486
:10CD1000B16232E0F312D0C00E94735481E090E01F
:10CD2000A0E0B0E00F2C04C0880F991FAA1FBB1F02
:10CD30000A94D2F72091340C282B2093340C2091A4
:10CD40009A05822B80939A0589899A890E946D1D84
:10CD5000F601EC5DF34F608371838283938382E0FD
:10CD6000F8121AC020917C1230917D1240917E12EF
:10CD700050917F1260912C0C70912D0C80912E0C93
:10CD800090912F0C0F944C2C60932C0C70932D0CC5
:10CD900080932E0C90932F0CF601EA50F84F1082DE
:10CDA0001182128213828F2D0E948A1C0E94E62A11
:10CDB000F601EC5DF34F80819181A281B381F60190
:10CDC000E059F84F80839183A283B38392E0F916F0
:10CDD000A9F18CE0EEEAF2E0DE01119601900D92ED
:10CDE0008A95E1F7E1E0F0E0EC0FFD1FEC0DFD1D91
:10CDF00080809180A280B38020E030E0A901C5014D
:10CE0000B4010F947D2581111EC066960FB6F8946B
:10CE1000DEBF0FBECDBFDF91CF911F910F91FF906D
:10CE2000EF90DF90CF90BF90AF909F908F907F90CA
:10CE30006F905F904F903F902F9008950E9494655F
:10CE40008111E3CFC6CF20E030E0A901C501B401D4
:10CE50000F94AD2E87FF04C0B7FAB094B7F8B09422
:10CE6000F601EC5DF34F6F01A3019201C501B4011E
:10CE70000F94E3259B01AC01F601608171818281F1
:10CE800093810F944C2CF60160837183828393838A
:10CE9000F2E080E090E0A0E4B1E4FF1621F080E051
:10CEA00090E0A8E4B2E48D879E87AF87B88BCE016F
:10CEB0000D960E94CB2AA9CF81E090E0A0E0B0E0DF
:10CEC0000F2C04C0880F991FAA1FBB1F0A94D2F70A
:10CED0002091340C282B2093340C20919A05822B1E
:10CEE00080939A0589899A890E946D1DF601EC5DEF
:10CEF000F34F60837183828393834ECFCF93DF930D
:10CF000000D01F92CDB7DEB780E090E0A0EAB0E499
:10CF100089839A83AB83BC8361E0CE0101960E9432
:10CF2000BE640F900F900F900F90DF91CF910895F6
:10CF30008F929F92AF92BF92CF92DF92EF92FF9229
:10CF40000F931F93CF93DF93CDB7DEB72C970FB618
:10CF5000F894DEBF0FBECDBF8B0140E050E068E427
:10CF600072E44D835E836F83788740E050E060EA2F
:10CF700070E449875A876B877C878130B9F18230AA
:10CF800009F459C020E030E040E050E460912C0CFE
:10CF900070912D0C80912E0C90912F0C0F944D2C94
:10CFA0004B017C0120E030E04BEE53E40F94AD2EBA
:10CFB000181634F4812C912C8BEEE82E93E4F92E84
:10CFC000F801A084B184C284D3849401A701B5017F
:10CFD000C6010F94AD2E181614F054016701C50157
:10CFE000D60189839A83AB83BC8348C0BE01675F47
:10CFF0007F4FC80108960E947664B8016C5F7F4F2E
:10D00000AE014B5F5F4FC8010E9454640E948130A3
:10D010002C960FB6F894DEBF0FBECDBFDF91CF9137
:10D020001F910F91FF90EF90DF90CF90BF90AF9046
:10D030009F908F900895F801208531854285538512
:10D0400060912C0C70912D0C80912E0C90912F0CD6
:10D050000F944D2C6B017C0120E030E04BEE53E44B
:10D060000F947D2587FD06C0C12CD12C2BEEE22E1E
:10D0700023E4F22EC982DA82EB82FC82BE01675F72
:10D080007F4FCE010196B7CFEF92FF920F931F9380
:10D09000CF93DF937C018B010E947B31C4E2DCE003
:10D0A00020916102309162024091630250916402CA
:10D0B000F70160817181828193810F94472D2C85C6
:10D0C0003D854E855F850F944D2C6C877D878E87BF
:10D0D0009F87C8010E94CB2ADF91CF911F910F91AA
:10D0E000FF90EF900C946B614F925F926F927F92E2
:10D0F000AF92BF92CF92DF92EF92FF920F931F9366
:10D10000CF93DF9300D000D01F921F92CDB7DEB730
:10D110005C0180E090E0A0E7B2E489839A83AB836E
:10D12000BC8380E090E0A0E8B0EC8D839E83AF8369
:10D13000B887BE016F5F7F4FCE0105960E9444689D
:10D1400068E873E180E090E00E94F025C12CD12CCA
:10D1500088ECE82E81E4F82EC982DA82EB82FC8228
:10D1600080E090E0A0E8B0E48D839E83AF83B88731
:10D17000BE016F5F7F4FCE0105960E9444680AE3AF
:10D180001CE0F80140AC51AC62AC73ACC0AED1AEA7
:10D19000E2AEF3AE80E090E0A0EAB1E489839A8346
:10D1A000AB83BC83F50180819181A281B3818D83A2
:10D1B0009E83AF83B887BE016F5F7F4FCE01059618
:10D1C0000E944468F80140AE51AE62AE73AE129A4E
:10D1D00064E670E080E090E00E94F02581E028960F
:10D1E0000FB6F894DEBF0FBECDBFDF91CF911F9178
:10D1F0000F91FF90EF90DF90CF90BF90AF907F9016
:10D200006F905F904F9008951F93CF93DF93CDB7AA
:10D21000DEB72C970FB6F894DEBF0FBECDBF182F28
:10D22000882379F020E030E0A9016091D205709167
:10D23000D3058091D4059091D5050F947D25882341
:10D24000F9F08091350C8117D9F00E946B618CE068
:10D25000EAEBF2E0DE01119601900D928A95E1F77A
:10D26000CE0101960E94191F8091350C882391F000
:10D2700084E29CE00E94F2261092350C0E94E62A7D
:10D280002C960FB6F894DEBF0FBECDBFDF91CF91C5
:10D290001F91089581E08093350C84E29CE00E9408
:10D2A0000621ECCF2F923F924F925F926F927F9226
:10D2B0008F929F92AF92BF92CF92DF92EF92FF92A6
:10D2C0000F931F93CF93DF93CDB7DEB7CB54D10924
:10D2D0000FB6F894DEBF0FBECDBF2DB73EB739AF46
:10D2E00028AF87E00E940F4E81110BC061E086E5F8
:10D2F0000E943E248DA3853060F087E39EE00E946B
:10D300002C38A8ADB9AD0FB6F894BEBF0FBEADBFF7
:10D3100040C33DA1332321F087E19EE00E942C38D9
:10D320006AE080E50E943E24182F8CEF810F8F3237
:10D3300018F083EF9DE0E3CF60E085E40E945A247B
:10D34000882309F448C081E08FABE0908012F09010
:10D350008112D7012D913D914D915C916091240CEA
:10D360007091250C8091260C9091270C0F944D2CD8
:10D37000AB01BC0188E50E94AC2469877A878B8762
:10D380009C87F70124813581468157816091280C63
:10D390007091290C80912A0C90912B0C0F944D2C9C
:10D3A000AB01BC0189E50E94AC246D877E878F8725
:10D3B000988BBE01635F7F4FCE0109960E94212E9C
:10D3C000382E81110BC063E68FED9DE00E949A3FDD
:10D3D00087EC9DE094CF92E09FABB7CF8CE40E94A6
:10D3E0002E1E082F882309F431C10E942A248EA3FF
:10D3F000803118F080EA9DE082CFFEA1F13009F47F
:10D4000027C160E083E50E945A248AAF882321F077
:10D41000011102C037E03EA38DA1833020F086E8E1
:10D420009DE00E942C389091350C9DAF80E00E94C9
:10D4300004690E94C31C1D8A1E8A1F8A188E198EB9
:10D440001A8E1B8E1C8E83EF9FE4A3ECB7E48D8FA6
:10D450009E8FAF8FB8A383EF9FE4A3ECB7EC89A3B3
:10D460009AA3ABA3BCA3A12FB0E0BCA7ABA7EDB719
:10D47000FEB724E0129FE019F10911240FB6F894C9
:10D48000FEBF0FBEEDBF8DB79EB701969CAF8BAFB1
:10D490002DA14FA9BE01635F7F4FCE0109960E9467
:10D4A000B5F99B01AC010F943F2F811162C20E941C
:10D4B00057FD611571058105910511F00F94032148
:10D4C000212C1BAA1CAA1DAA1EAAAEA1A150BB0BEF
:10D4D0002C96BFAFAEAF2C97E22DF0E0F8A7EFA3EC
:10D4E0002BA53CA5E217F3070CF074C23196FEA7FA
:10D4F000EDA73F932F93FF93EF9382E79DE09F93D8
:10D500008F938CE79DE09F938F931F920E9444F925
:10D510008DB79EB709960FB6F8949EBF0FBE8DBF0C
:10D520009EA1992309F458C10F94B4202AE030E059
:10D5300040E050E00F94E32B0F94842520E030E08E
:10D5400040EA50E40F94AD2E0FEF1FEF181614F0C1
:10D5500001E010E00F94B42028E631E040E050E014
:10D560000F94E32B0F9484252B013C010F94B420DE
:10D5700023E330E040E050E00F94E32B6B5F7F4FFC
:10D580008F4F9F4F0F9484254B015C01ADA1A430B8
:10D59000D1F4BC01A40184E69DE00E940841B301DE
:10D5A000A2018CE59DE00E94084186E59DE00E9475
:10D5B0002C380130110519F483E40E94F33782E519
:10D5C0009DE00E942C38312CC801110FAA0BBB0B17
:10D5D0002A968CAF9DAFAEAFBFAF2A972C96AEAD5B
:10D5E000BFAD2C973A161B060CF0F6C02A966CAD10
:10D5F0007DAD8EAD9FAD2A970F9484256B017C0184
:10D60000BAADBB2341F1AC019B010F944D2C20E03E
:10D6100030E040E952E40F94E3259B01AC01C301E3
:10D62000B2010F944D2C2B013C0120E030E044EB83
:10D6300053E40F94AD2E1816FCF420E030E044EBD8
:10D6400053E4C301B2010F944C2CEDCF1EA2D9CEEE
:10D6500022E02EA3D6CE0F94B42024E130E040E0A7
:10D6600050E00F94E32B675E7F4F8F4F9F4F0F94D7
:10D670008425A7019601CFCF20E030E0A901C301A6
:10D68000B2010F947D2587FF0BC020E030E044EB12
:10D6900053E4C301B2010F944D2C2B013C01ECCF9C
:10D6A0000091801210918112F80124813581468108
:10D6B00057816D857E858F8598890F944C2C229695
:10D6C0006CAF7DAF8EAF9FAF22972BED3FE049E46B
:10D6D00050E4C301B2010F94E32520E030E044E3BD
:10D6E00053E40F94472D6B017C010F94422D6FA7DB
:10D6F00078AB89AB9AABD8012D913D914D915C915E
:10D7000069857A858B859C850F944C2C26966CAF09
:10D710007DAF8EAF9FAF2697A50194016FA578A925
:10D7200089A99AA90F94E3259B01AC0126966CADBB
:10D730007DAD8EAD9FAD26970F944D2C69837A8376
:10D740008B839C83C701B6010F94ED2EA501940134
:10D750000F94E32522962CAD3DAD4EAD5FAD2297E3
:10D760000F944D2C6D837E838F83988742EC51E01C
:10D7700070E060E0CE0101960E94B3C142EC51E03E
:10D7800070E060E0CE0105960E94B3C1BDA1B43047
:10D7900099F449815A816B817C8186E49DE00E94E5
:10D7A00008414D815E816F81788584E39FE20E940C
:10D7B00008418AE00E94F337198A1A8A1B8A1C8A58
:10D7C000AE014F5E5F4FBE016B5F7F4FCE01019692
:10D7D0000E945464339402CF20E04FA9BE01635FDE
:10D7E0007F4FCE0109960E94B5F94B015C01312CA7
:10D7F000AC019B010F943F2F811102C0332433945D
:10D80000A5019401C501B4010F943F2F8111E2C01D
:10D81000EFA1F8A5EE0FFF1FEE0FFF1F2BAD3CADE4
:10D82000E20FF31F80829182A282B382A50194014C
:10D830006D8D7E8D8F8D98A10F94AD2E181624F4CA
:10D840008D8E9E8EAF8EB8A2A501940169A17AA19A
:10D850008BA19CA10F947D2587FF04C089A29AA269
:10D86000ABA2BCA2A50194016BA97CA98DA99EA91C
:10D870000F944D2C6BAB7CAB8DAB9EABADA5BEA519
:10D88000BD01BB0F880B990B0F9484256FA378A75C
:10D8900089A79AA79B01AC016BA97CA98DA99EA918
:10D8A0000F94472D2B013C014D8A5E8A6F8A788E3A
:10D8B000EBADFCADF8ABEFA710E0C12CD12C76019D
:10D8C000AFA5B8A96D917D918D919D91B8ABAFA792
:10D8D000A30192010F944C2C9B01AC010F94E32502
:10D8E0009B01AC01C701B6010F944D2C6B017C016B
:10D8F0001F5F211628F72FA138A549A55AA50F9417
:10D90000472D0F94FB2E698F7A8F8B8F9C8FBDA133
:10D91000B23068F18DA59EA50E9474E16BA57CA52F
:10D9200081E49DE00E942A418BE39DE00E942C3817
:10D9300043E0C501B4010E9435BA80E20E94F3378A
:10D9400081E0EDA1E3300CF480E0E12C8E010F5D6D
:10D950001F4F9E01235E3F4FAE01475E5F4FBE01EA
:10D960006B5E7F4F0E94E93E8AE00E94F33723946A
:10D97000B3CD0E9494650E94AA1C8DAD0E940469DB
:10D980000E94813088AD99AD0FB6F8949EBF0FBE4E
:10D990008DBFE8ADF9AD0FB6F894FEBF0FBEEDBF79
:10D9A000C55BDF4F0FB6F894DEBF0FBECDBFDF9172
:10D9B000CF911F910F91FF90EF90DF90CF90BF908C
:10D9C000AF909F908F907F906F905F904F903F901F
:10D9D0002F9008950E949465332069F280E39DE0C2
:10D9E0000E942C3881E0FDA11F160CF080E0EE248F
:10D9F000E3948E010F5D1F4F9E01235E3F4FAE01EA
:10DA0000475E5F4FBE016B5E7F4F0E94E93E698DAE
:10DA10007A8D8B8D9C8D0052110926E042E00F9487
:10DA20004A209F938F938FE19DE09F938F9389E28C
:10DA30009DE09F938F931F920E9444F92DB73EB7AC
:10DA4000295F3F4F0FB6F8943EBF0FBE2DBF93CF57
:10DA50002F923F924F925F926F927F928F929F92FE
:10DA6000AF92BF92CF92DF92EF92FF920F931F93EC
:10DA7000CF93DF93CDB7DEB76A970FB6F894DEBFCA
:10DA80000FBECDBF83E50E942E1E182F3090350C9F
:10DA9000882319F00E944A24382E4090240C50907C
:10DAA000250C6090260C7090270C8091280C90918A
:10DAB000290CA0912A0CB0912B0C8B8B9C8BAD8BDD
:10DAC000BE8B80912C0C90912D0CA0912E0CB091BE
:10DAD0002F0C8F8B988FA98FBA8F112329F03110BB
:10DAE00003C080E00E94046986E50E942E1E8A8B96
:10DAF00020E030E0A9016091D2057091D3058091BA
:10DB0000D4059091D5050F947D25882309F4C9C0CB
:10DB100083E40E942E1E882309F49DC00E94822463
:10DB20006B017C01ACE8B7E0B987A887BF83AE83FF
:10DB3000F5E0FD831D861E8628EC2F8702EC1A86F1
:10DB4000212C88EC8B8792E49C87AE81BF81B98BB6
:10DB5000A88B15E0E889F98981909190A190B19006
:10DB6000F98BE88B2A85322D4B855C85C501B40184
:10DB70000F947D2587FF04C08A86292CAB86BC863E
:10DB80002D853E854F85502FC501B4010F94AD2ED4
:10DB9000181624F48D869E86AF860B2D1150D1F673
:10DBA000FD81F150FD838E819F8144969F838E83FA
:10DBB000F111CBCF2D853E854F85502F6A85722D73
:10DBC0008B859C850F944D2C20E030E040E05FE396
:10DBD0000F94E325A70196010F944D2C4B015C0196
:10DBE0002DEB37E346E855EB0F94AD2E87FD0AC0C9
:10DBF0002DEB37E346E855E3C501B4010F947D25CD
:10DC000018164CF580E00E94046910E0E884F9845D
:10DC100000E0D7016D917D918D919D917D016D0108
:10DC2000B4E0CB1AD108A50194010F944C2CF60155
:10DC30006083718382839383602F812F0E9419F800
:10DC40000F5F053031F71F5F888599854496998766
:10DC500088871530D9F6AA89AA2381F020E030E020
:10DC6000A9016091D2057091D3058091D40590915E
:10DC7000D5050F947D2581110E9471408AE50E948F
:10DC80002E1E882351F00E94822469837A838B831D
:10DC90009C83CE0101960E94E1F6832D0E940469C7
:10DCA0000BC0311003C09A89992341F30E94FF4DA4
:10DCB00080E69CE00E942C38332051F08091350C96
:10DCC000811106C00E94FB4D81E49CE00E942C382B
:10DCD0000E94FF4D83E39CE00E942C388091350C1C
:10DCE0000E94EA400E94FF4D86E29CE00E942C3890
:10DCF000C090C808D090C908E090CA08F090CB083E
:10DD000020E030E0A901C701B6010F94AD2E18162E
:10DD10000CF053C042E0C701B6010E9435BA8DE055
:10DD20000E94F3378AE00E94F337A30192016091C9
:10DD3000240C7091250C8091260C9091270C0F9447
:10DD40007D2581111FC02B893C894D895E89609199
:10DD5000280C7091290C80912A0C90912B0C0F9417
:10DD60007D2581110FC02F89388D498D5A8D609185
:10DD70002C0C70912D0C80912E0C90912F0C0F94E7
:10DD80007D2581110E9481306A960FB6F894DEBF1E
:10DD90000FBECDBFDF91CF911F910F91FF90EF90FC
:10DDA000DF90CF90BF90AF909F908F907F906F90BB
:10DDB0005F904F903F902F90089581E29CE00E94E9
:10DDC0002C38B3CF8F929F92AF92BF92EF92FF9277
:10DDD0000F931F93CF93DF9380E00E94046910920A
:10DDE000CE051092CF051092D0051092D105109259
:10DDF000CA051092CB051092CC051092CD05109259
:10DE0000D6051092D7051092D8051092D905109218
:10DE1000D2051092D3051092D4051092D5050CE8C6
:10DE200017E0C0E0812C912C80ECA82E8FE7B82E53
:10DE30007801D0E0F70181929192A192B1927F0195
:10DE40006D2F8C2F0E9419F8DF5FD53099F7CF5FC7
:10DE50000C5E1F4FC53061F7DF91CF911F910F917D
:10DE6000FF90EF90BF90AF909F908F90089590910A
:10DE7000851280918612981308C0809100099091B4
:10DE80000109892B11F40C94E81E80E00E94075AC6
:10DE9000EECF83E50E947C1E8823E9F00E9457FDA7
:10DEA0006093721170937311809374119093751134
:10DEB0000E94822420E030E04AE754E40F94E325F6
:10DEC0000F94C02D60931302709314028093150277
:10DED0009093160208958091330584FD0AC08091C5
:10DEE000350587FD06C080913605837011F40C94CA
:10DEF000376F0E946B6188E50E942E1E882331F0E7
:10DF00005F9A8091340C8E7F8093340C89E50E9457
:10DF10002E1E882331F08A9A8091340C8D7F809355
:10DF2000340C8AE50E942E1E882359F08091080146
:10DF300080958170809306018091340C8B7F809353
:10DF4000340C85E40E942E1E81110C94E61E089567
:10DF50002F923F924F925F926F927F928F929F92F9
:10DF6000AF92BF92CF92DF92EF92FF920F931F93E7
:10DF7000CF93DF93CDB7DEB7A6970FB6F894DEBF89
:10DF80000FBECDBF80E797E00E94132A8091E20B7D
:10DF900083FD7EC02091300C3091310C4091320CC9
:10DFA0005091330C60917C0770917D0780917E07C2
:10DFB00090917F070F947D25882309F469C0109103
:10DFC000FF08111161C080915F029091600201977A
:10DFD0002091E7113091E811281739073CF40E948D
:10DFE000FF4D80E299E10E942C3811E02091300C25
:10DFF0003091310C4091320C5091330C60917C0780
:10E0000070917D0780917E0790917F070F944C2C33
:10E010006B017C0120E030E0A9010F94AD2E87FF59
:10E0200004C0F7FAF094F7F8F0942091610230916F
:10E0300062024091630250916402C701B6010F94DD
:10E04000E32520E030E84BE354E40F94AD2E18169E
:10E05000ECF40E94FF4D81E099E10E942C38809100
:10E060007C0790917D07A0917E07B0917F078093F8
:10E07000300C9093310CA093320CB093330C8CE79E
:10E0800097E00E947C6104C010E0B0CF1111E7CF8F
:10E090002AE037ED43E25CE3609141027091420275
:10E0A00080914302909144020F94E3256B017C011F
:10E0B0006091670270916802072E000C880B990B23
:10E0C0000F9484259B01AC01C701B6010F94E32591
:10E0D000698B7A8B8B8B9C8B8091350C882309F113
:10E0E0008090C8089090C908A090CA08B090CB084A
:10E0F000C0907807D0907907E0907A07F0907B077E
:10E1000020E030E0A901C501B4010F947D258823EA
:10E11000D1F1A7019601C501B4010F94AD2E1816D7
:10E1200094F1C12CD12C76018E010F5E1F4F2CE78C
:10E1300037E048E757E064E777E080E797E00E9440
:10E140009AF480E1E0E7F7E0A4E2BCE001900D92F0
:10E150008A95E1F7A6960FB6F894DEBF0FBECDBF45
:10E16000DF91CF911F910F91FF90EF90DF90CF90B3
:10E17000BF90AF909F908F907F906F905F904F90E7
:10E180003F902F9008952091240C3091250C4091C0
:10E19000260C5091270C6091700770917107809147
:10E1A0007207909173070F944C2C6D8B7E8B8F8B25
:10E1B000988F2091280C3091290C40912A0C509175
:10E1C0002B0C609174077091750780917607909180
:10E1D00077070F944C2C698F7A8F8B8F9C8F2091AF
:10E1E0002C0C30912D0C40912E0C50912F0CC7010E
:10E1F000B6010F944C2C6D8F7E8F8F8F98A320913A
:10E20000300C3091310C4091320C5091330C6091B4
:10E210007C0770917D0780917E0790917F070F9416
:10E220004C2C6B017C0120E030E0A9016D897E89D6
:10E230008F89988D0F947D2581110CC020E030E0EE
:10E24000A901698D7A8D8B8D9C8D0F947D258823F6
:10E2500009F467CF2D893E894F89588DCA01B901CC
:10E260000F94E3254B015C01298D3A8D4B8D5C8D1C
:10E27000CA01B9010F94E3259B01AC01C501B401AA
:10E280000F944D2C4B015C012D8D3E8D4F8D58A16F
:10E29000CA01B9010F94E3259B01AC01C501B4018A
:10E2A0000F944D2C4B015C01A7019601C701B601EB
:10E2B0000F94E3259B01AC01C501B4010F944D2CD3
:10E2C0000F94FB2E4B015C012DEB37E346E855E341
:10E2D0000F947D2587FF0FC020E030E0A901C70122
:10E2E000B6010F94AD2E4601570187FF04C0B7FA5F
:10E2F000B094B7F8B0942DEB37E346E855E3C50189
:10E30000B4010F947D2587FD1CCF20E030E040EA6A
:10E3100051E4C501B4010F94472D0F94C02D1B018A
:10E32000672B19F422242394312CB10190E080E072
:10E330000F9482259B01AC0160E070E080E89FE3D0
:10E340000F94472D2B013C01AC019B01C501B40189
:10E350000F94E3254B015C01A30192016D897E8935
:10E360008F89988D0F94E3256D8B7E8B8F8B988F83
:10E37000A3019201698D7A8D8B8D9C8D0F94E3257D
:10E38000698F7A8F8B8F9C8FA30192016D8D7E8D0B
:10E390008F8D98A10F94E3256D8F7E8F8F8F98A31B
:10E3A000A3019201C701B6010F94E32569A37AA3E3
:10E3B0008BA39CA380E1E4E2FCE08E010F5F1F4F82
:10E3C000D80101900D928A95E1F70E9457FD2B012B
:10E3D0003C0128EC420E511C611C711C0DA31EA3B4
:10E3E00081E0281A310809F460C00E9457FD8B01B2
:10E3F0009C01041915092609370937FD59C02B015D
:10E400003C0128EC420E511C611C711C80E00E94F2
:10E41000075A2D893E894F89588D69817A818B8170
:10E420009C810F944D2C69837A838B839C83298DE7
:10E430003A8D4B8D5C8D6D817E818F8198850F9497
:10E440004D2C6D837E838F8398872D8D3E8D4F8DD0
:10E4500058A169857A858B859C850F944D2C698799
:10E460007A878B879C8729A13AA14BA15CA16D85F6
:10E470007E858F8598890F944D2C6D877E878F8739
:10E48000988B750164018E010F5E1F4F9E01235F03
:10E490003F4FAE01475F5F4FBE016B5F7F4F8DA166
:10E4A0009EA10E949AF481119BCF750164013CCE1C
:10E4B0000E94F5C1AECF8F929F92AF92BF92CF9242
:10E4C000DF92EF92FF92CF93DF9380904102909082
:10E4D0004202A0904302B0904402FC01C080D1806F
:10E4E000E280F38020E030E0A901C701B6010F947B
:10E4F0007D25882341F0C0924102D0924202E092F1
:10E500004302F0924402C0916702D091680284E60F
:10E5100090E09093680280936702C0906102D0906F
:10E520006202E0906302F090640280E090E0A0E874
:10E53000BFE38093610290936202A0936302B09361
:10E5400064020E94A86F8092410290924202A092BF
:10E550004302B0924402D0936802C0936702C09213
:10E560006102D0926202E0926302F0926402DF9153
:10E57000CF91FF90EF90DF90CF90BF90AF909F90A2
:10E580008F9008950F931F93CF93DF9300D01F9226
:10E59000CDB7DEB79C0100E717E090E1E4E2FCE0D4
:10E5A000D80101900D929A95E1F7F901208131810E
:10E5B00042815381F80160857185828593850F942E
:10E5C0004D2CF801608771878287938780E090E007
:10E5D000A0EAB0E489839A83AB83BC83CE01019621
:10E5E0000E945B720F900F900F900F90DF91CF9170
:10E5F0001F910F9108952F923F924F925F926F92C9
:10E600007F928F929F92AF92BF92CF92DF92EF92C2
:10E61000FF921F93CF93DF93CDB7DEB72C970FB642
:10E62000F894DEBF0FBECDBF7A011901DC012D9138
:10E630003D914D915C912D833E834F835887FB0123
:10E6400040805180628073808090240C9090250CD3
:10E65000A090260CB090270CA50194016D817E81BD
:10E660008F8198850F947D2581110EC011E0A30143
:10E6700092016091280C7091290C80912A0C909144
:10E680002B0C0F947D25811110E0D1012D913D912E
:10E690004D915C9129873A874B875C87F701C08051
:10E6A000D180E280F38020910B0230910C024091E6
:10E6B0000D0250910E02C701B6010F947D258823EB
:10E6C00009F44EC0C0920B02D0920C02E0920D02EF
:10E6D000F0920E028091300C9091310CA091320C8E
:10E6E000B091330C4091280C5091290C60912A0C68
:10E6F00070912B0C8092700790927107A092720714
:10E70000B092730740937407509375076093760730
:10E7100070937707C0927807D0927907E0927A07D2
:10E72000F0927B0780937C0790937D07A0937E07F0
:10E73000B0937F0720E030E040E05FE36091660C3B
:10E740007091670C8091680C9091690C0F94E3258F
:10E7500069837A838B839C83CE0101960E945B72CE
:10E760002D813E814F81588520937007309371072A
:10E770004093720750937307409274075092750745
:10E780006092760770927707D1012D913D914D915E
:10E790005C9160917C0770917D0780917E079091DC
:10E7A0007F070F944D2C60937C0770937D078093B7
:10E7B0007E0790937F0711112FC020E030E0A90160
:10E7C00069857A858B859C850F947D25811133C061
:10E7D00060E070E088EC92E469837A838B839C83A9
:10E7E000CE0101960E945B722C960FB6F894DEBFA4
:10E7F0000FBECDBFDF91CF911F91FF90EF90DF90C3
:10E80000CF90BF90AF909F908F907F906F905F90D0
:10E810004F903F902F9008952AEF3EE74AE25FE342
:10E8200060916A0C70916B0C80916C0C90916D0CE6
:10E830000F94E325D1CF60E070E080EA91E4CCCF83
:10E840000F931F93CF93DF9300D000D01F921F929E
:10E85000CDB7DEB78B01FC0123A5211102C00E94B8
:10E86000A2FB1D821E821F82188620E030E040E05D
:10E870005FE360912C0C70912D0C80912E0C909187
:10E880002F0C0F944D2C69837A838B839C839E017C
:10E890002B5F3F4FAE014F5F5F4F68E27CE084E249
:10E8A0009CE00E94FB721D821E821F82188620E05F
:10E8B00030E040E05FE3F8016085718582859385F3
:10E8C0000F944D2C69837A838B839C83B8016C5F92
:10E8D0007F4F9E012B5F3F4FAE014F5F5F4FC801DF
:10E8E0000E94FB7228960FB6F894DEBF0FBECDBF14
:10E8F000DF91CF911F910F9108959B01AC01485F6B
:10E900005F4FBC016C5F7F4F0C94FB722F923F9264
:10E910004F925F926F927F928F929F92AF92BF922F
:10E92000CF92DF92EF92FF920F931F93CF93DF93DB
:10E93000CDB7DEB7A6970FB6F894DEBF0FBECDBF3A
:10E940008C011B015A8749874090240C5090250C5C
:10E950006090260C7090270C8090280C9090290CC9
:10E96000A0902A0CB0902B0CDB018D919D910D9005
:10E97000BC91A02D8B8B9C8BAD8BBE8B9C01AD0174
:10E98000C301B2010F944C2C6B017C01D101149690
:10E990008D919D910D90BC91A02D8F8B988FA98FFB
:10E9A000BA8F9C01AD01C501B4010F944C2C6B8F43
:10E9B0007C8F8D8F9E8FA985BA858D919D910D90AD
:10E9C000BC91A02D8B879C87AD87BE879C01AD0134
:10E9D000C301B2010F944C2C6F8F78A389A39AA323
:10E9E000A985BA8514968D919D910D90BC91A02D0D
:10E9F0008F87988BA98BBA8B9C01AD01C501B4019F
:10EA00000F944C2C6BA37CA38DA39EA3A70196010E
:10EA1000C701B6010F94E3256B017C012B8D3C8D62
:10EA20004D8D5E8DCA01B9010F94E3259B01AC01A8
:10EA3000C701B6010F944D2C4B015C012B893C8919
:10EA40004D895E896B857C858D859E850F944C2CC8
:10EA50002B013C012F89388D498D5A8D6F8578891E
:10EA600089899A890F944C2C6B017C01A301920136
:10EA7000C301B2010F94E3252B013C01A7019601CC
:10EA8000C701B6010F94E3259B01AC01C301B2019C
:10EA90000F944D2C0F94FB2E6B017C012F8D38A110
:10EAA00049A15AA1CA01B9010F94E3252B013C01E8
:10EAB0002BA13CA14DA15EA1CA01B9010F94E32590
:10EAC0009B01AC01C301B2010F944D2C9B01AC0121
:10EAD000C501B4010F94AD2E1816B4F520E030E056
:10EAE000A901C701B6010F94AD2E87FF2AC0C70147
:10EAF000B601905820E030E040EA50E40F94AD2E8B
:10EB0000181614F5A10169857A85C8010E948674DA
:10EB1000A6960FB6F894DEBF0FBECDBFDF91CF91A2
:10EB20001F910F91FF90EF90DF90CF90BF90AF902B
:10EB30009F908F907F906F905F904F903F902F901D
:10EB40000895C701B601D6CF20E030E040E050E4A0
:10EB5000C501B4010F94AD2E181624F4B101C801FB
:10EB60000E94207419821A821B821C82BE016F5F70
:10EB70007F4FC1010E947D742DEC3CEC4CEC5CE3BA
:10EB8000C701B6010F94E3259B01AC01F801608138
:10EB90007181828193810F94E3256D837E838F83BE
:10EBA0009887D8019B968C919B978823C9F02AE976
:10EBB00039E949E95FE314966D917D918D919C91BE
:10EBC00017970F94E32569837A838B839C83BE0117
:10EBD0006F5F7F4F80E797E00E947D74F80113A676
:10EBE000BE016B5F7F4F89859A850E947D7490CFAF
:10EBF0003F924F925F926F927F928F929F92AF92CD
:10EC0000BF92CF92DF92EF92FF920F931F93CF9319
:10EC1000DF93CDB7DEB76C970FB6F894DEBF0FBEAB
:10EC2000CDBFDB010C91142F100F153008F067C118
:10EC30001196DC90C22ECD0CB4E0BC1508F45FC177
:10EC4000ED2DF0E0E650FB4F8080912CB12CA12CF3
:10EC5000002E04C0B694A794979487940A94D2F790
:10EC600080FE4DC1EC2DF0E0E650FB4F8080912CF2
:10EC7000B12CA12C012E04C0B694A794979487942C
:10EC80000A94D2F780FE3BC1322E642F7C01409063
:10EC9000CA055090CB056090CC057090CD05809151
:10ECA000D2059091D305A091D405B091D505898F57
:10ECB0009A8FAB8FBC8F660F770B072E000C880BDB
:10ECC000990B0F9484254B015C01602F000F770B8B
:10ECD000880B990B0F948425298D3A8D4B8D5C8D73
:10ECE0000F94E325A30192010F944D2CA5019401EB
:10ECF0000F944D2C6D877E878F87988B612F110F16
:10ED0000770B880B990B0F948425298D3A8D4B8DA9
:10ED10005C8D0F94E325A30192010F944D2CA50166
:10ED200094010F944C2C69837A838B839C8340904D
:10ED3000CE055090CF056090D0057090D1058091A0
:10ED4000D6059091D705A091D805B091D905898FA6
:10ED50009A8FAB8FBC8F632D660F770B072E000C3D
:10ED6000880B990B0F9484254B015C016D2DDD0CF4
:10ED7000770B880B990B0F948425298D3A8D4B8D39
:10ED80005C8D0F94E325A30192010F944D2CA501F6
:10ED900094010F944D2C698B7A8B8B8B9C8B6C2DF3
:10EDA000CC0C770B880B990B0F948425298D3A8D09
:10EDB0004B8D5C8D0F94E325A30192010F944D2C94
:10EDC000A50194010F944C2C6D837E838F839887CB
:10EDD000F70180859185A285B38589879A87AB875E
:10EDE000BC878D8B9E8BAF8BB88F41EC51E061E07F
:10EDF00070E0CE0141960E94B3C141EC51E061E068
:10EE000070E0CE0105960E94B3C141EC51E061E093
:10EE100070E0CE010D960E94B3C141EC51E061E07B
:10EE200070E0CE0101960E94B3C189889A88AB88B0
:10EE3000BC8827E137EB41ED58EBC501B4010F94D5
:10EE4000AD2E87FD5CC023E030E041EE53E4C50108
:10EE5000B4010F947D2518160CF451C08D849E8446
:10EE6000AF84B88827E137EB41ED58EBC501B40119
:10EE70000F94AD2E87FD43C023E030E041EE53E414
:10EE8000C501B4010F947D251816CCF18D809E80AC
:10EE9000AF80B88427E137EB41ED58EBC501B401F1
:10EEA0000F94AD2E87FD2BC023E030E041EE53E4FC
:10EEB000C501B4010F947D2518160CF189809A8044
:10EEC000AB80BC8027E137EB41ED58EBC501B401C5
:10EED0000F94AD2E87FD13C023E030E041EE53E4E4
:10EEE000C501B4010F947D2518164CF0AE014F5F9B
:10EEF0005F4FBE01635F7F4FC7010E9486746C96AF
:10EF00000FB6F894DEBF0FBECDBFDF91CF911F913A
:10EF10000F91FF90EF90DF90CF90BF90AF909F90B8
:10EF20008F907F906F905F904F903F9008952F92B9
:10EF30003F924F925F926F927F928F929F92AF9289
:10EF4000BF92CF92DF92EF92FF920F931F93CF93D6
:10EF5000DF93CDB7DEB7CC58D1090FB6F894DEBF3A
:10EF60000FBECDBF80E19CE00E942C3887E00E945C
:10EF70000F4E81116EC084E50E947C1E882329F00B
:10EF80000E946F2481110E9423BA80E090E0A0E8E3
:10EF9000BFE389839A83AB83BC838D839E83AF83D6
:10EFA000B8878DEC9CECACE4BEE389879A87AB878D
:10EFB000BC8780E090E0A0E2B1E48D879E87AF87B8
:10EFC000B88B8CE390E09A8B898B8DEC90E09C8BD6
:10EFD0008B8B8DEC9CECACECBEE38D8B9E8BAF8B66
:10EFE000B88F80E090E0A0EEBFE3898F9A8FAB8F5F
:10EFF000BC8F1BA61CA64AE959E969E97EE38FE4A8
:10F000000E94AC246D8F7E8F8F8F98A360E083E485
:10F010000E945A2489A360E08BE40E945A248AA3A8
:10F0200082E40E947C1E882381F10E946F24009755
:10F0300061F19C01285231092536310520F16CE837
:10F0400070E082EE9BE00E942A418DED9BE00E94E1
:10F050002C38C457DF4F0FB6F894DEBF0FBECDBFBC
:10F06000DF91CF911F910F91FF90EF90DF90CF90A4
:10F07000BF90AF909F908F907F906F905F904F90D8
:10F080003F902F9008959A8B898B8CE40E947C1E70
:10F090008823E1F00E9482246B017C01C986DA8614
:10F0A000EB86FC8620E030E0A9010F94AD2E87FDB1
:10F0B0000AC020E030E040E050E4C701B6010F9400
:10F0C0007D2518161CF485EB9BE0C1CF81E50E94DD
:10F0D0002E1E882331F18091030590910405892B20
:10F0E000E9F00E9482246B017C01CD82DE82EF82F6
:10F0F000F8862DEC3CEC4CE45DE30F94AD2E87FDDF
:10F100000AC020E030E040E751E4C701B6010F94A7
:10F110007D25181634F484E89BE099CF89E59BE0BF
:10F1200096CF83E50E947C1E8823E9F00E9482240A
:10F130006B017C01CD8ADE8AEF8AF88E2DEC3CECE7
:10F140004CEC5DE30F94AD2E87FD0AC020E030E06B
:10F1500040E050E4C701B6010F947D2518161CF459
:10F1600082E39BE074CF80E50E942E1E882341F14C
:10F170008091030590910405892B19F48AEF9AE098
:10F1800066CF8BA58F5F8BA70E9482246B017C01C9
:10F19000CD86DE86EF86F88A20E030E0A9010F9464
:10F1A000AD2E87FD0AC020E030E048EC51E4C701F5
:10F1B000B6010F947D2518161CF482ED9AE047CF16
:10F1C00086E40E947C1E8823E9F00E9482246B0161
:10F1D0007C01C98EDA8EEB8EFC8E20E030E040E8B8
:10F1E0005FE30F94AD2E87FD0AC020E030E040E8D9
:10F1F00050E4C701B6010F947D2518161CF489EA66
:10F200009AE025CFC98CDA8CEB8CFC8C8D889E889B
:10F21000AF88B88CA7019601C701B6010F94E3250A
:10F220009B01AC0160E070E084E490E40F94472D12
:10F2300029813A814B815C810F94E3252B013C01AC
:10F24000A5019401C501B4010F94E325A70196011E
:10F250000F94E3252CEE31E548EB5DE30F94472D49
:10F260009B01AC01C301B2010F94E32569837A834A
:10F270008B839C8388E40E947C1E882379F00E9403
:10F280006F24009759F09C01255A31092F303140E5
:10F2900018F08BE79AE0DBCE9C8B8B8B85E50E9488
:10F2A0002E1E8823C9F00E9457FD61157105810546
:10F2B000910511F00F9403218091030590910405AD
:10F2C000892B91F00E9482246093FF0470930005C3
:10F2D000809301059093020582E50E942E1E811104
:10F2E00008C087E49AE0B3CE60E070E088E492E47E
:10F2F000EBCF8091030590910405892B61F00E946A
:10F300006F24AD969FAF8EAFAD97181619064CF0CF
:10F3100083E19AE09CCE8AE190E0AD969FAF8EAFFC
:10F32000AD9789E50E947C1E882381F10E9482248A
:10F330002091D0083091D1084091D2085091D30843
:10F340000F944C2C6B017C0188E50E947C1E882365
:10F3500031F10E9482242091CC083091CD08409157
:10F36000CE085091CF080F944C2C6BA37CA38DA397
:10F370009EA3CFA2D8A6E9A6FAA6CE0183960E94A4
:10F38000ED1D811115C089EE99E061CEC090280C69
:10F39000D090290CE0902A0CF0902B0CD5CF6091E6
:10F3A000240C7091250C8091260C9091270CDDCFB8
:10F3B00084E40E942E1E91E089270E94046980E067
:10F3C00090E0A0EAB0E48DA79EA7AFA7B8AB60E03D
:10F3D000CE018D960E94BE649091F507CD57DF4F08
:10F3E0009883C358D0401092F5070E94E71B88EC21
:10F3F00099E00E942C3889899A898A3191050CF00C
:10F4000044C08B899C890E94041F61E080E00E94B7
:10F41000C3BC811142C06FEF8DED99E00E949A3F0D
:10F420008CA5811104C0CE0101960E94A2FB80E050
:10F4300090E0A0EAB0E48093780790937907A093D6
:10F440007A07B0937B071DA61EA61FA618AABE01A9
:10F45000635D7F4F80E797E00E947D74CD57DF4F5B
:10F460005881C358D0405093F5070E94E71B8AA1EA
:10F470008111EFCD10927F1110927E110E947BBE00
:10F4800090E080E00E94041FE4CD0E94422281E0CF
:10F490000E944CBB8111B5CFBECF1092300C1092A0
:10F4A000310C1092320C1092330C80E39CE00E94DD
:10F4B0007C618BA5882309F452C020E030E040E74E
:10F4C00051E460916A0C70916B0C80916C0C90917E
:10F4D0006D0C0F94472D6DA77EA78FA798AB80E189
:10F4E000E4E2FCE0A0E7B7E001900D928A95E1F735
:10F4F0002D853E854F85588960917C0770917D07E9
:10F5000080917E0790917F070F944D2C60937C072C
:10F5100070937D0780937E0790937F07CE018D9631
:10F520000E945B722D853E854F85588960917C07CE
:10F5300070917D0780917E0790917F070F944C2CEE
:10F5400060937C0770937D0780937E0790937F077D
:10F550008CA5811104C0CE0101960E94A2FBEAEFA6
:10F56000F4E085E0DF011D928A95E9F780E1E4E2AD
:10F57000FCE0A0E7B7E001900D928A95E1F789855C
:10F580009A85AB85BC858093780790937907A09383
:10F590007A07B0937B071DA61EA61FA618AABE0158
:10F5A000635D7F4F80E797E00E947D74BE01635EDC
:10F5B0007F4F80E797E00E947D7489A1882309F43A
:10F5C0001CC42091240C3091250C4091260C5091A4
:10F5D000270CE5962CAF3DAF4EAF5FAFE59780911E
:10F5E000280C9091290CA0912A0CB0912B0CE1963B
:10F5F0008CAF9DAFAEAFBFAFE197312C212C9FEF09
:10F60000A4969FAFA497AFEFA896AFAFA897BFEF10
:10F61000C158DF4FB883CF57D040EFE4C058DF4F19
:10F62000E883C058D040F3ECCF57DF4FF883C15880
:10F63000D04027E4CE57DF4F2883C258D04081E026
:10F6400090E0A0E0B0E0022C04C0880F991FAA1F30
:10F65000BB1F0A94D2F7CC57DF4F88839983AA83C4
:10F66000BB83C458D040AAEFB4E0E796BFAFAEAFBB
:10F67000E79710E000E09101032C000C440B550BC0
:10F68000C857DF4F288339834A835B83C858D040EB
:10F69000C457DF4F2882CC58D040E796AEADBFADFF
:10F6A000E7978D91E796BFAFAEAFE79790E0B0E0F8
:10F6B000A0E0CC57DF4F288139814A815B81C45853
:10F6C000D04082239323A423B523892B8A2B8B2B11
:10F6D00009F024C1C857DF4F688179818A819B81F5
:10F6E000C858D0400F9484252091D2053091D3057D
:10F6F0004091D4055091D5050F94E3252091CA057A
:10F700003091CB054091CC055091CD050F944D2CF7
:10F71000EB966CAF7DAF8EAF9FAFEB97B801012E2C
:10F72000000C880B990B0F9484252091D6053091FD
:10F73000D7054091D8055091D9050F94E325209124
:10F74000CE053091CF054091D0055091D1050F9451
:10F750004D2C6B017C01EB962CAD3DAD4EAD5FADFC
:10F76000EB97E5966CAD7DAD8EAD9FADE5970F94B3
:10F770004C2C2B013C01A7019601E1966CAD7DADAF
:10F780008EAD9FADE1970F944C2C4B015C01A30112
:10F790009201C301B2010F94E3252B013C01A501A5
:10F7A0009401C501B4010F94E3259B01AC01C30191
:10F7B000B2010F944D2C0F94FB2E4B015C01EB9684
:10F7C0002CAD3DAD4EAD5FADEB976BA17CA18DA196
:10F7D0009EA10F944C2C2B013C01A70196016FA117
:10F7E00078A589A59AA50F944C2C6B017C01A301E7
:10F7F0009201C301B2010F94E3252B013C01A70143
:10F800009601C701B6010F94E3259B01AC01C3012A
:10F81000B2010F944D2C0F94FB2E20E030E040E716
:10F8200051E40F94472DA50194010F944D2C6B01C9
:10F830007C018090FF0490900005A0900105B0909D
:10F84000020520E030E040E85FE3C501B4010F9419
:10F85000AD2E1816F4F4C501B4010F94B92D4B0167
:10F860005C0160E070E0CB01181419041A041B0459
:10F8700034F40F94B420A50194010F94E32B0F945A
:10F8800084259B01AC01B601C7010F944D2C6B017F
:10F890007C01C158DF4F2881CF57D040C058DF4F7F
:10F8A0003881C058D040CF57DF4F4881C158D04031
:10F8B000CE57DF4F5881C258D040B601C7010F94D0
:10F8C0007D2587FF2BC0A4960FAFA497C457DF4FA9
:10F8D0003881CC58D040A8963FAFA897EC96CFAED1
:10F8E000EC97ED96DFAEED97EE96EFAEEE97EF96D6
:10F8F000FFAEEF97C158DF4FC882CF57D040C058F6
:10F90000DF4FD882C058D040CF57DF4FE882C15870
:10F91000D040CE57DF4FF882C258D0400F5F1F4F04
:10F920000530110509F0B9CE4FEF241A340A55E01D
:10F930002516310409F083CEA4968FADA497E82F45
:10F94000F0E0E650FB4F208181E090E0A0E0B0E0E5
:10F95000A8960FACA89704C0880F991FAA1FBB1FB9
:10F960000A94D2F7822B8083A8969FADA8976A96B7
:10F970009FAF6A97A496AFADA4976B96AFAF6B9706
:10F98000EC968FADEC97ED969FADED97EE96AFAD03
:10F99000EE97EF96BFADEF976F968CAF9DAFAEAF82
:10F9A000BFAF6F97A896BFADA897BF3F09F409C234
:10F9B000A496EFADA497EF3F09F403C26B2FBB0FE2
:10F9C000770B880B990B0F9484252091D2053091E9
:10F9D000D3054091D4055091D5050F94E32520918E
:10F9E000CA053091CB054091CC055091CD050F94BF
:10F9F0004D2C162F072F382E292E862F902FA32D12
:10FA0000B22D65968CAF9DAFAEAFBFAF6597A49694
:10FA1000FFADA4976F2FFF0F770B880B990B0F94F7
:10FA200084252091D6053091D7054091D805509175
:10FA3000D9050F94E3252091CE053091CF05409153
:10FA4000D0055091D1050F944D2C6B017C01699626
:10FA5000CCAEDDAEEEAEFFAE6997CE018F5A9F4FB2
:10FA60000E94ED1D882309F4B0C120E030E040EA97
:10FA700050E4612F702F832D922D0F944D2C4B014C
:10FA80005C01CB01D50121968CAF9DAFAEAFBFAF6E
:10FA900021972596CCAEDDAEEEAEFFAE2597A896AB
:10FAA0002FADA8972111E3C1A4963FADA4973111C2
:10FAB000B3C120E030E040EA50E4C701B6010F9442
:10FAC0004D2C6B017C01A4964FADA497442309F4FF
:10FAD000C5C1A4968FADA49784300CF0BFC122EDB0
:10FAE000422E23E5522E2BE7622E21E4722E219620
:10FAF0008CAC9DACAEACBFAC219725968CAD9DADCA
:10FB0000AEADBFAD2597A7968CAF9DAFAEAFBFAFE3
:10FB1000A7979C01AD0169966CAD7DAD8EAD9FAD93
:10FB200069970F944C2CAB966CAF7DAF8EAF9FAFA7
:10FB3000AB97A501940165966CAD7DAD8EAD9FAD83
:10FB400065970F944C2C2D966CAF7DAF8EAF9FAF09
:10FB50002D97AB962CAD3DAD4EAD5FADAB9761969D
:10FB60002CAF3DAF4EAF5FAF6197A501940160919F
:10FB7000240C7091250C8091260C9091270C0F94E9
:10FB80004C2C4B015C01A7962CAD3DAD4EAD5FAD4D
:10FB9000A7976091280C7091290C80912A0C909164
:10FBA0002B0C0F944C2CA7966CAF7DAF8EAF9FAFF4
:10FBB000A797812F902FA32DB22D8DA79EA7AFA71A
:10FBC000B8ABC9AADAAAEBAAFCAAC984DA84EB8486
:10FBD000FC84CDAADEAAEFAAF8AE2DEC3CEC4CECEE
:10FBE0005CE3C301B2010F94E32529813A814B8183
:10FBF0005C810F94E3252091300C3091310C4091C1
:10FC0000320C5091330C0F944D2C69AF7AAF8BAFFF
:10FC10009CAFA5019401C501B4010F94E3254B01EC
:10FC20005C01A7962CAD3DAD4EAD5FADA797CA0167
:10FC3000B9010F94E3259B01AC01C501B4010F94F8
:10FC40004D2C20E030E040E050E40F94AD2E18162B
:10FC5000ACF420E030E040E05FE3C701B6010F9470
:10FC60004D2C29966CAF7DAF8EAF9FAF2997BE010B
:10FC7000635C7F4FCE0101960E94207489859A852E
:10FC8000AB85BC8529968CAF9DAFAEAFBFAF299732
:10FC9000A3961CAE1DAE1EAE1FAEA397BE01615A49
:10FCA0007F4FCE01CD960E947D748CA58823C1F034
:10FCB0002AE939E949E95FE36D817E818F81988581
:10FCC0000F94E325A3966CAF7DAF8EAF9FAFA39744
:10FCD000BE01615A7F4F80E797E00E947D741CA6A9
:10FCE000E090620CF090630C0091640C1091650C34
:10FCF000A0905E0CB0905F0CC090600CD090610C36
:10FD00009501A601B701C8010F94AD2E181614F481
:10FD1000750186018090410290904202A0904302BA
:10FD2000B09044022DEC3CEC4CEC5DE3B701C80113
:10FD30000F94E32560934102709342028093430243
:10FD40009093440240E0BE01675B7F4FCE018D96E9
:10FD50000F94B51480E1E4E2FCE0A0E7B7E0019085
:10FD60000D928A95E1F78092410290924202A09210
:10FD70004302B092440220E04FEFBE01675A7F4F2A
:10FD8000CE0101960E94F87520E041E0BE01675A5D
:10FD90007F4FCE0101960E94F8752FEF40E0BE0123
:10FDA000675A7F4FCE0101960E94F87521E040E02E
:10FDB000BE01675A7F4FCE0101960E94F8750E94DE
:10FDC0006B618091A00C8093A10CAD964EAD5FADA0
:10FDD000AD9741505109AD965FAF4EAFAD97452BF2
:10FDE00009F419CB6A968FAD6A9787FD14CB6B9691
:10FDF0008FAD6B9787FFE1CB0ECB2BA13CA14DA123
:10FE00005EA1E5962CAF3DAF4EAF5FAFE5978FA1FA
:10FE100098A5A9A5BAA5EBCB812F902FA32DB22D24
:10FE200021968CAF9DAFAEAFBFAF219720E030E001
:10FE300040EA50E4C701B6010F944C2C25966CAFF4
:10FE40007DAF8EAF9FAF2597A4965FADA49754303A
:10FE50000CF42FCE182D092D3A2C2B2C92ED492E77
:10FE600093E5592E9BEF692E90E4792E40CEA8960B
:10FE70009FADA89794300CF452C0A496AFADA49750
:10FE8000A4300CF120E030E040EA50E4612F702F04
:10FE9000832D922D0F944C2C21966CAF7DAF8EAF9D
:10FEA0009FAF219720E030E040EA50E4C701B6015F
:10FEB0000F944C2C6B017C01A496EFADA497E43019
:10FEC0000CF40DCECBCF812F902FA32DB22D2196E8
:10FED0008CAF9DAFAEAFBFAF219720E030E040EADE
:10FEE00050E4C701B6010F944D2C25966CAF7DAF41
:10FEF0008EAF9FAF2597A496BFADA497B111D2CF77
:10FF000020E030E040EA50E4612F702F832D922DE5
:10FF10000F944C2C162F072F382E292E9FCFA496E6
:10FF2000FFADA497F1110DC020E030E040E251E4B4
:10FF3000B401C5010F944C2C162F072F382E292EF3
:10FF4000CECDA4962FADA49724309CF020E030E0D5
:10FF500040E251E4B401C5010F944C2C21966CAFE2
:10FF60007DAF8EAF9FAF2197182D092D3A2C2B2CEA
:10FF7000B6CD182D092D3A2C2B2C82ED482E83E579
:10FF8000582E8BEF682E81E4782EB1CD2F923F92C0
:10FF90004F925F926F927F928F929F92AF92BF9299
:10FFA000CF92DF92EF92FF920F931F93CF93DF9345
:10FFB000CDB7DEB7EE970FB6F894DEBF0FBECDBF5C
:10FFC0008091350C888B87E50E942E1E882309F4CA
:10FFD00023C120E030E0A9016091D2057091D305E2
:10FFE0008091D4059091D5050F947D25811108C08D
:10FFF0000E94FB4D8DE09DE00E942C3810E01FC157
:020000021000EC
:100000008AE50E947C1E882339F10E948224209177
:10001000D4083091D5084091D6085091D7080F9454
:100020004C2C6B017C0120E030E040E251ECC70138
:10003000B6010F94AD2E87FD0AC020E030E040E20B
:1000400051E4C701B6010F947D25181674F40E947F
:10005000FB4D80E09DE0D0CFC0902C0CD0902D0CBB
:10006000E0902E0CF0902F0CDECF40E050E060ECE2
:100070007FE788E50E94AC242091CC083091CD0820
:100080004091CE085091CF080F944C2C2B013C018D
:1000900040E050E060EC7FE789E50E94AC242091CD
:1000A000D0083091D1084091D2085091D3080F94D4
:1000B0004C2C4B015C016FEF89E40E943E24182F09
:1000C0006FEF8AE40E943E24082FA3019201C3012E
:1000D000B2010F943F2F81116EC0A5019401C5019B
:1000E000B4010F943F2F811166C08BA19CA1ADA1DB
:1000F000BEA18BAB9CABADABBEAB2091CA05309122
:10010000CB054091CC055091CD05C301B2010F94B0
:100110004C2C2B013C0120E030E040E05FE36BA978
:100120007CA98DA99EA90F94E3259B01AC01C30175
:10013000B2010F944D2C2BA93CA94DA95EA90F9497
:10014000472D0F94B92D162F4FA058A469A47AA457
:100150002091CE053091CF054091D0055091D10529
:10016000C501B4010F944C2C4B015C0120E030E040
:1001700040E05FE3C301B2010F94E3259B01AC01B2
:10018000C501B4010F944D2CA30192010F94472D8A
:100190000F94B92D062F812F012E000C990B97FD7E
:1001A00033C005979CF5802F002E000C990B97FD0E
:1001B0002FC005977CF5153008F020CF053008F0EA
:1001C0001DCF80E00E94046995E01902F00111241E
:1001D000E00FF11D07FDFA95EE0FFF1FEE0FFF1F59
:1001E000E457F84FC082D182E282F382602F812FE0
:1001F0000E9419F888890E9404698889882309F473
:10020000FDCE0E948130FACE10E0CDCF14E0CBCFEE
:1002100000E0D1CF04E0CFCF8AE40E942E1E182F39
:10022000811127C070E060E086E50E9473249A8304
:100230008983059708F18BED9CE00E942C38812F73
:10024000EE960FB6F894DEBF0FBECDBFDF91CF9113
:100250001F910F91FF90EF90DF90CF90BF90AF90E4
:100260009F908F907F906F905F904F903F902F90D6
:1002700008950E94E26EC2CE60E084E40E945A2497
:100280008F8740E050E0BA018AE50E94AC246BA75A
:100290007CA78DA79EA740E050E86BE376E483E55A
:1002A0000E94AC2420E030E040E752E40F94472D58
:1002B00060933D0270933E0280933F029093400210
:1002C000E0908012F0908112D7018D909D90AD90BA
:1002D000BC9020E030E0A901C501B4010F944D2C81
:1002E0006BAF7CAF8DAF9EAF20E030E040E450E4D8
:1002F0000F947D2587FF06C01BAE1CAEB0E4BDAFDA
:10030000E0E4EEAF20E030E041EE53E4C501B4019B
:100310000F944D2C662E7BAB8FAB98AF20E030E86E
:100320004FED53E40F94AD2E18163CF4612CF0E819
:10033000FBAB2FED2FAB33E438AFD70114968D9084
:100340009D90AD90BC90179720E030E0A901C501C9
:10035000B4010F944D2CD62EE72EF82E092F20E055
:1003600030E040E951E40F947D2587FF05C0D12C92
:10037000E12CF0E9FF2E01E420E030E041EE53E40F
:10038000C501B4010F944D2CB62EC72E89AF9AAF7C
:1003900020E030E048ED53E40F94AD2E181634F40D
:1003A000B12CC12CB8EDB9AFE3E4EAAF88E40E9408
:1003B0002E1E882309F416C20E9482240F94B92DA0
:1003C0001B0177FF02C06F5F7F4F75956795719531
:1003D000619571096F517F4F072E000C880B990BA7
:1003E0000F948425762E872E982EA92E2D2D3E2D06
:1003F0004F2D502F0F94AD2E18161CF4D72C7401CE
:100400000A2D2BAD3CAD4DAD5EAD672D782D892D00
:100410009A2D0F94AD2E181624F07BAC8CAC9DACAD
:10042000AEAC872D982DA92DBA2D8B8B9C8BAD8BC7
:10043000BE8B8D2D9E2DAF2DB02F8F8B988FA98FBA
:10044000BA8FB101330C880B990B0F9484251B01D3
:100450002C01AC019B016D2D7E2D8F2D902F0F94C3
:100460004D2CD62EE72EF82E092F2B2D3C2D49ADE5
:100470005AAD0F947D2587FF04C0BD2CCE2CF9AE5C
:100480000AAFA2019101672D782D892D9A2D0F9425
:100490004D2CD62EE72EF82E092F262D3BA94FA93D
:1004A00058AD0F947D2587FF04C06D2CEBAAFFAAE1
:1004B00008AF862D9BA9AFA9B8AD8B8F9C8FAD8F50
:1004C000BE8F8B2D9C2DA9ADBAAD8F8F98A3A9A3FC
:1004D000BAA3BE01695E7F4FCE0143960E94212ED2
:1004E000882309F4B0C1BE01615E7F4FCE014B96F7
:1004F0000E94212EE82E882309F4A5C12F89388D6A
:10050000498D5A8D6F8D78A189A19AA10F944C2C99
:1005100020E030E040E85EE30F94E3254B015C010E
:100520002B893C894D895E896B8D7C8D8D8D9E8D4F
:100530000F944C2C20E030E040E85EE30F94E3257C
:100540006BA37CA38DA39EA38FA298A6A9A6BAA6EF
:1005500089819A811816190674F489EA9CE00E9430
:100560002C388F85882321F08FE99CE00E942C385D
:100570008AE00E94F3370E946B610E94C31C80E0F6
:100580000E94046980E090E0A0E2B1E48FA798ABFC
:10059000A9ABBAAB60E0CE018F960E94BE642091F9
:1005A000D2053091D3054091D4055091D5056BA16A
:1005B0007CA18DA19EA10F947D25811130C0209139
:1005C000D6053091D7054091D8055091D9056FA136
:1005D00078A589A59AA50F947D25811120C0209129
:1005E000CA053091CB054091CC055091CD056B8962
:1005F0007C898D899E890F947D25811110C0209161
:10060000CE053091CF054091D0055091D1056F892D
:10061000788D898D9A8D0F947D258823A9F00E946D
:10062000E26E88E0FE01B396A2EDB5E001900D9276
:100630008A95E1F788E0FE017396AAECB5E0019097
:100640000D928A95E1F7188A60E085E40E945A24A9
:10065000882309F4FBC0F1E0FBAB1B861C861D86DA
:100660001E861A8A9E2C4FE6C42E4CE0D42E5DE7DF
:10067000A52E5CE0B52E1A8915300CF0F7C06B85FD
:100680007C858D859E859B01AC010F943F2F811148
:10069000EDC0992009F4DDC031E03FAB35E0232EF9
:1006A00091E09926F12EFF0CFF0CF10EF394898B4B
:1006B00019896A89121509F4D5C0062E000C770B2A
:1006C000880B990B0F9484252FA138A549A55AA50D
:1006D0000F94E3252F89388D498D5A8D0F944D2C19
:1006E0002B013C01612F110F770B880B990B0F9495
:1006F00084252BA13CA14DA15EA10F94E3252B895C
:100700003C894D895E890F944D2C6B837C838D834E
:100710009E834F82588669867A8689819A81892B41
:1007200079F06F2D8BE89CE00E94004169E170E058
:1007300089E89CE00E942A4186E89CE00E942C38CF
:100740001F9299E19F931F92FF92DF92CF92BF92E7
:10075000AF921F920E9444F929814BA9BE01695FA3
:100760007F4FCE0103960E94B5F92B013C014B86C9
:100770005C866D867E860FB6F894DEBF0FBECDBF59
:10078000AC019B010F943F2F811169C089883A8881
:1007900025E0382D320380011124030D111D37FC93
:1007A0001A95000F111F000F111F0457184FA301B6
:1007B00092016BA57CA58DA59EA50F944D2CD8010B
:1007C0006D937D938D939C931397632D882D0E9439
:1007D00019F8188A81E00E94075AF3948989BFA901
:1007E0008B0F65CF4D2D5E2D6F2D702F86E40E94EF
:1007F000AC241B012C014BAD5CAD6DAD7EAD8CE42A
:100800000E94AC246B8B7C8B8D8B9E8B2F8A388EB9
:10081000498E5A8E4B2D5C2D69AD7AAD82E40E94D3
:10082000AC246B017C01462D5BA96FA978AD82E5F4
:100830000E94AC246B8F7C8F8D8F9E8FCF8ED8A221
:10084000E9A2FAA246CE8FEB9CE0F7CC22E02BABDC
:1008500004CF8FEF8FAB22242A9484E021CF8889A4
:100860000E9404698A898F5F8A8B05CF0E94AFE45A
:100870000E949465882359F088890E94046980E069
:1008800090E0A0ECBFE78B879C87AD87BE876B8528
:100890007C858D859E859B01AC010F943F2F811136
:1008A00059C08F85811126C082E0F82E02E094E0C5
:1008B000C92E12E0DC2CD11A21E041E0612F802FFB
:1008C0000E945B2221E04FEF612F8F2D0E945B225F
:1008D0002FEF41E06D2D802F0E945B222FEF4FEF15
:1008E0006D2D8F2D0E945B22115020F70150F39443
:1008F0000F3FF9F60E9471400E94891E8F85811179
:1009000024C08CE29CE00E94731D4B015C0184E2D8
:100910009CE00E94191F9B01AC01C501B4010F941A
:10092000E3259B01AC0160912C0C70912D0C809102
:100930002E0C90912F0C0F944C2C60932C0C7093D8
:100940002D0C80932E0C90932F0C8F858111E888AD
:10095000E092350C0E94AA1C8091350C81110E94F6
:10096000E62A0E947E670E9481306B857C858D859A
:100970009E8511E09B01AC010F943F2F81115FCC4C
:100980003DCB8F929F92AF92BF92CF92DF92EF9228
:10099000FF920F931F93CF93DF9300D01F92CDB799
:1009A000DEB75C016B017A01122F0023E1F10E9496
:1009B000FF4D88E999E00E942C3861E0812F0E9468
:1009C000203A9090140583E08093140581E0809391
:1009D000230C0E94174082E080938D1140E368E869
:1009E00079E084E799E00E941C4040E069E171E110
:1009F0008DE699E00E941C4061E088E699E00E9443
:100A0000FE3F8AE799E00E9417228091230C8823F9
:100A100041F060E0812F0E94203A81E00E94075A55
:100A2000F4CF9092140520E030E0A901F501608137
:100A30007181828193810F947D25882371F080E0FC
:100A400090E0A0ECB0E489839A83AB83BC83BE01C1
:100A50006F5F7F4FC5010E94446820E030E0A9012C
:100A6000F60160817181828193810F947D258823B5
:100A700051F18090720C9090730CA090740CB09017
:100A8000750C80E090E0A0E7B1E48093720C909345
:100A9000730CA093740CB093750C80E090E0A0EA06
:100AA000B1E489839A83AB83BC83BE016F5F7F4FC0
:100AB000C6010E9444688092720C9092730CA092BE
:100AC000740CB092750C20E030E0A901F701608150
:100AD0007181828193810F94AD2E181674F480E099
:100AE00090E0A0E4B0E489839A83AB83BC83BE0129
:100AF0006F5F7F4FC7010E9444688091E90429E13C
:100B000031E1882311F029E439E047E559E061E655
:100B100079E081E00E943F400E94174081E00F9001
:100B20000F900F900F90DF91CF911F910F91FF9039
:100B3000EF90DF90CF90BF90AF909F908F900895EF
:100B4000CF93C82F8091E20B83FD14C08091FF08E2
:100B5000811110C080915F02909160029C01215030
:100B600031094091E9115091EA114217530714F4E9
:100B70000E94041FCC2329F061E080E0CF910C9407
:100B8000C3BC8091FF0891E0892780933C0280914B
:100B90003C02882389F08091E7119091E81120911F
:100BA000E9113091EA11821B930B97FF03C09195D5
:100BB00081959109029744F410923C028091E20BD6
:100BC00083FF06C0C1E01AC080E00E94075ADFCF51
:100BD000C091FF08C11112C080915F029091600224
:100BE00001972091E9113091EA112817390754F73C
:100BF0000E94FF4D8BE299E00E942C388C2FCF9100
:100C00000895AF92BF92CF92DF92EF92FF920F932F
:100C10001F93CF93DF93CDB7DEB764970FB6F894E9
:100C2000DEBF0FBECDBF0E94FE4E87FDAFC08AE57E
:100C30000E947C1E882309F4BAC040E050E0BA014B
:100C40008AE50E94AC247B018C0120912C0C309110
:100C50002D0C40912E0C50912F0C60E070E08BEE2B
:100C600093E40F944C2C5B016C019701A8010F9445
:100C7000AD2E181614F07501860120E030E0A901B0
:100C8000B701C8010F94AD2E181624F4E12CF12CF5
:100C900000E010E0B701C8010F94B92D072E000C39
:100CA000880B990B0F948425698B7A8B8B8B9C8B8B
:100CB00020E030E0A9010F947D25882321F0CE01AA
:100CC00041960E94C27280E090E0A0EAB1E48D8774
:100CD0009E87AF87B88B19861A861B861C868CE484
:100CE0000E942E1E882309F467C00E9482246B0193
:100CF0007C0120E030E0A901C701B6010F94AD2EC0
:100D000087FF04C0F7FAF094F7F8F094CD82DE8202
:100D1000EF82F8862091E9113091EA1124303105F3
:100D200074F08091E7119091E811821B930B97FF6B
:100D300003C091958195910901E004970CF400E0BE
:100D400080E00E94A085882359F022E0AE01435F35
:100D50005F4FBE016B5F7F4FCE0109960E94C18439
:100D600069897A898B899C898B019C013058098318
:100D70001A832B833C8320E030E0A9010F947D256A
:100D8000882321F0CE0101960E94C27264960FB6AC
:100D9000F894DEBF0FBECDBFDF91CF911F910F91B1
:100DA000FF90EF90DF90CF90BF90AF900895E12C2F
:100DB000F12C00E211E449CFC090C505D090C605E2
:100DC000E090C705F090C80594CF7F928F929F92D4
:100DD000AF92BF92CF92DF92EF92FF920F931F9349
:100DE000CF93DF9300D000D01F921F92CDB7DEB714
:100DF0006C015B014A01722E7801009112060E947B
:100E0000101F8091E9119091EA118E159F051CF435
:100E1000C7010E94041F80E00E94A085882331F052
:100E2000272DA401B501C6010E94C1841E141F0410
:100E30003CF4C7010E94041F60E080E00E94C3BC34
:100E400081E00E94A08580E090E0A0E7B2E4898381
:100E50009A83AB83BC8380E090E0A0E8B0EC8D8304
:100E60009E83AF83B887BE016F5F7F4FCE0105962B
:100E70000E94446887E00E94FD29811158C080913A
:100E80002C0C90912D0CA0912E0CB0912F0C409118
:100E9000EE045091EF046091F0047091F104C09061
:100EA000EA04D090EB04E090EC04F090ED04C092E2
:100EB0007007D0927107E0927207F0927307409327
:100EC0007407509375076093760770937707809344
:100ED000780790937907A0937A07B0937B0780E017
:100EE00090E0A8E4B2E489839A83AB83BC83CE010B
:100EF00001960E945B728091F2049091F304A0919C
:100F0000F404B091F5048093780790937907A09347
:100F10007A07B0937B0780E090E0A0EAB0E4898391
:100F20009A83AB83BC83CE0101960E945B72C12C75
:100F3000D12C80E7E82E82E4F82EC982DA82EB8297
:100F4000FC8280E090E0A0E8B0E48D839E83AF83D4
:100F5000B887BE016F5F7F4FCE0105960E9444683F
:100F600020E030E0A9016091F6047091F7048091CF
:100F7000F8049091F9040F947D2587FF0BC0C98276
:100F8000DA82EB82FC82BE016F5F7F4F86EF94E0D6
:100F90000E9444688091F6049091F704A091F804AF
:100FA000B091F9048093300C9093310CA093320CE3
:100FB000B093330C80937C0790937D07A0937E07BA
:100FC000B0937F078CE797E00E947C618091C90510
:100FD00081110E945FF761E087EB99E00E94673F13
:100FE00080911F11815080931F1146E658E16FEBED
:100FF00079E085E00E9434E380911F11882339F065
:101000000E94FCAA80911F11815080931F1180E0E3
:101010000E9426F90E947B3180912011823011F4C8
:101020000E943A380E94AFE428960FB6F894DEBFCB
:101030000FBECDBFDF91CF911F910F91FF90EF9029
:10104000DF90CF90BF90AF909F908F907F9008954A
:10105000CF92DF92EF92FF920F931F93CF93DF9384
:1010600000D01F92CDB7DEB77C016B018A0161E031
:101070008CE399E00E94673F46E658E163E479E03B
:1010800085E00E9434E390911F1181E0890F8093E5
:101090001F1180912D1482FF06C08B7F80932D1429
:1010A0009E5F90931F110E942C3980E1E4E2FCE0E6
:1010B000AAEEB4E001900D928A95E1F70E946B616F
:1010C00081E00E9426F920E030E0A901F70160816B
:1010D0007181828193810F947D258823F1F0809125
:1010E000FF0881110CC080915F029091600201970E
:1010F0002091E7113091E8112817390774F080E04A
:1011000090E0A0E7B2E489839A83AB83BC83BE01FD
:101110006F5F7F4FC7010E94446887E00E94FD29EE
:10112000811103C0B6010E94986720E030E0A90158
:10113000F80160817181828193810F947D258823DC
:1011400041F080E00E94A085882319F0C8010E9428
:101150007468129A64E670E080E090E00E94F025E6
:1011600081E00F900F900F900F90DF91CF911F9122
:101170000F91FF90EF90DF90CF900895CF92DF9284
:10118000EF92FF92CF93DF936B017C01D42FC0913C
:10119000140583E08093140581E08093230CC1142F
:1011A000D104E104F10431F00E9457FDC60ED71EB0
:1011B000E81EF91E8091230C882389F0C114D10404
:1011C000E104F10421F48D2F0E94075AF3CF0E940D
:1011D00057FD6C197D098E099F0997FDF4CF109278
:1011E000230CC0931405DF91CF91FF90EF90DF9017
:1011F000CF9008950F931F93CF93DF93C82F162F8F
:101200000E94FF4DC11194C0CFE8D8E0CE010E94EA
:101210002C3861E0812F0E94203A0E9457FD6853CC
:1012200070458F4F9F4F60930E0670930F0680930B
:10123000100690931106109212060091140583E097
:101240008093140530E020E049E151E16DE179E05F
:1012500082E00E943F408DE199E00E94172281E0E8
:101260008093230C8091230C882309F464C060E0F0
:10127000812F0E94203A80911206882309F454C0DD
:101280000E94FF4D83E099E00E942C3830E020E07E
:101290004DEE58E064EF78E082E00E943F4084EF3A
:1012A00098E00E94172241E060E070E0CB010E94CC
:1012B000BE8830E020E050E040E060EE78E085E07D
:1012C0000E943F4080EE98E00E9482350E94101FED
:1012D00080E00E94A0850E94FF4DCE010E942C3824
:1012E0000E9457FD685370458F4F9F4F60930E06C5
:1012F00070930F06809310069093110610921206B9
:1013000030E020E049E151E164ED78E082E00E94C4
:101310003F4083EC98E00E94172281E08093230CE9
:1013200061E0812F0E94203A81E00E94075A9ACF03
:10133000C4EAD8E06BCF00931405DF91CF911F91E1
:101340000F910895CF92DF92EF92FF920F931F9328
:10135000CF93DF93CDB7DEB7A0970FB6F894DEBF7B
:101360000FBECDBF0E94FE4E87FDCCC085E40E941B
:101370002E1E882309F4D5C00E9482246B017C01B3
:1013800020E030E0A9010F94AD2E87FF04C0F7FAEA
:10139000F094F7F8F094F7FAF094F7F8F094CD8E13
:1013A000DE8EEF8EF8A28CE0E6ECF2E0DE01119624
:1013B00001900D928A95E1F78AE50E947C1E8823B0
:1013C00051F040E050E0BA018AE50E94AC24698700
:1013D0007A878B879C8788E50E947C1E882351F042
:1013E00040E050E0BA0188E50E94AC2469837A832A
:1013F0008B839C8389E50E947C1E882351F040E00A
:1014000050E0BA0189E50E94AC246D837E838F830E
:10141000988785E50E942E1E882309F489C00E94C2
:1014200082246B017C0120E030E0A901C701B601F4
:101430000F94AD2E87FF04C0F7FAF094F7F8F094FC
:10144000F7FAF094F7F8F094C98EDA8EEB8EFC8EF2
:101450001D8A1E8A1F8A188E8CE40E942E1E8823E5
:1014600009F46FC00E9482246B017C0120E030E00F
:10147000A901C701B6010F94AD2E87FF04C0F7FA8A
:10148000F094F7F8F094C98ADA8AEB8AFC8A62E071
:1014900070E082E40E947324F82E80911F11811164
:1014A00031C021E0AE01475E5F4FBE016F5F7F4FED
:1014B000CE014D960E942888882321F16F2D81E06E
:1014C0000E94FA8882E50E947C1E882309F442C0AB
:1014D0000E946F2440E050E060EA71E44D875E872F
:1014E0006F87788B20911F11222361F08C012F2DA3
:1014F000AE01435F5F4FBE016F5E7F4FCE014596E9
:101500000E94E586A0960FB6F894DEBF0FBECDBF51
:10151000DF91CF911F910F91FF90EF90DF90CF90CF
:101520000895C12CD12C80E8E82E80E4F82E33CF2A
:10153000C090C105D090C205E090C305F090C405ED
:1015400072CFC090C505D090C605E090C705F09059
:10155000C8058CCF90E080E0BDCFCF92DF92EF92B4
:10156000FF920F931F93CF93DF93CDB7DEB76C97A6
:101570000FB6F894DEBF0FBECDBF8CE40E942E1EC6
:10158000882309F4B0C00E9482246B017C0120E012
:1015900030E0A9010F94AD2E87FF04C0F7FAF09454
:1015A000F7F8F094F7FAF094F7F8F094C98EDA8E21
:1015B000EB8EFC8E8CE0E6ECF2E0DE011196019001
:1015C0000D928A95E1F788E50E947C1E8823A1F0A0
:1015D00040E050E0BA0188E50E94AC242091CC089C
:1015E0003091CD084091CE085091CF080F944C2CEB
:1015F00069837A838B839C8389E50E947C1E882380
:10160000A1F040E050E0BA0189E50E94AC242091AD
:10161000CC083091CD084091CE085091CF080F945E
:101620004C2C6D837E838F8398878AE50E947C1E75
:10163000882351F040E050E0BA018AE50E94AC24D2
:1016400069877A878B879C871D861E861F86188AE6
:1016500080911F11811138C020E0AE01435F5F4FC0
:10166000BE016F5F7F4FCE0149960E942888882374
:1016700059F18091C90581110E945FF760E080E017
:101680000E94FA88898D9A8DAB8DBC8DB0588D8B58
:101690009E8BAF8BB88F198A1A8A1B8A1C8A1D866B
:1016A0001E861F86188A80911F11882369F010E01A
:1016B00000E020E0AE014B5E5F4FBE016F5E7F4FEA
:1016C000CE010D960E94E5866C960FB6F894DEBFAB
:1016D0000FBECDBFDF91CF911F910F91FF90EF9083
:1016E000DF90CF900895C12CD12C80E8E82E80E4C3
:1016F000F82E58CF2F923F924F925F926F927F9227
:101700008F929F92AF92BF92CF92DF92EF92FF9211
:101710000F931F93CF93DF93CDB7DEB7E5970FB647
:10172000F894DEBF0FBECDBF8DAB209114052CAB5E
:1017300021E020931405809132058D3409F405C60B
:10174000843511F40C94CDA0873409F091C18091B7
:101750003005909131058B31910509F4DDC108F018
:1017600079C18430910508F030C12091E5068230BE
:10177000910508F48EC1213009F091C111E0029762
:1017800009F010E00E94C32419821A821B821C8275
:101790001D821E821F82188682E50E947C1E88237D
:1017A00009F490C10E9482246B017C0120E030E0AA
:1017B000A9010F947D25882309F4EAC04090240CE8
:1017C0005090250C6090260C7090270C8091280C6E
:1017D0009091290CA0912A0CB0912B0C8CA79DA75D
:1017E000AEA7BFA78090700790907107A090720776
:1017F000B09073078091740790917507A091760758
:10180000B091770788AB99ABAAABBBABA5019401AC
:10181000C301B2010F947D2581110DC028A939A9FA
:101820004AA95BA96CA57DA58EA59FA50F947D25D2
:10183000882309F4ADC0A3019201C501B4010F943E
:101840004C2C20E030E040E05FE30F94E32568A7F4
:1018500079A78AA79BA72CA53DA54EA55FA568A93A
:1018600079A98AA99BA90F944C2C20E030E040E094
:101870005FE30F94E3252B013C0120E030E0A90158
:10188000C701B6010F947D25881F8827881F181768
:1018900009F40FC180E090E0A0E8BFEB8CA79DA702
:1018A000AEA7BFA728A539A54AA55BA5CA01B9015E
:1018B0000F94E3254B015C01A3019201C301B20126
:1018C0000F94E3259B01AC01C501B4010F944D2C8D
:1018D0000F94FB2E4B015C01AC019B01C701B601CB
:1018E0000F944C2C68AB79AB8AAB9BABA5019401F0
:1018F000C701B6010F944D2C9B01AC0168A979A9D1
:101900008AA99BA90F94E3256B017C0120E030E0BC
:10191000A9010F94AD2E87FDD1C0C701B6010F9468
:10192000FB2E6B017C01C301B2019058A50194010B
:101930000F94472D2CA53DA54EA55FA50F94E3253B
:10194000A70196010F94E32528A539A54AA55BA513
:101950000F944D2C69837A838B839C83A50194011A
:1019600068A579A58AA59BA50F94472D2CA53DA513
:101970004EA55FA50F94E325A70196010F94E325DB
:10198000A30192010F944D2C6D837E838F839887E2
:1019900020E030E0A90169817A818B819C810F94DC
:1019A0007D258111A3C020E030E0A9016D817E81F9
:1019B0008F8198850F947D25811198C00E94FB4DE1
:1019C0008BEB9FE00E942C386AC08531910509F4A9
:1019D00066C08A31910509F49CC0049709F048C09B
:1019E00080E50E947C1EC12CD12C7601882321F039
:1019F0000E94FC236B017C0183E50E947C1E8823EE
:101A000061F00E94822420E030E04AE754E40F9421
:101A1000E3250F94C02D6B017C010E946B618091C6
:101A20002111811105C060E081ED9FE00E949A3F85
:101A30000E9457FDC60ED71EE81EF91E0E9457FDD4
:101A40006C197D098E099F0997FF29C080E00E94CB
:101A5000075AF4CF8A32910509F4ECC260F48D3153
:101A6000910509F415C208F470C04E9709F468C2D4
:101A70000E9478F914C08B35910509F4BEC38C35EA
:101A8000910509F4BEC38A35910591F71092F007CC
:101A900006C0213021F40E94C3240E94A86F3DA9F2
:101AA000311102C00F9462148CA9809314050C9418
:101AB0002E9980E090E0A0E8BFE3F0CEC12CD12CBD
:101AC000760131CF89E40E947C1E882331F00E9488
:101AD000822469837A838B839C838AE40E947C1EA0
:101AE000882309F455CF0E9482244ECF412FBE0196
:101AF0006F5F7F4F80E797E00F94B5140E9457FD0A
:101B00006093721170937311809374119093751197
:101B1000C6CF0E949777C3CF87E00E940F4E8111F6
:101B2000BECF8CE0E2EDF2E0DE01119601900D9265
:101B30008A95E1F770E060E080E50E941C24BE0118
:101B40006F5F7F4F0E949867AACF87E00E94FD29B0
:101B5000811106C060E08FE40E945A2481119FCF5A
:101B60000E946B61109246026091350C8CE40E94D9
:101B70005A24E82E80E00E9404690E9457FD609379
:101B800072117093731180937411909375110E9468
:101B9000C31C81E08093A1060E94552B8AE50E9418
:101BA0002E1EF82E882369F081E00E94FD29182F4F
:101BB00082E00E94FD2911110C94F0A011E0811126
:101BC00001C010E088E50E942E1E81110C94E2A055
:101BD000111145C189E50E942E1E082F811307C0EF
:101BE000012FF11204C011E001E0FF24F39482E51B
:101BF0000E947C1E882309F435C10E9482246CA3B4
:101C00007DA38EA39FA320E030E0A9010F947D2542
